:080000000C94B9000C940000FF
:100008000C9400000C9400000C9400000C94000068
:100018000C9400000C9400000C9400000C94000058
:100028000C9400000C94E8000C9400000C94000060
:100038000C9400000C9400000C9400000C94000038
:100048000C944F010C9400000C941C010C940000BB
:100058000C9400000C9400000C9400000C94000018
:100068000C94325C0C9400000C9400000C9400007A
:100078000C9400001027E80364000A000100001037
:10008800000110000100000000000A000101010148
:1000980009001800010001000A0A0A0A0A0A0A0AE5
:1000A8000A0A0A0A0A0A0A0A01000A00D600010016
:1000B800FBFFFBFFFBFFFBFF2800E803000000003D
:1000C8000000000000000000000000000000000028
:1000D8000000000000000000000000000000000018
:1000E8000000000000000000000000000000000008
:1000F80000000000000000000000000000000000F8
:100108000700020002008E000200040090000100B7
:10011800080592000400E80594000100040798000F
:10012800010023079A00010025079C00010026070B
:100138009E0010002807A00001006907B000010018
:100148009507B2000100E707B40001002108B600D6
:1001580008008608B80001005209C00002005309CF
:10016800C2000100770908010000F894EE27EFBBF0
:10017800F1E0F5BFE5BF8DE0A2E0BB27ED938A95DE
:10018800E9F780E090E1A0E0B1E0ED930197E9F7AD
:10019800EAE0F1E085919591009761F0A591B5911C
:1001A80005901590BF01F00105900D920197E1F7B8
:1001B800FB01F0CFE4E0EEBBEFEFEDBFE0E1EEBF17
:1001C800C0E0D5E00C949C018A93AA93BA93EA9371
:1001D800FA93EFB7EA93E0E0E0937A00E0916B07D7
:1001E8000E94B55DAE0FBF1FE0917800F0917900D5
:1001F800ED93FC93E0916B07EF5FE0936B07A091A1
:100208006B07A83018F0E0E0E0936B07E0916B070C
:10021800E0937C0088E08A95F1F7E7ECE0937A00B8
:10022800E991EFBFF991E991B991A991899118954F
:10023800AA93EA93FA93EFB7EA931A930A93109161
:10024800C0000091C600E12FEC71E9F4E091720959
:10025800EF5FE0937209E150F0E0EF59F64F008349
:10026800A0917209A13119F4E0E0E0937209A0911C
:100278007409AF5FA0937409A13129F4E0E0E09319
:100288007409689432F809911991E991EFBFF991CD
:10029800E991A99118950A92AA93BA93EA93FA93C5
:1002A800EFB7EA93E0917D07F0917E073196E093EE
:1002B8007D07F0937E07A0917D07B0917E07A83B4C
:1002C800E0E0BE0719F4E1E0E0932D05A0917D0779
:1002D800B0917E07A037E1E0BE0741F4E2E0E09389
:1002E8002D05E0E0E0937D07E0937E070E94BB5D6B
:1002F8000E94C05D0E94BB5DE8EDF9E50E942C7785
:10030800E02149F0E091C707F091C8073196E093E2
:10031800C707F093C807E0912107EF5FE093210733
:10032800E991EFBFF991E991B991A99109901895CF
:10033800EF97249783E4A0E0B0E0E4ECF0E00E94BB
:100348007578FF2450E0E0E8E0936100E0E0E09396
:100358006100E1B9E2B9EAEFE4B9E5E0E5B9ECE357
:10036800E7B9E3ECE8B9E0EFEAB9ECE0EBB9E1EAC8
:10037800E4BDE3E0E5BDE0E0E6BD0E94C65DE1EA7C
:10038800E0938000E3E0E0938100E0E0E093850003
:10039800E0938400E0938700E0938600E09389006F
:1003A800E0938800E0938B00E0938A00E093B60026
:1003B800E1EAE093B000E2E0E093B100E0E0E0932E
:1003C800B200E093B300E093B400E1E0E0936E0084
:1003D800E0E0E0936F00E1E0E0937000E0E0E0939C
:1003E8006900EDBBE0936800E093C000E8E9E093A2
:1003F800C100E6E0E093C200E0E0E093C500EDE470
:10040800E093C400E0E0E093C900E0E8E0BFE0E08A
:10041800E0937F00E0937E00E0937C00E7EAE093BE
:100428007A00E0E0E0937B00ECBDA4E6B0E00E9437
:10043800965BE0E01A99E1E0E0931A057894299A2E
:10044800A4E60E94CA5D0E94CF5DA1E00E94C55B40
:10045800A0915A05A03861F40E94DE5DE0E0E093C7
:100468005C05E0E4E0935D050E94E45D0E94EB5DBD
:100478000E94F45DA0E00E94C55BA0E03799A1E06E
:100488000E94065EA0E03699A1E00E940B5EA09152
:100498005A05EFEF0E94F176E02909F453C10E9452
:1004A800DE5DE1E0E0935C05E2E3E0935D05E0E515
:1004B800E0935E05EEE1E0935F05E3E2E09360051B
:1004C800E2E3E0936105E4E60E94105EE2E3E09374
:1004D80064050E94165EE3E0E0936705E8EEE093AA
:1004E8006805E2E3E0936905E8ECE0936A05E2E376
:1004F800E0936B05EAE0E0936C05E0936D05E0930B
:100508006E05E1E0E0936F05E2E20E941C5EEAE01E
:100518000E94225EE6E9E0937505E9E0E09376053E
:10052800E4ECE0937705E3E0E0937805E4E80E94E3
:100538002A5EE6E9E0937B05E2E0E0937C05EEE7DE
:100548000E94305EE2E40E94365EE4EBE0938205AE
:10055800EAE0E0938305E1E0E0938405E2E00E94AD
:100568003E5EE0E0E0938805E4E6E09389050E94BA
:10057800465EE1E0E0938E05E0E0E0938F05E1E080
:100588000E94505EE4E20E945E5EE4E0E09399051A
:10059800E1E00E94665E0E946F5EE0935A05E6E421
:1005A800E0935B05E4EA0E947A5EE2E30E94845EDF
:1005B800EFEFE0936205E0936305EFE00E948A5E47
:1005C8000E948E5EE3E8E0936905E7E4E0936A053C
:1005D800E0E50E94945EE4E00E949E5EE0E00E94F6
:1005E800225EE0E0E0937505E3E0E0937605E8EE4F
:1005F800E0937705E0E0E09378050E942A5EE0E06A
:10060800E0937B05E0937C050E94305EE0E00E9469
:10061800365E0E94A25EEEE10E94AA5EE0E0E093F0
:100628008E05E6E9E0938F05E0E0E0939005E6E9C2
:10063800E0939105E0E0E0939205E0939305E4E60A
:10064800E0939405ECEFE09395050E94B05EECE32F
:100658000E94B75E0E94CA5DE0935A05E0E8E09305
:100668005B05E0E0E0935C05E1E0E0935D05EFE920
:10067800E0935E05E0E0E0935F05E1E00E94845EC0
:10068800E0E00E94105EE0E00E948A5EE4E6E0930B
:100698006705E0936805E2E3E0936905E0936A057E
:1006A800E0E00E94945EE0E00E949E5EE1E0E0935C
:1006B8007205E2E0E0937305E0E0E0937405E093EF
:1006C8007505E0937605EAE0E0937705E093780511
:1006D800E0E00E942A5EE0E0E0937B05EAE0E09338
:1006E8007C05E0E00E94305EE0E00E94365E0E94F9
:1006F800A25EE0E00E94AA5EE0E0E0938E05E0934F
:100708008F050E94505EE0E00E945E5EE0E0E093AC
:1007180099050E94665EE3E40E94B75E0E94C15E8E
:10072800E0935A05E0E0E0935B05E1E0E0935C05C7
:10073800E0935D050E94C65EE5E00E94B75EB0E00A
:100748000E94A774369950C0E0E0E0935A05EAE5A4
:100758000E94C95EE0E00E94845EE0E00E94105EB4
:10076800E3E0E0936405E8EE0E94165E0E948E5E68
:100778000E94CD5E0E94945EE0E00E949E5E0E9410
:10078800B05EE8E10E94B75E0E94CA5DE0935A0538
:10079800E2EA0E94C95EE0E00E94845EE0E00E9416
:1007A800105EE0E00E948A5E0E948E5E0E94CD5E2E
:1007B800E0936B05E0E0E0936C050E94B05EE3E136
:1007C8000E94B75E0E94CA5DE0935A05E9EB0E9459
:1007D800C95EE0E00E94845E0E94B05EE8E00E948C
:1007E800B75EB0E00E94A774189905C0689424F811
:1007F800E1E0E0935605689426F844E20E94D35E4F
:10080800E8ECF0E00E94DA5EE0EDF7E00E94DF5EDF
:10081800E8ECF0E0E0935C08F0935D080E94F45D7A
:10082800AFE30E94E45EEEA7E0915B05EC83E09104
:100838005C05ECA7E0915D05EAA7E0915E05E09311
:100848006007E0915F05E0936107E0916005E09340
:100858006207E0916105E9A7E0916205E8A7E091E8
:100868006305EBA3E0916405EF8FE0916505F0E087
:100878000E94E95EF0918707E0E00E94E95EE0915E
:100888006605F0E00E94EE5EEA0FFB1F0E94E95E3B
:10089800E0916705F0E00E94F35EE0916805F0E002
:1008A8000E94F85EE0916905F0E00E94FD5EE0912B
:1008B8006A05E0936507E0916B05E0936607E091B0
:1008C8006C05E0936707E0916D05F0E00E94025F18
:1008D800F091ED07E0E00E94025FE0916E05F0E024
:1008E8000E94075FEA0FFB1F0E94025FE0916F05FD
:1008F800E0931C05E0917005E0931E05E0917105F9
:10090800E0931D05A9EFB7E0E0917205F0E0ED93E3
:10091800FC93F091F907E0E0E093F907F093FA0708
:10092800A091F907B091FA07E0917305F0E0EA0F9A
:10093800FB1FE093F907F093FA07E0917405F0E0E4
:100948000E940C5FF091E907E0E00E940C5FE091E3
:100958007505F0E00E94115FEA0FFB1F0E940C5F13
:10096800E0917605F0E00E94165FF091F507E0E06F
:100978000E94165FE0917705F0E00E941B5FEA0F86
:10098800FB1F0E94165FABEFB7E0E0917805F0E03F
:10099800ED93FC93F091FB07E0E0E093FB07F09305
:1009A800FC07A091FB07B091FC07E0917905F0E006
:1009B800EA0FFB1FE093FB07F093FC07E0917A0531
:1009C800F0E00E94205FF0918B07E0E00E94205F3A
:1009D800E0917B05F0E00E94255FEA0FFB1F0E9473
:1009E800205FE0917C05FF27662777270E942A5F12
:1009F8000E94335FE8E00E94A9760E942A5FE09196
:100A08007D05F0E00E94335F0E943C5F0E942A5FF0
:100A1800E0917E05E0935405E0917F05F0E00E94A7
:100A2800415FF0919707E0E00E94415FE091800507
:100A3800F0E00E94465FEA0FFB1F0E94415FE091D1
:100A48008105E0930705E0918205E0930905E091AF
:100A58008305E0930A05E0918405E0930B05E09196
:100A68008505E0930C05E0918605E0930D05E0917E
:100A78008705E0936D07E0918805E0936E07E091A4
:100A88008905EB8FE0918A05EA8FE0918B05EF8B62
:100A9800E0918C05EE8BE0918D05ED8BE0918E0554
:100AA800EC8BE0918F05EB8BE0919005EA8BE09160
:100AB8009105F0E00E944B5FF0919F07E0E00E94F3
:100AC8004B5FE0919205F0E00E94505FEA0FFB1F38
:100AD8000E944B5FE0919305F0E00E94555FF09112
:100AE800AD07E0E00E94555FE0919405F0E00E94B8
:100AF8005A5FEA0FFB1F0E94555FE0919505E0934E
:100B08002007E0919605E0931505E0919705EC879D
:100B1800E0919805F0E00E945F5FF091F107E0E056
:100B28000E945F5FE0E0E0935805E6E40E94645F9E
:100B3800AAE30E94E45EF0E00E94735FEA0FFB1FE5
:100B48000E945F5FE0915B05E0933B05E0915C05E7
:100B5800E0933D05E0915D05E0934205E0915E0577
:100B6800EEA3E0915F05EAA3E0916005ECA3E091B4
:100B78006105EDA3E0916205E0931905E091630535
:100B8800FF27662777270E94785F0E94815F0E946F
:100B98008A5FE09164050E948E5F0E94915FE091F8
:100BA80065050E948E5F0E94915FE09166050E9434
:100BB8008E5F0E94785FE0916705E0934F05E091B2
:100BC8006805E0935005E0916905E0935105E091CF
:100BD8006A05E0935305E0916B05E0932F05E091DA
:100BE8006C05E0933305E0916D05E0933405E091E1
:100BF8006E05F0E00E94945FF091A107E0E00E948A
:100C0800945FE0916F05F0E00E94995FEA0FFB1F87
:100C18000E94945FA0912007A23098F0E09170059F
:100C2800F0E00E949E5FF0917F07E0E00E949E5FE7
:100C3800E0917105F0E00E94A35FEA0FFB1F0E949C
:100C48009E5FF698F198A09120070E94A85FA09156
:100C58002007E3E00E94F176E02921F0D0907205A8
:100C6800C0907305E0917405E0935009E091750513
:100C7800E0935109E0917605F0E00E94AD5FF091B4
:100C88005309E0E00E94AD5FE0917705F0E00E9433
:100C9800B25FEA0FFB1F0E94AD5FE0917805F0E0BC
:100CA8000E94B75FF0915509E0E00E94B75FE091BC
:100CB8007905F0E00E94BC5FEA0FFB1F0E94B75F56
:100CC800E0917A05F0E00E94C15FF091A808E0E0A9
:100CD8000E94C15FE0917B05F0E00E94C65FEA0FC9
:100CE800FB1F0E94C15FE0917C05F0E00E94CB5F92
:100CF800F0915709E0E00E94CB5FE0917D05F0E0BC
:100D08000E94D05FEA0FFB1F0E94CB5FE0917E0537
:100D1800F0E00E94D55FF0915909E0E00E94D55FAC
:100D2800E0917F05F0E00E94DA5FEA0FFB1F0E9466
:100D3800D55FE0918005F0E00E94DF5FF0915B09EC
:100D4800E0E00E94DF5FE0918105F0E00E94E45F4F
:100D5800EA0FFB1F0E94DF5FE0918205F0E00E942E
:100D6800E95FF0915D09E0E00E94E95FE0918305A9
:100D7800F0E00E94EE5FEA0FFB1F0E94E95FE0913E
:100D88008405E093F005E0918505E093BE05E091C8
:100D98008605E093F105E0918705E093F205E0917F
:100DA8008805E093F305E0918905E093F606E09164
:100DB8008A05E093F706E0918B05E093FB06ADEF1B
:100DC800B7E0E0918C05F0E0ED93FC93F091FD071E
:100DD800E0E0E093FD07F093FE07A091FD07B091D6
:100DE800FE07E0918D05F0E0EA0FFB1FE093FD0799
:100DF800F093FE07AFEFB7E0E0918E05F0E0ED93DA
:100E0800FC93F091FF07E0E0E093FF07F093000800
:100E1800A091FF07B0910008E0918F05F0E0EA0F7C
:100E2800FB1FE093FF07F0930008E0919005E09323
:100E3800FC0650919105E0919205E0930007E0913E
:100E48009305F0E00E94F35FE0E0E0935805E0E8E6
:100E58000E94645FAFE30E94E45EE0933505E09191
:100E68005B05F0E00E94F85FF091F307E0E00E9474
:100E7800F85FE0915C05F0E00E94FD5FEA0FFB1F60
:100E88000E94F85FE0915D05E093C805A091C80550
:100E9800A13061F4E0915E05E0932507F298A091F6
:100EA8002507A43019F4E1E0E0932507E0915F05F8
:100EB800E0933E05E0916005E0934305E09161050C
:100EC800E0933F05E0916205E0934405E0916305F6
:100ED800E98FE0916405E88FE0916505E0936F077D
:100EE800E0916605E0937007E0916705ED83E09176
:100EF8006805EE83E0916905E0930607E0916A05CD
:100F0800E0930707E0916B05E0930807E0916C0513
:100F1800E0930B07E0916D05E0933005E0916E05D5
:100F2800E0933105E0916F05E0930C07E0917005BF
:100F3800E0930E05E0917105E0930F05E0917205CD
:100F4800E0931005E0917305E0931105E0917405B5
:100F5800E0931205E0917505E0936307E09176054B
:100F6800E0936807E0917705E0934005E091780504
:100F7800E0934505E0917A05EF83E0917B05E093E6
:100F88003205E0917C05FF27662777270E940260DB
:100F98000E940B60E8E00E94A9760E940260E0913E
:100FA8007D05F0E00E940B600E943C5F0E94026099
:100FB8000E940B60E8E00E94A9760E940260E0911E
:100FC8007E05F0E00E940B600E943C5F0E94026078
:100FD800E0917F05F0E00E941460F091CF07E0E017
:100FE8000E941460E0918005F0E0A091CF07B091D5
:100FF800D007EA0FFB1F0E941460E0918105FF27CC
:10100800662777270E9419600E9422600E942B6041
:10101800E09182050E942F600E943260E091830572
:101028000E942F600E943260E09184050E942F6028
:101038000E941960E0918505FF27662777270E949F
:1010480035600E943E60E8E00E94A9760E94356003
:10105800E0918605F0E00E943E600E943C5F0E949D
:1010680035600E943E60E8E00E94A9760E943560E3
:10107800E0918705F0E00E943E600E943C5F0E947C
:101088003560E0918805FF27662777270E9447602B
:101098000E945060E8E00E94A9760E944760E091B3
:1010A8008905F0E00E9450600E943C5F0E94476002
:1010B8000E945060E8E00E94A9760E944760E09193
:1010C8008A05F0E00E9450600E943C5F0E944760E1
:1010D800E0918B05F0E00E945960F091A307E0E0F1
:1010E8000E945960E0918C05F0E00E945E60EA0F72
:1010F800FB1F0E945960E0918D05FF27662777271F
:101108000E9463600E946C60E8E00E94A9760E94D9
:101118006360E0918E05F0E00E946C600E943C5F85
:101128000E9463600E946C60E8E00E94A9760E94B9
:101138006360E0918F05F0E00E946C600E943C5F64
:101148000E946360E0919005FF27662777270E9439
:1011580075600E947E60E8E00E94A9760E94756032
:10116800E0919105F0E00E947E600E943C5F0E9441
:1011780075600E947E60E8E00E94A9760E94756012
:10118800E0919205F0E00E947E600E943C5F0E9420
:101198007560E0919305FF27662777270E9487608F
:1011A8000E949060E8E00E94A9760E948760E09122
:1011B8009405F0E00E9490600E943C5F0E94876066
:1011C8000E949060E8E00E94A9760E948760E09102
:1011D8009505F0E00E9490600E943C5F0E94876045
:1011E800E0919605FF27662777270E9499600E945D
:1011F800A260E8E00E94A9760E949960E0919705B4
:10120800F0E00E94AB600E9499600E94A260E8E052
:101218000E94A9760E949960E0919805F0E00E94EA
:10122800AB600E949960E1E0E0935805E0E00E941D
:10123800645FA3E00E94E45EE0937307E0915B05BE
:10124800E0937407E0915C05E0937507E0E0E093B4
:101258007607A091F606A43610F0E093F606A09162
:10126800F706A43618F0E0E0E093F706EC81E030EA
:1012780009F05CC0689431F8E1E0EEA7E9E1EC839D
:10128800E3E2E0936007E2E3E0936107E4E6E093DA
:101298006207E9EFF7E00E94AD60EBEFF7E00E942C
:1012A800AD60EDEFF7E00E94AD60EFEFF7E00E9470
:1012B800AD60EFE0E0931905ECE2F1E00E94025F17
:1012C800E4EFF1E00E945F5FE4E6E0930007ECEFF3
:1012D800F0E00E94F35FEEE7F2E00E94205FEEE1AB
:1012E800EAA7E3E1E0933505E4E6E8A7EEA3E4E046
:1012F800EC87E8EEF3E00E94E95EE3E8E0934F054F
:10130800E7E4E0935005E0E5E0935105E2E3F0E01F
:101318000E94F35EE8ECF0E00E94F85EE2E3F0E0A1
:101328000E94FD5EE4E2F0E00E94555F4A9912C017
:101338000E94B2600E94BB600E94C260E5E00E9409
:10134800B75E0E94D860E5E00E94B75E0E94C15E69
:10135800E0935505A0912507A13009F4F29AA091D0
:101368002507A23009F4F39AA0912507A33009F4C0
:10137800F49AAC85A43019F00E94FA6002C00E9469
:101388000861E0932205AAE00E94C15EE0932B0564
:101398000E941261E091F806F0E0AE0FBF1FE091E5
:1013A800F906F0E0AE0FBF1F0E94587814F4E1E090
:1013B80001C0E0E0E093FA06E1E07E2E0E941B61A6
:1013C8002D98A0912107AE30E0F3E0E0E0932107EB
:1013D8002D9AA0912D050E94A85FA0912D05E2E00D
:1013E8000E94F176E02909F493C5A13019F4E0E0F0
:1013F800E0932D05A0917B07B0917C07E5E0F0E034
:101408000E9432770E2EAC8DEEE00E940A77E02122
:1014180019F0EC8DEF5F03C023FC02C0E0E0EC8F15
:10142800AC8DAE3011F4689423F8A0911B05A1305F
:1014380029F4F69B02C0F69801C0F69AF79B02C001
:10144800F79801C0F79A0E942161E0E0F0E064E3B8
:1014580074E40E94F575E0930809F0930909609314
:101468000A0970930B090E942A610E9457750E940D
:1014780033610E943C610E9445610E94A7750E94E9
:101488004A610E9457750E9453610E942A610E9416
:101498005C6109F008F42BC0E091E808F091E908D4
:1014A8006091EA087091EB080E9463610E943361C1
:1014B800E0917F07F091800731960E949E5FE0914E
:1014C8008107F09182073196E0938107F0938207B4
:1014D8000E946A610E9473610E94785FE0918307AD
:1014E800F09184073196E0938307F09384070E9474
:1014F8004A610E945C6109F008F411C0E091340966
:10150800F091350960913609709137090E9463613D
:101518000E9453610E94786131960E941460E091A4
:101528008507F091860739960E94A35FEA17FB07A3
:10153800E8F4E0917F07F0918007E0938507F09346
:101548008607E0E00E947D61E6E00E94B75E0E94A7
:10155800CA5D0E9498610E94EB5DAAE00E94CA5D84
:101568000E94A6610E94EB5D0E94B0610E94B46176
:101578000E94C05D0E94B9610E94BE61E02161F1D4
:101588000E94C361A091EC08B091ED088091EE082B
:101598009091EF080E94F575E0931409F0931509EE
:1015A80060931609709317090E94CC61A3E9B7E00C
:1015B8000E94D561A0911409B0911509809116096E
:1015C800909117090E94DA61E0930009F0930109EC
:1015D80060930209709303090E94E161A091830757
:1015E800B0918407AE17BF0708F07AC00E943C612B
:1015F8000E94E661A0910009B09101098091020959
:10160800909103090E9450750E94ED610E945775E0
:10161800E093F408F093F5086093F6087093F708E0
:101628000E94CC610E94ED610E94F575A0E0B0E0D7
:1016380081E695E40E94A775A0E6B8E00E94F661ED
:101648000E943C61E091F808F091F9086091FA086D
:101658007091FB080E9450750E94FB610E94046211
:10166800A5E6B8E086EB9AE30E9450750E940D62E9
:101678000E940462A091F808B091F9088091FA08D4
:101688009091FB080E94F575A2E6B8E00E94F66109
:101698000E941662E3E6F0E00E9426770E2E0E9472
:1016A8001662E0E0F0E00E942077E029B9F0E3E676
:1016B800F0E0E0936208F0936308E0E0E093EC0860
:1016C800E093ED08E093EE08E093EF08E093F0086C
:1016D800E093F108E093F208E093F308689403C0FC
:1016E800E894F799689422F80E941B620E94246289
:1016F8000E942B620E9434620E943F620E945362E1
:101708000E945C62A0910709AA23DAF40E941B6276
:101718000E942462A0911809B091190980911A09B0
:1017280090911B090E9467620E943F62A091200964
:10173800B091210980912209909123090E94726237
:1017480012C00E941B620E9424620E947D620E9455
:1017580057750E9486620E943F620E948F620E94B3
:1017680057750E949862E1E0E0932707A091270748
:10177800AF3008F0EBC00E942B620E945C6109F058
:1017880008F417C00E94A1620E946361E0930C09EB
:10179800F0930D0960930E0970930F090E946C6015
:1017A8000E945C7834F40E94AA620E94B3620E948C
:1017B80063600E9453620E945C6109F008F417C0DC
:1017C8000E94B8620E946361E0931009F0931109C6
:1017D80060931209709313090E947E600E945C78DE
:1017E80034F40E94C1620E94B3620E947560A091A5
:1017F8000F09AA238AF40E94A1620E94CA620E9469
:1018080034620E946C600E94CF6234F40E94AA6223
:101818000E9473610E946360A0911309AA238AF44D
:101828000E94B8620E94CA620E945C620E947E6046
:101838000E94CF6234F40E94C1620E9473610E94C8
:101848007560A0911B09AA23CAF4E0911809F091C8
:10185800190960911A0970911B090E94CA620E94B5
:1018680067620E94995FAF3FEFEFBE0738F4E091DF
:10187800A107F091A20731960E94945FA0912309D5
:10188800AA23CAF4E0912009F09121096091220964
:10189800709123090E94CA620E9472620E945E606F
:1018A800AF3FEFEFBE0738F4E091A307F091A4072C
:1018B80031960E9459600E947D620E945C6109F025
:1018C80008F41DC0E0911C09F0911D0960911E09E2
:1018D80070911F090E9463610E9486620E943E60A7
:1018E8000E94CF6264F4E091C808F091C908609141
:1018F800CA087091CB080E9473610E9435600E94EB
:101908008F620E945C6109F008F41DC0E09124090F
:10191800F091250960912609709127090E94636159
:101928000E9498620E9450600E94CF6264F4E09125
:10193800CC08F091CD086091CE087091CF080E9434
:1019480073610E9447600E94D76210CF0E941B6299
:10195800E0E0F0E068EC72E40E94DD620E94DA6187
:101968000E94E2620E945775E0932809F0932909C2
:1019780060932A0970932B090E94B2600E94EB625F
:101988000E9468770E94E2620E941B750E943A7664
:1019980070F0E0E0E0932809E0932909E0932A0930
:1019A800E0932B090E94F06231960E944B5F0E94DF
:1019B800F5620E9466760E2E0E941B620E944561A7
:1019C8000E94FB620E942677E02151F1E091B8085D
:1019D800F091B9086091BA087091BB080E94EB6257
:1019E8000E949377DF01CB010E9405630E9444782F
:1019F8000E94F5750E940E630E9450750E9417633D
:101A08000E940E630E945775E0933809F0933909D4
:101A180060933A0970933B09AAE6B8E00E94F66120
:101A28000E94815FA038E6E9BE07E8E98E07E0E09A
:101A38009E0748F0E0E0E0933108E0933208E09335
:101A48003308E09334080E941E630E2EE091F806D6
:101A5800A091F6060E94F1760E22A091F706E09179
:101A6800F9060E94F176E02169F0A0911D07A330E4
:101A780030F4E0911D07EF5FE0931D0703C0E0E03D
:101A8800E093FA06AE8DAC3319F4E2E0E093FA067F
:101A9800A0912D05A23009F03BC2E0E0E0932D05AE
:101AA8000E9423630E9473610E9402600E94216168
:101AB8000E945C78A4F40E942C630E9422600E9419
:101AC80042780E945775A5E2B8E00E94E4740E942B
:101AD8002E780E9431630E9473610E9487600E9481
:101AE8009060E0E1FEE060E070E00E94B077E09393
:101AF8003D08F0933E0860933F08709340080E94A9
:101B08009060ECE3F0E060E070E00E94B0777F93D3
:101B18006F93FF93EF930E943A630E944363AF91E0
:101B2800BF918F919F910E947676A0933908B093C8
:101B38003A0880933B0890933C08E0913908F0916B
:101B48003A0860913B0870913C080E9443630E94E8
:101B580090600E9447780E9471767F936F93FF93FD
:101B6800EF930E943A63A0E1BEE080E090E00E941B
:101B78006877AF91BF918F919F910E947676A093DD
:101B88003508B093360880933708909338080E9438
:101B98004A630E2E0E94A2600E9451630E945877E9
:101BA800E02931F0EFA5F8A90E94AB600E94996086
:101BB800E0911908F0911A0860911B0870911C08AF
:101BC800A091CF07B091D007882799270E94627803
:101BD80021F10E94786166277727E0931908F0932E
:101BE8001A0860931B0870931C08E091A307F091F2
:101BF800A4070E9450600E9456630E9451630E948D
:101C08009377DF01CB010E947861662777270E94CE
:101C1800D577E093CD07F093CE07AF8D0E945B6335
:101C28000E94F5620E9438770E220E941E630E946D
:101C380060630E94656369F0EE8DEF5FEE8FEF8D54
:101C4800F0E03296AE8DB0E0EA17FB0711F4ECE352
:101C5800EE8FA0912607A33629F4E1E0EE8FE0E0AD
:101C6800E093FA06A394A0911405A13028F4E0911A
:101C78001405EF5FE09314050E946F63E8E5F2E056
:101C88000E942C770E2E0E94465F0E94BE610E2293
:101C9800A091FA060E940B5EA0911A050E94746337
:101CA80099F0E0919907F0919A073196E093990796
:101CB800F0939A070E946F630E947963EA1BFB0BFB
:101CC800E0939D07F0939E07ECE3EA1509F0E6C060
:101CD800AA24D394E091D907E17091F00E947E6321
:101CE800EE7F0E948363E0E6E0935B05E091500994
:101CF8000E948B63E3E00E94B75EB0E00E94A77485
:101D0800E091D907E27091F00E947E63ED7F0E9416
:101D18008363E1E6E0935B05E09151090E948B63E0
:101D2800E3E00E94B75EB0E00E94A774E091D90793
:101D3800E470A1F00E947E63EB7F0E948363EEE66D
:101D4800E0935B05E0915E09E0935C05E0915D0935
:101D58000E948E630E94EB5D0E94B061E091D907FA
:101D6800E870A1F00E947E63E77F0E948363E2E649
:101D7800E0935B05E0915409E0935C05E091530919
:101D88000E948E630E94EB5D0E94B061E091D907CA
:101D9800E071A1F00E947E63EF7E0E948363E4E617
:101DA800E0935B05E0915609E0935C05E0915509E5
:101DB8000E948E630E94EB5D0E94B061E091D9079A
:101DC800E072A1F00E947E63EF7D0E948363E8E6E3
:101DD800E0935B05E0915809E0935C05E0915709B1
:101DE8000E948E630E94EB5D0E94B061E091D9076A
:101DF800E074A1F00E947E63EF7B0E948363EAE6B1
:101E0800E0935B05E0915A09E0935C05E09159097C
:101E18000E948E630E94EB5D0E94B061E091D90739
:101E2800E078A1F00E947E63EF770E948363ECE67E
:101E3800E0935B05E0915C09E0935C05E0915B0948
:101E48000E948E630E94EB5D0E94B061E091DA0708
:101E5800E170D9F0E091DA07EE7FE093DA07E0E08D
:101E6800E0935A05E6E6E0935B05E091A808F09157
:101E7800A9080E94D776E0935C05E091A8080E9423
:101E88008E630E94EB5D0E94B061ECE3ED1531F4C6
:101E9800DD24C394E4E1EC1509F4CC24ED89E030A9
:101EA80019F4E0E0E0931605AD89A130C9F4E0919A
:101EB8001705EF5FE0931705A0911705A23080F092
:101EC800E0911605EF5FE0931605E0E0E093170553
:101ED800ED89A0911605EA1718F4E0E0E0931605DD
:101EE800AD89A23079F40E9491630E9496630E94A2
:101EF8009B630E94BE61E02911F0E0E001C0E1E0CF
:101F0800E0931605AD89A33019F4E1E0E0931605D6
:101F1800E8EC5E1648F45394EEE1E51529F40E94C6
:101F2800A163E0E0E09369070E94A7630E94D2766C
:101F38003B97A4F10E94A7630E94E776E0932D08DF
:101F4800F0932E0860932F08709330080E94AC63BA
:101F58000E94B1630E9468770E941B75AFE6B2E1E8
:101F680083E89AE30E94A7750E94BC63ADE2B8E0DB
:101F78000E94E4740E942E780E94C363ACEDB8E01E
:101F88000E94CC63E0910805EF5FE09308050E948A
:101F9800D16320F000912D0810912E08E0E03699C9
:101FA800E1E07E2EE091FA06E03059F4E0E04A994B
:101FB800E1E06E2E0E94D7638E2EE0E03799E1E0D3
:101FC800BE2EA091FA060E94A85F0E9412610E948C
:101FD8009663E02159F1E0E03699E1E0E093BF052E
:101FE800E0E04A99E1E0E093C0050E94D763E093FE
:101FF800C105E0E03799E1E0E093C205A091BF0593
:102008000E94065EA091C0050E94DF63A091C105F1
:102018000E94DF63A091C205E0E00E94F176E0290A
:1020280029F0E0E0E0931D07E0931E07A091FA066F
:10203800A23039F40E941B61E0E0E093F806E093D7
:10204800F906A091BF050E94065EA091C3050E94F3
:102058000B5EA9A10E94746389F0E1E0E093C305D7
:10206800E091F806E65FE093F806A091F806A4363A
:1020780028F0E091F806E456E093F806A091C00530
:102088000E94065EA091C4050E94746379F0E1E0A5
:10209800E093C405E091F806EF5FE093F806A0919D
:1020A800F806A43618F0E0E0E093F806A091C10520
:1020B8000E94065EA091C5050E94746389F0E1E064
:1020C800E093C505E091F906E65FE093F906A09173
:1020D800F906A43628F0E091F906E456E093F906EB
:1020E800A091C2050E94065EA091C6050E94746375
:1020F80079F0E1E0E093C605E091F906EF5FE0933F
:10210800F906A091F906A43618F0E0E0E093F90684
:10211800A091BF05A13019F4E0E0E093C305A091B8
:10212800C005A13019F4E0E0E093C405A091C10511
:10213800A13019F4E0E0E093C505A091C205A130F3
:1021480019F4E0E0E093C605E0914408F0914508F1
:102158000E94D2760E94E463E0914608F091470815
:102168000E94D2760E94E963E0911505E03009F0FB
:10217800CEC0EAE0E51509F048C00E94EE63749706
:102188000E949163AE17BF0710F4E1E0E88B0E944C
:10219800EE630E9491630E9432770E2E0E94F363D1
:1021A8000E9491630E942C77E02111F0E2E0E88B15
:1021B8000E94F36374960E94F86310F4E3E0E88BDE
:1021C8000E94FC6374970E940164AE17BF0710F465
:1021D800E1E0EF870E94FC630E9401640E9432776D
:1021E8000E2E0E9406640E9401640E942C77E02152
:1021F80011F0E2E0EF870E94066474960E94016481
:10220800EA17FB0710F4E3E0EF870E94EE63749788
:102218000E9491630E940B64A8890E94746311F064
:10222800E4E00CC00E94F36374960E9491630E94DC
:102238001464A8890E94746311F0E5E0E88B0E9499
:10224800FC6374970E9401640E940B64AF850E942E
:10225800746311F0E4E00CC00E94066474960E9456
:1022680001640E941464AF850E94746311F0E5E074
:10227800EF87A8890E945B63A8890E941D64C1F04A
:10228800EF85E03029F40E9422640E94E96302C0CD
:102298000E942764AC85A43028F4E8E2F0E00E94AC
:1022A800E46302C00E942D645C3511F40E94276427
:1022B800A8890E943364A8890E94386411F00E949A
:1022C8002764AF850E945B63AF850E941D6469F037
:1022D800E8E2F0E00E94E463A8890E945B63A889B1
:1022E8000E941D6411F00E942764AF850E94336428
:1022F800AF850E94386451F0AC85A43028F4ECE333
:10230800F0E00E94E46302C00E942D6403C0E0E094
:10231800E88BEF870E94EE630E94F86390F40E94B6
:102328003D640E9442640E9447640E943D640E948A
:10233800F363EA1BFB0BD0010E9498770E94E963C4
:1023480002C00E9427640E949163A93CE0E0BE0796
:1023580024F0E8ECF0E00E94E963E0914208E093A1
:1023680003070E94FC630E940164EA17FB0790F4CC
:102378000E944F640E9422640E9447640E944F6436
:102388000E940664EA1BFB0BD0010E9498770E940A
:10239800E46302C00E942D640E940164A93CE0E04D
:1023A800BE0710F00E9454640E945764A081A130B7
:1023B80030F10E945D64AFE6B2E183E09AE30E94E7
:1023C800DD620E9457640E9463640E94A7757F9330
:1023D8006F93FF93EF930E9457640E9463640E9477
:1023E8001763AF91BF918F919F910E946A640E9479
:1023F8006F640E9473640E94A7750E947964E091DB
:102408005405E03029F5AC85A330F0F4AFA5B8A9A0
:102418000E94587834F4EFA5F8A935960E947C6498
:1024280012C0A8A9AA2332F4EFA5F8A935970E94EB
:102438007C6409C0E0E0E0930409E0930509E093B7
:102448000609E093070904C0EFA5F8A90E947C6477
:10245800A0915405A130D9F50E948564A0EDB8E09B
:102468000E948A640E942E78A091D008B091D10869
:102478008091D2089091D308E0E0F0E060E874E43D
:102488000E94F575A0E0B0E48CE995E40E94A77578
:10249800DF01CB010E948F640E9494640E946A64E9
:1024A800DF01CB01E8EBFEE165ED70E40E94F57514
:1024B800DE019F960E94F661A0911405A13018F4E0
:1024C800E0E0EFA7E8ABEFA5F8A90E947C640E94C2
:1024D800D16330F0EFA5F8A9E0936608F093670898
:1024E800EE89E03009F09EC0A0914C08B0914D08EB
:1024F800A23DE1E0BE07F4F40E9485640E9499645D
:102508007F936F93FF93EF930E948564ED51F140A1
:10251800DF010E948564ED51F1400E94A364AF91F0
:10252800BF918F919F910E94AB64ACE6B8E00E9486
:10253800F66106C0E3E9F0E0E0936C08F0936D08FB
:102548000E94AD64E23DA1E0FA072CF50E94B86450
:102558000E94BD64FF93EF930E94AD640E9499644A
:102568007F936F93FF93EF930E94AD64ED51F14019
:102578000F010E94AD64ED51F140D0010E94A364A7
:10258800AF91BF918F919F910E94AB64AF91BF9122
:102598000E94E67409C00E94B864DF01AA0FBB1F3D
:1025A800A259B74FE3E9F0E0ED93FC930E94C564AC
:1025B800E23DA1E0FA072CF50E94B8640E94D064BD
:1025C800FF93EF930E94C5640E9499647F936F9371
:1025D800FF93EF930E94C564ED51F1400F010E94F3
:1025E800C564ED51F140D0010E94A364AF91BF9141
:1025F8008F919F910E94AB64AF91BF910E94E67446
:1026080009C00E94B864DF01AA0FBB1FA059B74FC9
:10261800E3E9F0E0ED93FC93EDEAFFEFE093B00817
:10262800F093B108AE89A13041F5A0914C08B09162
:102638004D0811960E94D864E0936C08F0936D08D9
:102648000E94B8640E94BD64BF010E94AD640E94EC
:10265800DD64DB01ED93FC930E94B8640E94D064B2
:10266800BF010E94C5640E94DD64DB01ED93FC9309
:10267800E0E0E093B008E093B1080E94B8643396B4
:10268800ACE6B8E0EE0FFF1FEA0FFB1FBF010E9488
:10269800E0640E9424780E94DD64DB01ED93FC93E2
:1026A800E0E0E0930F07E0931007A0914F05E3E8FF
:1026B8000E94E96409F458C0A0916E08B0916F08AF
:1026C8000E94F2641CF4E1E0E0930F07E0916E08C9
:1026D800F0916F080E94F9640E94016519F0E1E029
:1026E800E0931007A0917408B09175080E94F264F5
:1026F8001CF4E2E0E0930F07E0917408F09175088C
:102708000E94F9640E94086519F0E2E0E09310075E
:10271800A0917A08B0917B080E94F2641CF4E3E06F
:10272800E0930F07E0917A08F0917B080E94F96422
:102738000E940F6519F0E3E0E0931007A09180086C
:10274800B09181080E94F2641CF4E4E0E0930F0762
:10275800E0918008F09181080E94F9640E94166552
:1027680019F0E4E0E0931007A0915005E7E40E9417
:10277800E96409F458C0A0917008B09171080E94EA
:102788001D651CF4E5E0E0930F07E0917008F091F7
:1027980071080E94F9640E94016519F0E5E0E09370
:1027A8001007A0917608B09177080E941D651CF467
:1027B800E6E0E0930F07E0917608F09177080E9431
:1027C800F9640E94086519F0E6E0E0931007A0910B
:1027D8007C08B0917D080E941D651CF4E7E0E09339
:1027E8000F07E0917C08F0917D080E94F9640E942F
:1027F8000F6519F0E7E0E0931007A0918208B09107
:1028080083080E941D651CF4E8E0E0930F07E0913F
:102818008208F09183080E94F9640E94166519F0F5
:10282800E8E0E0931007A0915105E5E60E94E9640D
:1028380009F458C0A0917208B09173080E942465E9
:102848001CF4E9E0E0930F07E0917208F091730837
:102858000E94F9640E94016519F0E9E0E09310070D
:10286800A0917808B09179080E9424651CF4EAE0E8
:10287800E0930F07E0917808F09179080E94F964D5
:102888000E94086519F0EAE0E0931007A0917E081D
:10289800B0917F080E9424651CF4EBE0E0930F07D9
:1028A800E0917E08F0917F080E94F9640E940F650C
:1028B80019F0EBE0E0931007A0918408B091850827
:1028C8000E9424651CF4ECE0E0930F07E091840873
:1028D800F09185080E94F9640E94166519F0ECE0F1
:1028E800E09310070E94D16308F4B0C0E0916C082F
:1028F800F0916D08E0938608F0938708E8E8F8E01F
:102908000E942B65EAE8F8E00E942B65ECE8F8E005
:102918000E942B65A0916E08B0916F080E943065E7
:1029280034F4E0916E08F0916F080E943765A09129
:102938007408B09175080E94306534F4E091740809
:10294800F09175080E943765A0917A08B0917B08CC
:102958000E94306534F4E0917A08F0917B080E9477
:102968003765A0918008B09181080E94306534F4E1
:10297800E0918008F09181080E943765A091700865
:10298800B09171080E943C6534F4E0917008F091B0
:1029980071080E944365A0917608B09177080E945B
:1029A8003C6534F4E0917608F09177080E9443651D
:1029B800A0917C08B0917D080E943C6534F4E091B8
:1029C8007C08F0917D080E944365A0918208B0912F
:1029D80083080E943C6534F4E0918208F0918308F2
:1029E8000E944365A0917208B09173080E944865DF
:1029F80034F4E0917208F09173080E944F65A09139
:102A08007808B09179080E94486534F4E091780814
:102A1800F09179080E944F65A0917E08B0917F08D7
:102A28000E94486534F4E0917E08F0917F080E9486
:102A38004F65A0918408B09185080E94486534F4D8
:102A4800E0918408F09185080E944F65E091F005B7
:102A58000E9454650E942878A0E0B1E080E090E0F0
:102A68000E946877DF01CB01E091F005F0E0EE5DB0
:102A7800FA4FE081F0E00E943C5FA8EDB8E00E94C8
:102A8800CC630E945C65E0E0F0E66AEE76E40E94C2
:102A98003A7609F008F40AC00E946565A0E0B0E043
:102AA80080E897E40E9450750E946E65AC85A4305A
:102AB80061F50E945C65E0E0F0E060EA71E40E9484
:102AC800DD62EAA5F0E00E948A640E94F575E09351
:102AD8003009F093310960933209709333090E94E9
:102AE800255FE6E00E948877A8EDB8E00E94776548
:102AF8000E945C65E0E0F0E563EC77E40E94F57520
:102B08000E947B650E9484652FC00E9465650E94B3
:102B1800547831F4E0E0F0E86BE375E40E946E6508
:102B28000E945C65A030E0E8BE07EBE38E07E5E4B1
:102B38009E0789F00E946565A6E6B6E686E690E4FB
:102B48000E94F575DF01CB010E948F650E94946495
:102B58000E94846509C0E0E0E093D408E093D508BA
:102B6800E093D608E093D7080E94D16318F10E9439
:102B78002C63ACEAB8E00E94F6610E9494650E945A
:102B880096630E2E0E949465E0E0F0E00E942077A4
:102B9800E02911F0E5E001C0E0E0E0930D07E0E096
:102BA800E0930805E091B808F091B908E093AE0801
:102BB800F093AF080E949163E8ECF0E00E9414776C
:102BC8000E2EA091C905E2E30E940A77E021D1F018
:102BD800E091C905EF5FE093C905A091C905A2334B
:102BE80089F40E947B650E949965DF01CB010E94F0
:102BF800C3630E941B750E94F575A5E3B5E00E94AA
:102C0800E474EC93A09135050E94065EA091C90575
:102C1800E2E30E94F176E02119F0E0E0E093C905D3
:102C2800A09135050E945B63A091C9050E94746359
:102C380019F0E2E3E093C905E09104070E949D655D
:102C48000E9466760E94A4650E94F1760E220E9478
:102C5800A9650E220E94BB5D0E94BE61E021B9F009
:102C6800E0910407E65FE09304070E94AE653196A1
:102C78000E94B3650E94B865EA0FFB1FBF010E945E
:102C8800BE65DB01ED93FC93E2E3E093CA050E9485
:102C9800C5650E94CD650E220E94CF650E94D4654D
:102CA80071F1E1E0F0E0E093C707F093C807E3EBC8
:102CB800F7E00E94DA65E5EBF7E00E94DA65E7EBFA
:102CC800F7E00E94DA65E9EBF7E00E94DA65EBEBE2
:102CD800F7E00E94DA65EDEBF7E00E94DA65EFEBCA
:102CE800F7E00E94DA65E1ECF7E00E94DA65E3ECD0
:102CF800F7E00E94DA65E5ECF7E00E94DA650E94E9
:102D0800BB5D0E94C05D0E94DF650E94E86529F0F6
:102D1800E0E0E093C707E093C8070E94EA650E94D5
:102D2800587804F50E94C1620E94EB620E94937772
:102D3800DF01CB010E94EF650E94E7760E94D577FC
:102D4800A4EEB8E00E941D750E942E78E091E40878
:102D5800F091E5086091E6087091E708DE01D196E8
:102D68000E94F6610E94F4650E94B1630E94487750
:102D7800EF930E94F965E250F040604070400E9475
:102D88006C600E945077AF91EA230E2EA52DEEE1DC
:102D98000E94F176E02191F00E94F9650E94C260DC
:102DA800E5E00E94B75E0E94D860E5E00E94B75E49
:102DB8000E94CA5DE0937F07E0938007AB2D0E94D5
:102DC800065EA0E0F3FCA1E00E940B5E0E94FB659A
:102DD800E02199F1E4E1EA876894F3F8AC85A4303E
:102DE80011F40E94A163A0912507A13021F4F29863
:102DF800F39AE2E020C0A0912507A230A9F4F39845
:102E0800F49AA09162070E945B63A0916107E0E0D9
:102E18000E94F176E02911F0E3E003C0F498F29AF9
:102E2800E1E0E093250709C0A0912507A33029F424
:102E3800F498F29AE1E0E0932507AB2D0E94065E34
:102E48000E94FB650E220E94DF650E940166E02158
:102E580011F1A0910E07A03128F4E0910E07EF5F61
:102E6800E0930E07A0910E07AF30A9F4AC85A4300B
:102E780011F40E94A163E4E1EA87A0912507A43038
:102E880038F4E4E0E0932507F29AF398F49803C045
:102E9800E1E0E0932507E1E0EB1519F4E0E0E093C9
:102EA8000E07E0914208E0932C050E9409660E2E59
:102EB8000E94CD650E940F6609F444C00E94136603
:102EC800E081A0E4B9E00E9419660E9421660E9490
:102ED800E6610E942A660E942A66E0934009F09300
:102EE800410960934209709343090E942E66E0816C
:102EF800F0E00E9491630E948E770E9434660E94DF
:102F0800E9630E943A660E9473640E946A640E94A0
:102F180021660E94A775A0913C09B0913D09809156
:102F28003E0990913F090E945775E0933C09F09340
:102F38003D0960933E0970933F090E943A660E94DA
:102F4800796409C0E0E0E0933C09E0933D09E0932F
:102F58003E09E0933F090E9443660E944966E0816A
:102F6800A8E4B9E00E9419660E944366A081A130D6
:102F780049F40E944E660E9494640E9417630E945E
:102F88005A6606C00E945A66E0E0F0E068E472E41F
:102F98000E94F575E0934809F093490960934A093E
:102FA80070934B09AC85E2E00E940F770E2EA0913A
:102FB80025070E941D6409F4B5C00E94CD650E2E38
:102FC8000E946366ECE2F1E00E942C77E02151F068
:102FD800E0915F09F09160093196E0935F09F09301
:102FE800600902C00E946866E0910307A091020789
:102FF800AE1710F4E0930207E0910307A0910107D0
:10300800EA1710F4E09301070E942C63A091D307FC
:10301800B091D4070E946E6630F40E942C63A3ED31
:10302800B7E00E94D5610E942C63A091D107B091AE
:10303800D2070E946E6609F008F406C00E942C634D
:10304800A1EDB7E00E94D561A0910207BB27E091EE
:103058000107F0E0AE1BBF0BBD01A0910007E2E045
:10306800EA9FF001DB010E9426770E2EA09100074F
:10307800E4E60E940A77E0211E2EA091D107B091C4
:10308800D207E091D307F091D407EA1BFB0BDF01CD
:103098000E9475660E9432770E2E0E947A66EBEFC8
:1030A800F0E00E942C770E220E942161E0E0F0E01F
:1030B80060E87FE30E945A76E021E12991F00E94BE
:1030C8006866E0910307E0930207E09301070E9416
:1030D8002C63A1EDB7E00E94D561E093D307F0938C
:1030E800D4070E947F660E9460766E2FA0911D050E
:1030F8000E948266A0911D050E948B66EF930E9434
:103108007F660E9466766E2FA0911C050E948266DB
:10311800A0911C050E948B66AF91EA2B19F0E1E0A3
:10312800E0936A07A72D0E94065E0E94FB650E22A7
:10313800A0E0F0FCA1E00E940B5EA0916A070E944B
:10314800906609F443C0E0E0E0936A076894F0F8F9
:103158000E9468660E9495660E94547801F50E9454
:103168002C63A2EBB8E00E94F661E0E0E09344092A
:10317800E0934509E0934609E09347090E9491636B
:103188000E94587814F4E4E1E8870E944264ACE2B3
:10319800B9E00E949E66689420F8E894F4F8A0913B
:1031A800B408B091B5080E9496630E2E0E94F5628D
:1031B8000E94FB620E941477E02141F0E091B4087C
:1031C800F091B508E093B208F093B308AB89A13049
:1031D800E9F50E94CD650E2EA0912C05E0E50E9430
:1031E8000A770E94A2660E94AC660E94B3660E220D
:1031F800A0E0F4FCA1E00E94BB6631F00E94956655
:103208000E946F640E94C0660E940164E2E3F0E0DD
:103218000E94C966E0E5F0E00E942C770E94A26651
:103228000E94CC660E9466760E94B366E02171F027
:103238000E9495660E9463610E94C0660E94D166E2
:103248000E94D56619F0E3E00E94DB66AB89A230E4
:1032580009F04CC00E9421610E9445610E94DD6214
:103268000E94E26633960E948A640E946676EF9313
:103278000E94E766E0E0F0E060EA70E40E946676AB
:10328800AF91EA23EF930E942C630E94BC63DF0195
:10329800CB010E94E2660E948A640E946076EF93E6
:1032A8000E94E7660E94AC66AF91EA23AF91EA2BD1
:1032B800E9F0A091D708AA234AF00E942C630E9443
:1032C800FC660E9405670E94577508C00E942C631F
:1032D8000E94FC660E9405670E946A64E0934409A4
:1032E800F093450960934609709347090E94116756
:1032F8000E949B630E9417670E94A2660E94CC6688
:103308000E943877E02119F0E0E0EC8F05C0AC8D21
:10331800A23010F4E89423F80E941C670E945C789D
:103328003CF40E949566ABE7B7E00E94D56106C001
:103338000E944264E0937B07F0937C070E944264FA
:10334800309729F4E89420F86894F4F839C0A0E09C
:1033580020FCA1E00E94065E0E94CD650E22AB898A
:103368000E9474631E2E0E941C670E94CC660E94F5
:1033780066760E942567A0912C05EFE40E940F77DE
:103388000E22AB890E94BB661E2AA091B208B0919A
:10339800B308E0E0F0E00E941A770E9425670E94D7
:1033A8002B6771F00E94E266E093B408F093B508C9
:1033B8000E9432670E942764E89421F8689420F8F4
:1033C8004B9908C00E943267E89421F8689420F865
:1033D800E1E001C0E0E0E093FD06E09105050E9410
:1033E8009163F0E0EA17FB0724F4E0914208E093C8
:1033F80005050E944067EF930E947F660E946676EB
:10340800AF91EA230E2EA0911C050E940B5E0E942C
:10341800D566EF930E944067EF930E947F660E94F3
:103428006076AF91EA230E2EA0911D050E940B5ED7
:103438000E94D566AF91EA2B61F0E0914208E093D3
:1034480005050E94D1660E94486719F0E2E00E94D3
:10345800DB660E941C670E945C780CF043C021FC6C
:1034680003C0E1E0E0932B05689421F80E944264D0
:103478000E941C670E948A640E943A7690F10E941A
:1034880095660E947964AB89A23059F5A0914409E8
:10349800B09145098091460990914709E0E0F0E034
:1034A80068E473E40E943A7609F008F402C00E94C6
:1034B8004C670E9455670E941C670E9457750E94BE
:1034C8007964A0914308AA2362F4E1E0F0E00E9445
:1034D800E9630E941C670E9455670E9450750E940C
:1034E8004C6702C0E89421F80E945E670E946367F7
:1034F8000E22A0E025FCA1E00E940B5E0E94D5668A
:1035080031F0689425F80E9442640E94DA5E0E94B5
:103518005E670E946367E02161F10E9475670E94FF
:103528007D67A0F0A0912D08B0912E080E948567B4
:10353800EA1BFB0BA3E0B0E00E9460770E948A6759
:10354800AE1BBF0BA093B608B093B7080E9475676F
:103558000E945C7828F40E948F6732970E94DA5E96
:10356800A091B708AA232AF4E0E0E093B608E09314
:10357800B7080E945E670E94627860F50E949467AF
:103588000E947D6770F00E94075FE0912D08F0911E
:103598002E08EA1BFB0B0E948A67EA0FFB1F0E949A
:1035A800DA5E0E949467A230E0E0BE07E0E08E0792
:1035B800E0E09E0728F00E948F6731960E94DA5E4D
:1035C8000E948A67AB3FE0E0BE0724F0EAEFF0E034
:1035D8000E94DA5E0E948F670E9491630E942077A2
:1035E8000E2E0E94D56611F0E89425F80E948F6788
:1035F8000E9491630E9426770E2E0E94D56621F0C4
:103608000E948F670E94E9630E944E66AFA5B8A921
:103618000E9432770E2EA09157050E940B5E0E94E1
:10362800D56639F0E1E0E09357050E949E670E9455
:10363800DF5E0E944E66AFA5B8A9EA17FB0748F5FA
:103648000E944E660E94A467139770F00E944E660F
:103658000E94A467E4E0F0E00E94A967AE1BBF0BDC
:10366800A0935E08B0935F080E944E660E94A4670C
:103678000E94587828F40E94B06735970E94DF5E50
:10368800A0915F08AA232AF4E0E0E0935E08E093A3
:103698005F080E944E66AFA5B8A9AE17BF0750F5E0
:1036A8000E944E660E94B567149760F00E944E66AD
:1036B8000E94B567E5E0F0E00E94A967EA0FFB1FEA
:1036C8000E94DF5E0E944E660E94B5670E9458788D
:1036D80028F40E94B06735960E94DF5EA0915E08CC
:1036E800B0915F08A53CE9E0BE0724F0E4ECF9E0FE
:1036F8000E94DF5E0E949E67DF010E94B0670E9401
:1037080020770E2E0E94D56619F0E0E0E093570569
:103718000E949E67DF010E94B0670E9426770E2EE6
:103728000E94D56641F0A0915E08B0915F080E94A2
:10373800BB670E94E9630E94C0670E949D650E9462
:103748006676EF930E94C067F0E00E947B760E9445
:1037580021610E948A640E946076AF91EA2B11F081
:10376800689427F80E94C9670E9466760E2E0E9408
:103778001167E02911F0E89427F827FE6AC0A091A4
:10378800D708AA23A2F00E94C067F0E00E94216136
:103798000E94AB647F936F93FF93EF930E945A66E6
:1037A8000E949965AF91BF918F919F911DC00E9412
:1037B80005630E94B1747F936F93FF93EF930E9408
:1037C800C067F0E0AF91BF918F919F910E94AB6469
:1037D8007F936F93FF93EF930E945A660E949965B7
:1037E800AF91BF918F919F910E94A775A0914C09AD
:1037F800B0914D0980914E0990914F090E946A64D9
:10380800E0934C09F0934D0960934E0970934F096A
:10381800A0914F09AA234AF4E0E0E0934C09E09311
:103828004D09E0934E09E0934F090E94C9670E9431
:103838003A7609F008F402C00E94D367E0914C0977
:10384800F0914D0960914E0970914F090E94796479
:1038580002C00E94D367E2EAF8E00E94D767E4EA70
:10386800F8E00E94D767E6EAF8E00E94D767AC85DF
:10387800A43060F0E2EAF8E00E94DC67E4EAF8E0ED
:103888000E94DC67E6EAF8E00E94DC670E94E167D4
:103898000E94EB67A0914F05E3E80E940A77E021B8
:1038A80091F00E94E1670E94F167E093A208F0930B
:1038B800A308A091A208B091A308549724F4E2EABF
:1038C800F8E00E94DA650E94F6670E94EB67A09113
:1038D8005005E7E40E940A77E02191F00E94F6671C
:1038E8000E94F167E093A408F093A508A091A408AA
:1038F800B091A508549724F4E4EAF8E00E94DA6548
:103908000E9400680E94EB67A0915105E5E60E94BD
:103918000A77E02191F00E9400680E94F167E09325
:10392800A608F093A708A091A608B091A7085497F5
:1039380024F4E6EAF8E00E94DA65E091A208F09142
:10394800A3080E94F86334F4E091A208F091A30858
:103958000E94E963E091A408F091A5080E94F86329
:1039680034F4E091A408F091A5080E94E963E0917D
:10397800A608F091A7080E94F86334F4E091A6081D
:10398800F091A7080E94E963E09118050E949163ED
:10399800F0E0EA17FB0724F4E0914208E0931805E9
:1039A800E0911805F0E035970E9491630E94207716
:1039B8006E2F0E2EA0E025FCA1E00E94BB661E2EF5
:1039C800062EA09157050E94BB661E2A062EA0E06F
:1039D80027FCA1E00E94BB66E12961F0E091420862
:1039E800E09318050E94D1660E94D56619F0E2E0BE
:1039F8000E94DB66A0911F05A13078F00E94276421
:103A0800A0911F05A13021F4EAE0F0E00E94E963EB
:103A1800E0911F05E150E0931F050E940A68AB89F9
:103A28000E9474631E2E0E940164EEE1F0E00E9481
:103A380032770E2EAB89E1E00E94F1760E94B366E0
:103A4800E0211E2A0E940A68AB890E940D680E9424
:103A580048671E2A0E940A680E942B67A9F0E0E0C6
:103A6800E09306050E941C670E945C781CF4E2E063
:103A7800E0931F05E0E0E0932C09E0932D09E09323
:103A88002E09E0932F0902C00E942D640E9442640F
:103A9800E093EF07F093F0070E940A68AA8D0E944E
:103AA800BB6611F02C9A01C02C980E940A68A0915C
:103AB800FD060E94906611F0E3E001C0E0E0E093AB
:103AC8004605A72D0E94065E0E94FB65E02121F0B5
:103AD800E091E307E0935205A0915205A130A8F0C8
:103AE800E09152050E940164F0E0EA17FB0728F014
:103AF800E0915205F0E00E94E4630E9491630E9405
:103B080058781CF4E0E0E0935205A0911E07AF3FFF
:103B180028F4E0911E07EF5FE0931E07A72D0E948F
:103B2800065E0E9412680E9411670E220E940966B2
:103B38000E220E94DF650E9401660E22A091FA06FD
:103B48000E940B5E0E9412610E949663E0211E2E65
:103B5800A0911E07E8EC0E9419680E94F6760E22D2
:103B68000E9411670E220E9409660E220E94DF65DC
:103B78000E9401660E22A091FA060E940D680E941A
:103B880012610E949663E021E12969F0AD8DAF3F93
:103B980018F4ED8DEF5FED8FAD8DA43119F4E2E0EF
:103BA800E093FA0602C0E0E0ED8FA0914808B091DA
:103BB800490815960E94A7630E9420770E2EA091AF
:103BC8001A050E94BB6681F0E0919507F09196076F
:103BD8003197E0939507F0939607309721F499244D
:103BE800E0E0E0931F071FC0EAE0F0E0E0939507EC
:103BF800F0939607A0911A05A13019F4E0E0E0933C
:103C08001E07A091FA06E0E00E94F6760E2EA0911B
:103C18001F070E94746339F0E1E0E0931F07E09307
:103C2800FA06E0E0ED8FA92DE0E00E94F1766E2F14
:103C38000E2EA0E0F099A1E00E940D680E941E637C
:103C48000E22A52FEDE50E94F6760E9460630E9481
:103C5800F1760E940F661E2E062EA0E0F099A1E0D4
:103C68000E940D680E941E630E9460630E94656343
:103C78001E2A0E9479630E946F630E9414770E2E99
:103C88000E941E630E220E94465F0E94BE61E021D0
:103C9800E12909F40BC1F09B09C1F098E0E00E940A
:103CA80098610E94EB5DAAE00E94CA5DE0935A0504
:103CB800E7E3E0935B05E091A007E0935C05E09102
:103CC8009F070E948E630E94EB5DAAE00E94CA5D76
:103CD8000E947D61E6E00E94B75E0E94CA5D0E9474
:103CE800A6610E94EB5DAAE00E94CA5DE0935A05B6
:103CF800EAE5E0935B05E091A207E0935C05E091BB
:103D0800A1070E948E630E94EB5DAAE00E94CA5D33
:103D1800E0935A05E4E8E0935B05E09125070E94EB
:103D28008B63E3E00E94B75E0E94CA5DE0935A0588
:103D3800E2EAE0935B050E9423630E94DC76E0934D
:103D48005C050E940B60E8E00E94C176E0935D0587
:103D5800E0911D08E0935E05E091D007E0935F05D0
:103D6800E091CF07E09360050E942260E8E10E949D
:103D7800C176E0936105E0912508F09126086091ED
:103D88002708709128080E94DC76E09362050E945B
:103D98002260E8E00E94C176E0936305E09125087F
:103DA800E09364050E943E60E0E10E94B576E093EE
:103DB80065050E943E60E8E00E94B576E0936605DE
:103DC800E091C808E09367050E945060E0E10E9416
:103DD800B576E09368050E945060E8E00E94B576E9
:103DE800E0936905E091CC08E0936A05E091A407A7
:103DF800E0936B05E091A307E0936C050E946C606B
:103E0800E0E10E94B576E0936D050E946C60E8E001
:103E18000E94B576E0936E05E091C008E0936F05C7
:103E28000E947E60E0E10E94B576E09370050E94F2
:103E38007E60E8E00E94B576E0937105E091C408E1
:103E4800E09372050E9431630E94DC76E09373056B
:103E58000E949060E8E00E94C176E0937405E091CA
:103E68002108E0937505E0912908F0912A086091EE
:103E78002B0870912C080E94DC76E09376050E944E
:103E8800A260E8E00E94C176E0937705E0912908F6
:103E9800E09378050E94B05EEFE10E941C68A4E6FA
:103EA800B0E00E94A774E2E3E0933705A82D0E94D2
:103EB800A85F0E94FB65E02139F0E894F2F8E0E0A1
:103EC800E0935605E0932905A82D0E94065EA0916F
:103ED80056050E940B5E0E94FB65E02171F0E0919F
:103EE8002905EF5FE0932905A0912905AA3029F457
:103EF800E0E0E0932905E0931B05A82D0E94065EEB
:103F0800A09156050E940B5EA0E0F2FCA1E00E9481
:103F18000B5E0E94FB65E021E1F1E4E1E98768942A
:103F2800F2F8E0911B05EF5FE0931B050E942468FF
:103F3800A0E0F0FCA1E00E94746319F0E1E0E093D6
:103F48001B05A0911B050E943364A0E0F0FCA1E0D2
:103F58000E94746319F0E2E0E0931B050E94246854
:103F6800AA8D0E940B5EAC85E3E00E94F676E02104
:103F780019F0E1E0E0931B05A0911B050E94336452
:103F8800A0E0F0FCA1E00E94BB6619F0E3E0E0933A
:103F98001B05E091FA06E03009F0CBC1E0E0E093C0
:103FA8004705E09348050E942B68E093FF06E091DF
:103FB8001B05E030B1F4F6980E942F680E22AA8DF6
:103FC8000E94386411F00E94C65DA0913B050E94D2
:103FD8005B630E94386811F00E943F68E0E0E98B5B
:103FE80062C0A0911B05A130E9F4A0913B05A33064
:103FF80010F40E943F68A0913B05A33019F4EBA18F
:10400800E09347050E944468E02121F00E94476838
:10401800E0E0E8BDAA8DA53021F40E944768EFEFE3
:10402800E8BD41C0A0911B05A230F1F4F69AA09119
:104038003B05A33010F40E943F68A0913B05A330D4
:1040480019F4ECA1E09347050E944468E02121F0AF
:104058000E944768E0E0E8BDAA8DA53021F40E94DF
:104068004768EFEFE8BD1FC0A0911B05A330D9F446
:10407800F69AA0913B05A33018F4E091F10501C030
:10408800EFEFE0934705EFEFE09348050E9444689F
:10409800E02119F0EFEFE7BDE8BDAA8DA53019F4CE
:1040A800EFEFE7BDE8BDA09146050E945168A091D9
:1040B8003B05E1E00E940F770E220E94386819F054
:1040C800EFEFE09347050E9456680E945A6829F06E
:1040D8000E943F68E1E0E093FE060E9461680E944A
:1040E8005A6811F00E9464680E9456680E946B68C2
:1040F80029F00E943F68E0E0E093FE060E946168B4
:104108000E946B6811F00E9472680E9456680E94B3
:10411800796829F00E943F68E1E0E093FE060E947A
:1041280061680E94796811F00E9472680E9456685E
:104138000E94806831F00E943F680E942B68E093DB
:1041480038050E9461680E94806841F00E94646896
:10415800A0913805AA3010F40E9487680E9456681A
:104168000E94906851F0A0911B05A13010F00E94A8
:104178003F680E942B68E09338050E9461680E949E
:10418800906841F00E946468A0913805AA3010F444
:104198000E9487680E949768EC91E0938A00E98DF5
:1041A800E03019F4E0E0E093B400A98DA13019F4EF
:1041B800EFEFE093B400E88DE03009F41598A88D8E
:1041C800A13009F4159AA88D0E94A85F0E949F68E3
:1041D800E4E6F0E00E942077E02111F0EFEFE7BD80
:1041E8000E94CD650E949B630E94BE610E220E94C0
:1041F80048671E2E0E9411670E949B630E941767E2
:104208000E22A72D0E940B5E0E9412680E94F56282
:104218000E9466760E22AA8D0E9474631E2AA091BF
:10422800FD060E94A85F0E94CD65E0211E2AA88D88
:104238000E94A85F0E949F68ECE2F1E00E9420774C
:104248000E220E949F68E4E6F0E00E942677E021B3
:10425800E12909F443C0A091FD06A13011F40E94A0
:104268002764AB8DA13019F4EFEFE0938800E0915B
:104278000405EF5FE0930405AB8DA33031F4E270E1
:10428800AFEFEA02F001E0938800A0910405E5E0B1
:104298000E940F770E2E0E94A468C1F0AA8DA33049
:1042A80011F40E94A968AA8DA43029F40E94A96873
:1042B8000E94B168E8BD0E94B168E0938A00AB8DA6
:1042C800A23021F40E94B168E0938800A09104050F
:1042D800A03118F0E0E0E09304052AC0E5E0E0939F
:1042E8000405E0E0E0938800A0E024FCA1E00E943F
:1042F800A85FA0911B050E947463D1F0E091280586
:10430800EF5FE0932805A0912805A13019F4EFEF9D
:10431800E0938A00A0912805A33019F4E0E0E09327
:104328008A00A0912805A43019F4E0E0E09328055C
:1043380007C00E94C65DE0E0E0938800E0938A0031
:10434800A091FA06A23008F07EC00E94B86835979E
:10435800EA17FB07F0F1A0915209A83230F4E09176
:104368005209EF5FE09352092CC0E091B300A8A571
:104378000E9419680E940A77E02161F0A091B300B9
:10438800E8A50E94C1680E946F640E94C668EA0F8F
:10439800A02DEC93E091B300A8A50E940A770E9493
:1043A800A4650E940A77E02161F0E091B300A8A516
:1043B8000E94C1680E946F640E94C668EA1BA02D13
:1043C800EC930E94D16819F0E8A5E093B3006894D3
:1043D800F6F80E94B8683596EA17FB0798F5E0E00A
:1043E800E0935209E091B300AEA10E9419680E94BF
:1043F8000A77E02151F0A091B300EEA10E94DD6898
:104408000E94C668EA0FA02DEC93E091B300AEA11C
:104418000E940A770E94A4650E940A77E02151F061
:10442800E091B300AEA10E94DD680E94C668EA1B55
:10443800A02DEC930E94D16819F0EEA1E093B3008F
:10444800E894F6F806C0E0E0E093B300E8E2E09311
:104458005209E1E0E61529F4E894F1F8E0E0E09388
:104468005505A62D0E94065EA09155050E940B5E7B
:10447800A0E0F1FCA1E00E940B5E0E94FB65E02138
:1044880049F16894F1F8E0911305EF5FE0931305A3
:10449800E0E0EE87AE85A53088F40E94E868A08148
:1044A800A13018F0E5E0EE8705C0E0911305EF5F55
:1044B800E0931305EE85EF5FEE87ECCFA09113052F
:1044C800A53018F0E0E0E09313050E94E868E08169
:1044D800E0932607A62D0E94065EA8A1EFEF0E9492
:1044E8000A77E02121F0E8A1EF5FE8A309C0A8A1BD
:1044F800A13030F0E894F1F8E0E0E8A3E0932B0570
:10450800A8A1A53119F4E1E0E0932B05A8A1A431F5
:1045180009F071C2A52FE0E00E9405770E94A4650A
:104528000E940A77E02129F05150E091CF05E093ED
:104538003905A0912607A33620F4E3E6E093260781
:104548005AC2E1E0E0932607E0E0E09313050E94F9
:10455800DE5DEEA5E0935C05EC81E0935D05ECA5DE
:10456800E0935E05EAA5E0935F05E0916007E093BC
:104578006005E0916107E0936105E0916207E093CF
:104588006205E9A5E0936305E8A5E0936405EBA15E
:10459800E0936505EF8DE0936605E0918807E09369
:1045A8006705E0918707E0936805E0917707E09356
:1045B8006905E0917907E0936A05E091E507E093E2
:1045C8006B05E0916507E0936C05E0916607E09361
:1045D8006D05E0916707E0936E05E091EE07E093C3
:1045E8006F05E091ED07E0937005E0911C05E093FD
:1045F8007105E0911E05E0937205E0911D05E093B9
:104608007305E091FA07E0937405E091F907E093E8
:104618007505E091EA07E0937605E091E907E093F4
:104628007705E091F607E0937805E091F507E093C8
:104638007905E091FC07E0937A05E091FB07E093A8
:104648007B05E0918C07E0937C05E0918B07E09374
:104658007D050E94335FE8E00E94C176E0937E0505
:10466800E0910508E0937F05E0915405E09380050B
:10467800E0919807E0938105E0919707E093820520
:10468800E0910705E0938305E0910905E09384052F
:10469800E0910A05E0938505E0910B05E093860516
:1046A800E0910C05E0938705E0910D05E0938805FE
:1046B800E0916D07E0938905E0916E07E0938A0524
:1046C800EB8DE0938B05EA8DE0938C05EF89E09301
:1046D8008D05EE89E0938E05ED89E0938F05EC89D1
:1046E800E0939005EB89E0939105EA89E0939205C0
:1046F800E091A007E0939305E0919F07E09394056C
:10470800E091AE07E0939505E091AD07E09396053B
:10471800E0912007E0939705E0911505E09398054F
:10472800EC85E0939905E091F2070E94665E0E948D
:104738006F5EE0935A05E6E4E0935B05E091F107CC
:10474800E0935C05E0913B05E0935D05E0913D0554
:10475800E0935E05E0914205E0935F05EEA1E093EA
:104768006005EAA1E0936105ECA1E0936205EDA183
:10477800E0936305E0911905E09364050E94815F69
:10478800E8E10E94C176E09365050E946A610E9493
:10479800DC76E09366050E94815FE8E00E94C176BE
:1047A800E0936705E0913108E0936805E0914F05D3
:1047B800E0936905E0915005E0936A05E0915105A1
:1047C800E0936B05E0915305E0936C05E0912F05AC
:1047D800E0936D05E0913305E0936E05E0913405B3
:1047E800E0936F050E94B05EE6E10E94B75E0E940A
:1047F800CA5DE0935A05E0E7E0935B05E091F005B8
:10480800E0935C05E091BE05E0935D05E091F1055C
:10481800E0935E05E091F205E0935F05E091F30512
:10482800E0936005E091F606E0936105E091F706F4
:10483800E0936205E091FB06E0936305E091FE07D3
:10484800E0936405E091FD07E0936505E0910008B9
:10485800E0936605E091FF07E0936705E091FC06A9
:10486800E093680550936905E0910007E0936A05B5
:10487800E091D507E0936B050E94B05EE2E10E94EB
:10488800B75E0E94CA5DE0935A05E0E8E0935B05D5
:10489800E0913505E0935C05E091F407E0935D0550
:1048A800E091F307E0935E05E091C805E0935F05AA
:1048B8000E94B05EE6E00E94B75E0E94CA5DE09387
:1048C8005A05E5E8E0935B05E0913E05E0935C0559
:1048D800E0914305E0935D05E0913F05E0935E05B7
:1048E800E0914405E0935F05E98DE0936005E88D6C
:1048F800E0936105E0916F07E0936205E09170072E
:10490800E0936305ED81E0936405EE81E09365052E
:10491800E0910607E0936605E0910707E0936705D5
:10492800E0910807E0936805E0910B07E0936905BB
:10493800E0913005E0936A05E0913105E0936B055D
:10494800E0910C07E0936C05E0910E05E0936D058E
:10495800E0910F05E0936E05E0911005E0936F0577
:10496800E0911105E0937005E0911205E09371055F
:10497800E0916307E0937205E0916807E09373059F
:10498800E0914005E0937405E0914505E0937505D5
:10499800EF81E0937705E0913205E09378050E9476
:1049A800B05EEFE10E94B75E0E94C15EE0935A05D7
:1049B800E0E0E0935B05E0917307E0935C05E0912C
:1049C8007407E0935D05E09175070E94C65EE5E017
:1049D8000E94B75E0E94C15E4E2EE0E0E09336056D
:1049E800A52FE8E30E94F1760E2E0E94F36819F0D5
:1049F800E1E0E0933A05A62D0E94065EA0E0F1FCF6
:104A0800A1E00E940B5EA52FE4E60E9400770E94B9
:104A180060630E94F176E02131F06894F1F85F5FFD
:104A2800543609F450E0E1E0E71511F4E894F0F8A1
:104A3800A72D0E94065EA0E0F0FCA1E00E940B5E9C
:104A4800A52FE0E00E94FB760E9460630E94F17649
:104A5800E02131F06894F0F851505F3F09F453E6D3
:104A6800AB2D0E94065E0E94F668C1F00E94FD68A8
:104A7800A9F4A0912605A43119F4E7E0E0932605EE
:104A8800E0E0E0932705E894F3F8A0912605A33029
:104A980028F0E0912605E150E0932605A82D0E9414
:104AA800065E0E94F668C1F00E94FD68A9F4A09114
:104AB8002605A43119F4E7E0E0932605E0E0E09349
:104AC8002705E894F2F8A0912605A33028F0E09194
:104AD8002605E150E0932605A82D0E94A85FAB2D7E
:104AE8000E94BB6631F0E0E0E0932705E4E1E09343
:104AF8002605AB2D0E94A85FA0E0F3FCA1E00E9470
:104B0800BB6629F0E894F3F8E0E0E0932B05AB2DC1
:104B18000E94065EA0E0F3FCA1E00E940B5E0E94EA
:104B2800F66809F430C5E1E0E0932B056894F3F8E2
:104B3800503049F4A881A43030F4E881EF5FE8836D
:104B4800E0E0E0932B05513049F4AEA5A13030F4F4
:104B5800EEA5EF5FEEA7E0E0E0932B05523041F4BD
:104B68000E940869AF3520F40E94C0670E9411694D
:104B7800533049F40E941769A83C28F40E941E6922
:104B8800EB5F0E942569543041F40E942A69AF30D6
:104B980020F40E9431690E941169553049F40E943D
:104BA8002E66A081A43620F40E9438690E941169FB
:104BB800563071F40E944E66E43FA1E0FA0740F4D3
:104BC8000E943F693A96FE93EE93E0E0E0932B054E
:104BD800573061F4A0911905A83C40F4E0911905FB
:104BE800EF5FE0931905E0E0E0932B05583061F49E
:104BF800A0913305A13040F4E0913305EF5FE093D5
:104C08003305E0E0E0932B05593049F40E94136620
:104C1800A081AA3020F40E944B690E9411695A3081
:104C280049F40E944366A081A33020F40E9452698F
:104C38000E9411695B3039F40E94596920F40E947E
:104C480061690E9411695C3099F40E945A5FA43628
:104C5800E0E0BE0768F40E94686931960E946D69B9
:104C68000E947A690E947C690E9485690E948A690B
:104C78005D3071F40E94EE5EA43CE9E0BE0740F4AA
:104C88000E94AC6331960E94E95EE0E0E0932B0558
:104C98005E3079F40E9491690E94075FAE17BF07E2
:104CA80040F40E94856731960E94025FE0E0E0933D
:104CB8002B055F30A9F40E947A69A6E6B6E68EE372
:104CC80091E40E94A7750E94735F0E946E6640F48B
:104CD8000E94856931960E945F5FE0E0E0932B05B2
:104CE800503171F40E944F64AF3FE0E0BE0740F4DA
:104CF8000E94FC6331960E94FD5EE0E0E0932B0584
:104D0800513171F40E943D64AF3FE0E0BE0740F4CA
:104D18000E94EE6331960E94F35EE0E0E0932B057B
:104D2800523171F40E949769AF3FE0E0BE0740F44A
:104D38000E94F36331960E94F85EE0E0E0932B0551
:104D4800533149F40E945764A081AA3020F40E948C
:104D58009C690E941169543161F4A0915305A130F6
:104D680040F4E0915305EF5FE0935305E0E0E093F2
:104D78002B05553161F4A0911D05AA3040F4E0914E
:104D88001D05EF5FE0931D05E0E0E0932B0556312C
:104D980061F4A0911C05AA3040F4E0911C05EF5F76
:104DA800E0931C05E0E0E0932B05573161F4A091F6
:104DB8001E05A23340F4E0911E05EF5FE0931E0547
:104DC800E0E0E0932B05583161F4A0910007A43688
:104DD80040F4E0910007EB5FE0930007E0E0E09328
:104DE8002B05593171F40E947A66AC3FE0E0BE07AA
:104DF80040F40E94756632960E94F35FE0E0E0930B
:104E08002B055A3149F4A9A5A13030F4E9A5EF5F83
:104E1800E9A7E0E0E0932B055B3149F4AB89A230C8
:104E280030F4EB89EF5FEB8BE0E0E0932B055C312E
:104E380049F4AC89A33030F4EC89EF5FEC8BE0E007
:104E4800E0932B055D3179F40E94B461AE3DE3E057
:104E5800BE0748F40E94E1613A960E94A3690E9445
:104E6800B8690E94C0695E3179F40E94B961A835B9
:104E7800E2E0BE0748F40E94DD693A960E94E269C2
:104E88000E94B8690E94C0695F3161F4A09107056A
:104E9800AA3040F4E0910705EF5FE0930705E0E0F2
:104EA800E0932B05503289F40E94F869A081AA3159
:104EB80060F40E94F8690E94FE69E0910D07E030F5
:104EC80021F4E0910905E0930E05513289F40E941E
:104ED800016AA081AA3160F40E94016A0E94FE69F9
:104EE800E0910D07E03021F4E0910A05E0930F0509
:104EF800523289F40E94076AA081AA3160F40E94A4
:104F0800076A0E94FE69E0910D07E03021F4E09104
:104F18000B05E0931005533289F40E940D6AA081B5
:104F2800AA3160F40E940D6A0E94FE69E0910D07A3
:104F3800E03021F4E0910C05E0931105543289F436
:104F48000E94136AA081AA3160F40E94136A0E9429
:104F5800FE69E0910D07E03021F4E0910D05E09342
:104F68001205553249F4AB8DA33030F4EB8DEF5F69
:104F7800EB8FE0E0E0932B05563249F4AA8DA5307B
:104F880030F4EA8DEF5FEA8FE0E0E0932B055732CB
:104F980049F4A98DA13030F4E98DEF5FE98FE0E0A5
:104FA800E0932B05583249F4A88DA13030F4E88DF0
:104FB800EF5FE88FE0E0E0932B05593261F4A091B0
:104FC8003B05A83040F4E0913B05EF5FE0933B05DB
:104FD800E0E0E0932B055A3261F4A0913405A43047
:104FE80040F4E0913405EF5FE0933405E0E0E093AE
:104FF8002B055B3239F50E94335FAE3DE3E0BE0717
:10500800E0E08E07E0E09E07E8F40E94B260E65F09
:10501800FF4F6F4F7F4F0E942A5F0E94AA62E8519C
:10502800FC4F6F4F7F4F0E9463600E9491690E94FE
:105038007E60662777270E946C760E947560E0E0A4
:10504800E0932B055C3249F4AA89A13030F4EA894F
:10505800EF5FEA8BE0E0E0932B055D3291F40E946C
:10506800815FAF37E6E9BE07E8E98E07E0E09E0713
:1050780040F40E946A61EC59FF4F6F4F7F4F0E94C6
:10508800196A5E3271F40E94505FA031E7E2BE07F0
:1050980040F40E94F0623A960E944B5FE0E0E09391
:1050A8002B055F3261F4A0912007A43040F4E09111
:1050B8002007EF5FE0932007E0E0E0932B055033F3
:1050C80061F4A0911505A13040F4E0911505EF5F5A
:1050D800E0931505E0E0E0932B05513349F4AC85E6
:1050E800A43030F4EC85EF5FEC87E0E0E0932B052B
:1050F800523349F4AF89A33030F4EF89EF5FEF8B77
:10510800E0E0E0932B05533349F4AD89A33030F444
:10511800ED89EF5FED8BE0E0E0932B05543361F40C
:10512800A0914F05A33840F4E0914F05EF5FE0935D
:105138004F05E0E0E0932B05553361F4A09150054D
:10514800A73440F4E0915005EF5FE0935005E0E0AC
:10515800E0932B05563361F4A0915105A53640F430
:10516800E0915105EF5FE0935105E0E0E0932B05F6
:10517800573389F4A0913905E3E00E940A770E2E8F
:105188000E94F36841F0E0913905EF5FE09339053B
:10519800E0E0E0932B05583351F4ACA5A63938F478
:1051A800ECA5EF5F0E942C6AE0E0E0932B055933F1
:1051B80059F40E94255FA03BE4E0BE0728F40E9452
:1051C8008F6531960E943F6A5A3349F4AAA5AC33D9
:1051D80030F4EAA5EF5FEAA7E0E0E0932B055B3344
:1051E80061F4A091F005A33040F4E091F005EF5F81
:1051F800E093F005E0E0E0932B055C3361F4A091C7
:105208003505AA3F40F4E0913505EF5FE093350599
:10521800E0E0E0932B055D33E9F4E0910005EF5FF2
:10522800E0930005A0910005AC3318F0E0E0E093AE
:1052380000050E94DE5D0E94586AE295E07F6E2FAD
:105248000E945C6AE60FE0935C050E94E45DE3E07F
:105258000E941C685E3361F4A091BE05A13040F441
:10526800E091BE05EF5FE093BE05E0E0E0932B051B
:105278005F3379F40E9485690E94FD5FAE17BF070E
:1052880040F40E94F46531960E94F85FE0E0E093F4
:105298002B05503471F4E091F706EF5FE093F706C1
:1052A800E0E0E0932B05A091F706A43610F0E09318
:1052B800F706513461F4A091FB06A13040F4E09167
:1052C800FB06EF5FE093FB06E0E0E0932B0552342A
:1052D80061F4A091FC06A13040F4E091FC06EF5F78
:1052E800E093FC06E0E0E0932B05533449F4AE89E3
:1052F800A13030F4EE89EF5FEE8BE0E0E0932B0510
:10530800543471F40E94115FA83BEBE0BE0740F4EF
:105318000E948F6431960E940C5FE0E0E0932B05B9
:10532800553461F4A0915405A13040F4E09154053E
:10533800EF5FE0935405E0E0E0932B05563471F4F9
:105348000E94465FA835E2E0BE0740F40E947963F8
:105358007E960E94415FE0E0E0932B05573449F4C4
:10536800AF8DAC3330F4EF8DEF5FEF8FE0E0E0937B
:105378002B05583461F4A0910B07A13040F4E0915B
:105388000B07EF5FE0930B07E0E0E0932B05593440
:1053980061F4A0910C07A43040F4E0910C07EF5F92
:1053A800E0930C07E0E0E0932B055A3461F4A091F8
:1053B800C805A13040F4E091C805EF5FE093C80547
:1053C800E0E0E0932B055B3469F40E9443660E9499
:1053D8004966A081AA3030F40E9443660E9449665B
:1053E8000E94FE695A35E1F40E94CF65EAE0F0E0D8
:1053F8000E942C770E2E0E94CF65AA0FBB1FAD54BA
:10540800B84F0E942478DF010E94BE61E02141F07C
:105418000E94AE6531960E94B365E0E0E0932B05EB
:105428005B3561F4A0914108AF3744F4E09141083D
:10543800EF5FE0934108E0E0E0932B055C3561F411
:10544800A0910605AA3F40F4E0910605EB5FE093C2
:105458000605E0E0E0932B055D3561F4A0915E0759
:10546800A33340F4E0915E07EF5FE0935E07E0E06E
:10547800E0932B055E3561F4A0914D05A13140F410
:10548800E0914D05EF5FE0934D05E0E0E0932B05DB
:105498000E94646A0E94BB6661F0A091F205AF3F6A
:1054A80040F4E091F205EF5FE093F205E0E0E0936D
:1054B8002B050E94646A0E94746361F0A091F30551
:1054C800AF3F40F4E091F305EF5FE093F305E0E0D0
:1054D800E0932B05503671F40E941B5FA83EE3E071
:1054E800BE0740F40E946D6A3A960E94165FE0E09B
:1054F800E0932B05513699F4A091F105AA3F40F4A9
:10550800E091F105E65FE093F105E0E0E0932B051B
:10551800A091F105AB3F18F0EAEFE093F1055236A0
:10552800B1F40E949768AC91AA3F31F40E94976841
:10553800EC91EB5F0E9425690E949768AC91AA3FA5
:1055480030F40E949768EC91E65F0E9425690E94FA
:10555800726A0E94BB6649F0A8A5AA3F30F4E8A584
:10556800E65FE8A7E0E0E0932B050E94726A0E94DC
:10557800746349F0AEA1AA3F30F4EEA1E65FEEA352
:10558800E0E0E0932B05A82D0E94A85FA0E0F2FCC4
:10559800A1E00E94BB6629F0E894F2F8E0E0E0930D
:1055A8002B05A82D0E94065EA0E0F2FCA1E00E9457
:1055B8000B5E0E94F66809F445C5E1E0E0932B050F
:1055C8006894F2F8503049F4A881A13030F0E881AD
:1055D800E150E883E0E0E0932B05513049F4AEA5B3
:1055E800A13030F0EEA5E150EEA7E0E0E0932B0506
:1055F800523049F40E940869A23028F00E94C0671E
:10560800E1500E942569533099F40E941769A5302A
:1056180020F00E941E69E55007C00E941769A1305A
:1056280038F00E941E69E150EC93E0E0E0932B050E
:10563800543049F40E942A69A13028F00E94316947
:10564800E1500E942569553051F40E942E66A081D0
:10565800A13028F00E943869E1500E94256956302F
:1056680061F40E944E663B9740F00E943F693A976A
:10567800FE93EE93E0E0E0932B05573061F4A091A0
:105688001905A23040F0E0911905E150E0931905A1
:10569800E0E0E0932B05583061F4A0913305A13088
:1056A80040F0E0913305E150E0933305E0E0E0930A
:1056B8002B05593051F40E941366A081A23028F0BE
:1056C8000E944B69E1500E9425695A3051F40E94AA
:1056D8004366A081A13028F00E945269E1500E94DF
:1056E80025695B3041F40E94596928F00E9461697C
:1056F800E1500E9425695C3089F40E945A5F5597F1
:1057080068F00E94686931970E946D690E947A6901
:105718000E947C690E9485690E948A695D3071F4E3
:105728000E94EE5EA538E3E0BE0740F00E94AC633D
:1057380031970E94E95EE0E0E0932B055E3099F432
:105748000E947A690E947B6A0E94075F0E946E66C7
:1057580009F008F408C00E94856731970E94025F2B
:10576800E0E0E0932B055F3079F40E9491690E9494
:10577800735FEA17FB0740F40E94856931970E941E
:105788005F5FE0E0E0932B05503169F40E944F64BD
:105798000E94587840F40E94FC6331970E94FD5E95
:1057A800E0E0E0932B05513169F40E943D640E94CA
:1057B800587840F40E94EE6331970E94F35EE0E06F
:1057C800E0932B05523169F40E9497690E9458783A
:1057D80040F40E94F36331970E94F85EE0E0E093A2
:1057E8002B05533151F40E945764A081A13028F051
:1057F8000E949C69E1500E942569543161F4A0918E
:105808005305A13040F0E0915305E150E093530572
:10581800E0E0E0932B05553161F4A0911D05A1301E
:1058280040F0E0911D05E150E0931D05E0E0E093B4
:105838002B05563161F4A0911C05A13040F0E09190
:105848001C05E150E0931C05E0E0E0932B0557317F
:1058580061F4A0911E05A23040F0E0911E05E150D0
:10586800E0931E05E0E0E0932B05583161F4A09128
:105878000007A63040F0E0910007E550E0930007EC
:10588800E0E0E0932B05593161F40E947A661397A2
:1058980040F00E94756632970E94F35FE0E0E09363
:1058A8002B055A3149F4A9A5A13030F0E9A5E150FA
:1058B800E9A7E0E0E0932B055C3149F4AC89A1301D
:1058C80030F0EC89E150EC8BE0E0E0932B055B31A4
:1058D80049F4AB89A13030F0EB89E150EB8BE0E083
:1058E800E0932B055D3171F40E94B4610E945878F1
:1058F80048F40E94E16131970E94A3690E94B86947
:105908000E94C0695E3171F40E94B9610E945878A2
:1059180048F40E94DD6931970E94E2690E94B869E3
:105928000E94C0695F3161F4A0910705A23040F080
:10593800E0910705E150E0930705E0E0E0932B05CF
:10594800503289F40E94F869A081A23060F00E9468
:10595800F8690E94826AE0910D07E03021F4E09135
:105968000905E0930E05513289F40E94016AA0816D
:10597800A13060F00E94016A0E94826AE0910D07DE
:10598800E03021F4E0910A05E0930F05523289F4E2
:105998000E94076AA081A13060F00E94076A0E94F5
:1059A800826AE0910D07E03021F4E0910B05E09365
:1059B8001005533289F40E940D6AA081A13060F06D
:1059C8000E940D6A0E94826AE0910D07E03021F47E
:1059D800E0910C05E0931105543289F40E94136A92
:1059E800A081A13060F00E94136A0E94826AE0914F
:1059F8000D07E03021F4E0910D05E09312055532D2
:105A080049F4AB8DA13030F0EB8DE150EB8FE0E045
:105A1800E0932B05563249F4AA8DA13030F0EA8D77
:105A2800E150EA8FE0E0E0932B05573249F4A98D65
:105A3800A13030F0E98DE150E98FE0E0E0932B05EB
:105A4800583249F4A88DA13030F0E88DE150E88F44
:105A5800E0E0E0932B05593261F4A0913B05A130B9
:105A680040F0E0913B05E150E0933B05E0E0E09336
:105A78002B055A3261F4A0913405A13040F0E09131
:105A88003405E150E0933405E0E0E0932B055B3208
:105A980049F50E94335FAB30E0E0BE07E0E08E07D7
:105AA800E0E09E07F8F00E94B2600E94B3620E9494
:105AB8002A5F0E94AA62E456F040604070400E944B
:105AC80063600E9468690E947E600E945663A0938A
:105AD800C408B093C5088093C6089093C708E0E04F
:105AE800E0932B055C3249F4AA89A13030F0EA89A9
:105AF800E150EA8BE0E0E0932B055D3269F40E9407
:105B0800815F0E94866A40F00E946A61EA50F04014
:105B1800604070400E94196A5E3269F40E94505FCA
:105B28000E94587840F40E94F06231970E944B5FBF
:105B3800E0E0E0932B055F3261F4A0912007A130EB
:105B480040F0E0912007E150E0932007E0E0E09387
:105B58002B05503361F4A0911505A13040F0E09178
:105B68001505E150E0931505E0E0E0932B0551336E
:105B780049F4AC85A13030F0EC85E150EC87E0E0E9
:105B8800E0932B05523349F4AF89A13030F0EF8907
:105B9800E150EF8BE0E0E0932B05533349F4AD89F6
:105BA800A13030F0ED89E150ED8BE0E0E0932B057A
:105BB800543361F4A0914F05A53140F0E0914F05B1
:105BC800E150E0934F05E0E0E0932B05553361F495
:105BD800A0915005A53140F0E0915005E150E093C7
:105BE8005005E0E0E0932B05563361F4A091510590
:105BF800A53140F0E0915105E150E0935105E0E016
:105C0800E0932B05573379F4A09139050E945B6323
:105C18000E94F36841F0E0913905E150E0933905BD
:105C2800E0E0E0932B05583351F4ACA5AD3338F0E0
:105C3800ECA5E1500E942C6AE0E0E0932B05593373
:105C480059F40E94255FA73DE1E0BE0728F00E94B5
:105C58008F6531970E943F6A5A3349F4AAA5AB3041
:105C680030F0EAA5E150EAA7E0E0E0932B055B33CA
:105C780061F4A091F005A13040F0E091F005E15009
:105C8800E093F005E0E0E0932B055C3361F4A0912C
:105C98003505A13040F0E0913505E150E093350538
:105CA800E0E0E0932B055D3331F5E0910105EF5F0E
:105CB800E0930105A0910105AD3018F0E1E0E09313
:105CC8000105E2E0E0935A05A0910105B0E00E94C9
:105CD800BB67E295E07F6E2F0E948E6AE60FE09325
:105CE8005B05E0915B05E05CE0935B050E94E45D89
:105CF800E2E00E941C685E3361F4A091BE05A13009
:105D080040F0E091BE05E150E093BE05E0E0E0938D
:105D18002B055F3379F40E9491690E94FD5FEA17B1
:105D2800FB0740F40E94F46531970E94F85FE0E0B9
:105D3800E0932B05503471F4E091F606EF5FE093A1
:105D4800F606E0E0E0932B05A091F606A43610F0E5
:105D5800E093F606513461F4A091FB06A13040F0BF
:105D6800E091FB06E150E093FB06E0E0E0932B05B1
:105D7800523461F4A091FC06A13040F0E091FC0699
:105D8800E150E093FC06E0E0E0932B05533449F43E
:105D9800AE89A13030F0EE89E150EE8BE0E0E0937F
:105DA8002B05543471F40E94115FA13DE7E0BE0752
:105DB80040F00E948F6431970E940C5FE0E0E0930E
:105DC8002B05553461F4A0915405A13040F0E091C1
:105DD8005405E150E0935405E0E0E0932B05563478
:105DE80069F40E94465F0E94587840F40E947963E3
:105DF8007E970E94415FE0E0E0932B05573449F419
:105E0800AF8DA13030F0EF8DE150EF8FE0E0E093FF
:105E18002B05583461F4A0910B07A13040F0E091B4
:105E28000B07E150E0930B07E0E0E0932B055934B2
:105E380061F4A0910C07A13040F0E0910C07E1500B
:105E4800E0930C07E0E0E0932B055A3461F4A0914D
:105E5800C805A13040F0E091C805E150E093C805BD
:105E6800E0E0E0932B055B3469F40E9443660E94EE
:105E78004966A081A23030F00E9443660E944966BC
:105E88000E94826A5A35D9F40E94CF650E945878D8
:105E9800B0F40E94AE6531970E94B365E0E0E093EC
:105EA8002B050E94AE65309751F4E9E0E0930407B2
:105EB800E0E0E093C707E093C807E093CA055B35C5
:105EC80069F4A0914108E1E8EA1744F4E091410837
:105ED800E150E0934108E0E0E0932B055C3561F484
:105EE800A0910605A13040F0E0910605E550E09349
:105EF8000605E0E0E0932B055D3561F4A0915E07AF
:105F0800A13040F0E0915E07E150E0935E07E0E0E9
:105F1800E0932B055E3561F4A0914D05A13040F06A
:105F2800E0914D05E150E0934D05E0E0E0932B054D
:105F38000E94646A0E94BB6661F0A091F205A130DC
:105F480040F0E091F205E150E093F205E0E0E093E3
:105F58002B050E94646A0E94746361F0A091F305A6
:105F6800A13040F0E091F305E150E093F305E0E063
:105F7800E0932B05503661F40E941B5F559740F063
:105F88000E946D6A3A970E94165FE0E0E0932B0545
:105F9800513699F4A091F105A13040F0E091F10556
:105FA800EA50E093F105E0E0E0932B05A091F105BC
:105FB800AA3018F4E0E0E093F105523639F5E091A3
:105FC8001B05F0E0BF01DE019296AE0FBF1FAC913A
:105FD8000E945B63FB01DE019296AE0FBF1FAC917E
:105FE800EFEF0E940A77E02131F00E949768EC9168
:105FF800EA500E9425690E949768AC91AF3F31F43E
:106008000E949768EC91E5500E9425690E94726A87
:106018000E94BB6649F0A8A5A13030F0E8A5EA5077
:10602800E8A7E0E0E0932B050E94726A0E9474637F
:1060380049F0AEA1A13030F0EEA1EA50EEA3E0E0C5
:10604800E0932B05A72D0E94065EA9A1EFEF0E9401
:106058000A770E9460630E940A770E22AD8D0E9423
:10606800746319F0E9A1EF5FE9A3A72D0E94A85F67
:106078000E94FB650E22AD8D0E94746321F0E894A6
:10608800F0F8E0E0E9A3A9A1EEE10E94F1760E9410
:10609800A4650E940A770E22A091FA06E2E00E9407
:1060A800F176E02121F0E1E0E093FA06EE8FEF8D42
:1060B800E03011F4E0E0EE8F0E94F5620E9466760F
:1060C8000E2E0E941E630E22AE8D0E948B6611F06A
:1060D800E1E0EE8FAE8DAC3311F40E945464A091D0
:1060E8000605A13028F0E0910605F0E00E94E9637A
:1060F800AA890E94A85F0E9401640E94BE61E021F3
:1061080041F1EB85EF5FEB87F0E03196BF010E942C
:10611800966AE617F70798F40E9485690E94B163AA
:106128000E9440770E2E0E949C6AE4EAF1E060E04B
:1061380070E00E943877E02911F00E942D640E94D7
:10614800966AAB85B0E0EA17FB0710F4E0E0EB874E
:1061580002C0E0E0EB870E940A680E9485690E94FD
:10616800B1630E9458770E220E94735FE4EAF1E05F
:106178000E941A770E22AC850E941D6451F00E947D
:106188000164A639E0E0BE0720F4E6E9F0E00E94E9
:10619800E463E8ECE51509F01EC1E09150090E949E
:1061A8009D650E943A7609F008F40CC00E947E634F
:1061B800E1600E94A56A0E940563A0E5B9E00E941B
:1061C800E474EC93E0915109ABA9BCA9F0E00E94FA
:1061D80026770E2EE0915109ADA9BEA90E94AA6AA0
:1061E800AFA9B8AD0E94AA6AA9ADBAADF0E00E9405
:1061F8002677E02989F10E947E63E2600E94A56A01
:10620800E0915109ABA9BCA9F0E0EA17FB071CF41F
:10621800EBA9E0935109E0915109ADA9BEA9F0E0BD
:10622800EA17FB071CF4EDA9E0935109E091510925
:10623800AFA9B8ADF0E0EA17FB071CF4EFA9E093AB
:106248005109E0915109A9ADBAADF0E0EA17FB0791
:106258001CF4E9ADE0935109E0915D09F0915E0904
:10626800AFA5B8A90E9432770E2E0E944A63E0219A
:1062780049F00E947E63E4600E94A56AEFA5F8A930
:106288000E94E95FE0915309F0915409D8010E94F6
:106298002C770E2EE8ECF0E00E942677E02149F0FA
:1062A8000E947E63E8600E94A56A009353091093D8
:1062B8005409E0915509F0915609E017F10748F49F
:1062C8000E947E63E0610E94A56A009355091093BD
:1062D80056090E94B16AE0915709F09158090E9445
:1062E800C9660E9417670E220E94E86559F00E944D
:1062F8007E63E0620E94A56AE0918808F0918908AF
:106308000E94CB5F0E94B66AE0915909F0915A0940
:106318000E94C9660E9417670E220E94E86559F01C
:106328000E947E63E0640E94A56AE0918A08F09169
:106338008B080E94D55F0E94BB6AE0915B09F091CF
:106348005C090E94C9660E9417670E220E94E865D0
:1063580059F00E947E63E0680E94A56AE0918C086B
:10636800F0918D080E94DF5FEFA5F8A90E94E776FB
:106378000E94C06AF8010E94C96A0E94E7760E94DA
:1063880093770E94C06A0E94C96A0E94D26AE09309
:10639800B808F093B9086093BA087093BB08E09105
:1063A800A808F091A908A091B808B091B9088091FF
:1063B800BA089091BB080E94E7760E9462785CF464
:1063C800E091DA07E160E093DA07E091B808F0912C
:1063D800B9080E94C15FA0912607A33610F00C945B
:1063E800F23CA0E025FCA1E00E94A85FA09157051F
:1063F8000E94D66AA0E027FCA1E00E94906621F0E6
:10640800E894F799689401C0E894F5F8E0912105BB
:10641800E170EE0FAE2FE0912105E6950E94DB6A50
:10642800EA0F0E2EE0912105E695E695E170AE2F74
:10643800E0E0F5FCE1E0EA2BEE0FEE0FE00DE09373
:106448005C07A8890E945B63AF850E94E06A29F017
:10645800E0915C07EF5FE0935C070E94E868E081E9
:10646800E0932607A09120050E945B63AC850E94FB
:10647800E56A49F4F79907C0A0E0F699A1E0EA2F88
:10648800E295E07F19C0A0E0F699A1E0EA2FE29535
:10649800E07F0E2EA0E0F299A1E0EA2FEE0FEE0FBA
:1064A8000E0EA0E0F399A1E0EA2FEE0FA02DAE0F9B
:1064B800E0E0F499E1E0EA0FE0935D07A8A9AA23D8
:1064C8001AF4E05AE0935D070E94EA6A0E94FE6AA5
:1064D800E89430F8A091FD06A13011F46894F5F81D
:1064E800EC89E03019F4E9E0E0935B07AC89A1306E
:1064F80081F4A0E021FCA1E0EA2FEE0FE75F0E2E69
:10650800A0E021FCA1E0EA2FEE0FEE0FE00DE093F2
:106518005B07AC89A23069F4E9E0E0935B07A0E08F
:1065280021FCA1E00E940C6BA0E021FCA1E00E94EC
:10653800136BAC89A33031F4E0E021FCE1E0E85FC3
:10654800E0935B07E0E0F799E1E0E09302050E9441
:106558007A69AEEAB7E489E091E40E941E6B09F01B
:1065680008F403C0E1E0E09302050E947A69ABE712
:10657800B4E182E191E40E941E6B09F008F403C0C3
:10658800E3E0E09302050E947A69ADE3BAE08BE1AB
:1065980091E40E941E6B09F008F403C0E7E0E09361
:1065A80002050E947A69AFE1B5E88FE191E40E94A3
:1065B8001E6B09F008F403C0EFE0E09302050E94A7
:1065C8007A69A1EEBAE788E291E40E941E6B09F0AD
:1065D80008F403C0EFE1E0930205A0912507A43079
:1065E80019F5A0E0F799A1E00E940C6BA0E0F799DB
:1065F800A1E00E94136BA0E0F799A1E00E94A85FB8
:10660800A0912B050E94746311F0E1E00BC0A0E09B
:10661800F799A1E00E94065EA0912B050E94BB6637
:1066280019F0E0E0E0932B05A0910305A431D0F523
:106638000E949465A83EE3E0BE0734F0E7EEF3E07D
:10664800E093AC08F093AD080E949465AD39EFEF84
:10665800BE0734F4EDE9FFEFE093AC08F093AD0822
:10666800A091AD08AA2372F00E949465A436E0E0D8
:10667800BE0724F00E94286BE0932B070E94336B1F
:106688000E94356BA091AD08AA235AF4EDE0E0937F
:106698002B07E091AC08F091AD080E943D6B0E9479
:1066A800356B0AC0F79B04C0E0E4E0932B0702C0F7
:1066B8000E94416BE0932C07AA85A13098F0EA85E7
:1066C800E150EA87EEE5E0932B07A0912507A43077
:1066D80018F4E091250704C0E0E5E0932B07EAE011
:1066E800E0932C07A985A13050F0E985E150E987AE
:1066F800E8E3E0932B07E0911B05E0932C07A885BE
:10670800A13048F0E885E150E887E9E3E0932B07FA
:10671800E0E5E0932C07E0911605E03009F041C070
:10672800E0915C07E058E0935C07EAE0E093290712
:10673800E0E0E0932A07A0916608B09167080E94FC
:10674800587874F40E94BB670E94456B0E944A6B9C
:106758001A9724F00E944F6B0E94516B0E94596B4C
:10676800A0916708AA23EAF4E0916608F091670807
:106778000E943D6B0E94456BE0E4E0932907E0919D
:106788006808E0932A070E944A6B1A9744F00E940F
:106798004F6B0E94516B0E94596B689401C0E8943A
:1067A80030F8A0911605A13009F044C0E0915D07CA
:1067B800E85FE0935D070E94616BFF2392F4E0E4D9
:1067C800E09329070E94616BE73FAFEFFA0714F4E3
:1067D800689401C0E89430F80E94616B0E947B764F
:1067E80004C0E89430F80E94616BE0936808F09365
:1067F80069080E944A6B1A9724F00E944F6B0E9406
:10680800516B0E94596B0E94616BBF01DF01E3E687
:10681800F0E00E9426770E2EDB01EDE9FFEF0E94E3
:106828002077E02939F0E89430F8E0E4E09329078C
:10683800E0932A07E0910C07E030F9F4D8010E94B0
:106848006C6BE0932D07D8010E94BB670E94766BA2
:10685800E0932E07D8010E947C6BE0932F0706393E
:10686800E0E01E0754F4E0E4E0932D07E0932E07E0
:10687800E0932F07E0E0E0930205A0910C07A13018
:1068880008F4D9C0A13079F50E947A69A2E5B8EB7D
:106898008AE391E40E94A7757F936F93FF93EF9328
:1068A8000E947A690E947B6AAF91BF918F919F91F4
:1068B8000E946A640E94816B0E948A6B7F936F9327
:1068C800FF93EF930E947A690E947B6AD8010E9425
:1068D800EC760E9444780E946A64AF91BF918F91D0
:1068E8009F910E94996BA0910C07A230E9F40E9435
:1068F800075F0E948569EA1BFB0BA0EEB8E00E94C7
:1069080077650E948A6B7F936F93FF93EF930E9442
:10691800075FF801EA1BFB0BAF91BF918F919F9125
:106928000E9494640E94996BA0910C07A33081F493
:106938000E94F965A0EEB8E00E94CC630E948A6BC1
:10694800DF01CB010E94AA620E941D750E94996B0B
:10695800A0910C07A430B1F40E9468690E94335FCB
:10696800662777270E946877A0EEB8E00E94CC637C
:106978000E948A6BDF01CB010E94C1620E941D75D3
:106988000E94996BE091E008F091E1086091E208BB
:106998007091E3080E94E6749F01EAE0E0932F07F4
:1069A8002436E0E03E072CF023E630E0E3E2E09313
:1069B8002F0733232AF420E030E0ECE1E0932F079F
:1069C800D9010E94BB670E94766BE0932D07E09186
:1069D8002D07E03019F4EAE0E0932D07D9010E9471
:1069E8007C6BE0932E07E0E0F799E1E0E093020585
:1069F8000024021603061CF4E1E0E09302052431AA
:106A0800E0E03E071CF0E3E0E09302052832E0E016
:106A18003E071CF0E7E0E09302052C33E0E03E0778
:106A28001CF0EFE0E09302052035E0E03E071CF0A3
:106A3800EFE1E0930205A0914808B0914908E2E32C
:106A4800F0E00E9420770E2EA0914A08B0914B08E2
:106A5800E2E3F0E00E9420770E22A52DE6E40E94F2
:106A68000A77E02119F0E0E0E0932607E091260795
:106A7800E03079F4EEE3E0933107E5E0E0933207A4
:106A8800ECE70E949C6BE7E30E94A26BEEE5E093C3
:106A98003707A0912607A13009F058C0A8890E949D
:106AA800065EAF850E94746311F00E94A86B0E9475
:106AB800A35FA83EE3E0BE0790F0E0915B07E05ECD
:106AC800E0935B070E94A35F0E94B46BE0933507D5
:106AD8000E94BE6BE09336070E94CA6B17C0E09114
:106AE8005B07E056E0935B070E94A35FA436E0E0F3
:106AF800BE0720F00E94BE6BE09335070E94CA6B68
:106B08000E94D26BE09336070E94A35FEAE0F0E0B0
:106B18000E94DA77E0933707E9E0EC1518F4E2E031
:106B2800E0933007AC2DBB270E947C6BE0933107C4
:106B3800AD2DB0E00E94BB670E94766BE0933207F0
:106B4800AD2DBB270E947C6BE0933307A0912607ED
:106B5800A23009F05EC0E0915B07E054E0935B0768
:106B68000E94815FA034E2E4BE07EFE08E07E0E018
:106B78009E0750F00E94815FE0E4F2E46FE070E06D
:106B88000E94D76BE09331070E94815FA03AE6E844
:106B9800BE07E1E08E07E0E09E0750F00E94815FAB
:106BA800E0EAF6E861E070E00E94D76BE093320714
:106BB8000E94815F0E94E26B40F00E94815F0E9408
:106BC800EA6B0E94D76BE09333070E94815F0E94B3
:106BD800EF6B40F00E94815F0E94F76B0E94D76BB9
:106BE800E09334070E94815F0E94FC6B40F00E9492
:106BF800815F0E9451630E94D76BE09335070E9422
:106C0800046C0E94D76BE09336070E94046C0E94C4
:106C18000B6CA0912607A33089F5E7E70E94106C5A
:106C28000E946C600E94E26B24F00E946C600E94DB
:106C3800166C0E946C600E94EF6B24F00E946C60DE
:106C48000E94246C0E946C600E94FC6B44F00E94BD
:106C58006C600E94D26A0E94326CE09335070E94F1
:106C68006C600E94866A34F00E943B6C0E94426C01
:106C7800E09336070E943B6C0E94456CA091260762
:106C88000E943364A0912607E9E00E94F176E0298A
:106C980099F10E944A6CA93019F4E2E0E0933007B8
:106CA800EEE30E94106C0E947E600E94E26B24F06A
:106CB8000E947E600E94166C0E947E600E94EF6BAC
:106CC80024F00E947E600E94246C0E947E600E94D4
:106CD800FC6B44F00E947E600E94D26A0E94326C73
:106CE800E09335070E94526C0E94426CE09336078D
:106CF8000E94526C0E94456CA0912607E5E00E9414
:106D0800F1760E2EEAE00E94F176E02909F457C0E8
:106D18000E944A6CAA3019F4E2E0E0933007EEE3EF
:106D28000E94106CE0E5E0933307A0916B08AA235A
:106D38001AF4E0E4E09335070E94EA65AD39EFEF15
:106D4800BE071CF4E0E4E0933407A0916B08AA2383
:106D5800BAF00E94EA65A436E0E0BE0734F00E946B
:106D6800EA650E946C6BE09335070E94EA650E9411
:106D7800BB670E94766BE09336070E94EA6519C0EC
:106D88000E94596CE436A0E0FA0744F00E94596C5E
:106D98000E9434660E94766BE09335070E94EF6587
:106DA8000E943D6B0E94766BE09336070E94596CF7
:106DB800DF01EAE0F0E00E94DD77E0933707A09179
:106DC8002607A630C9F50E945D6CE0E0E093310724
:106DD8000E94636CA9A9BAA9A031E7E2BE0724F012
:106DE800EFE0F7E2E9ABFAABAAA9AA231AF4E0E0CC
:106DF800E9ABEAABA9A9BAA9A83EE3E0BE0724F02B
:106E08000E946A6CE0933407A9A9BAA9A436E0E005
:106E1800BE0724F00E946C6BE0933507A9A9BAA9B4
:106E28000E94BB670E94766BE0933607A9A9BAA9AE
:106E38000E947C6BE0933707A0912607A73009F0E2
:106E48004DC00E9401640E94587800F5ECE0E09380
:106E580031070E942264F695E795E436A0E0FA0728
:106E680030F00E9401640E946F6CE09332070E9428
:106E78002264F695E7953A9730F00E9401640E94E3
:106E8800756CE09333070E94226421C0EBE0E09325
:106E980031070E947B6CE436A0E0FA0740F0A0912D
:106EA800EF07B091F0070E946F6CE09332070E94E1
:106EB8007B6C3A9740F0A091EF07B091F0070E94E1
:106EC800756CE0933307E091EF07F091F007F695C2
:106ED800E795DF010E94D26BE0933407A091260763
:106EE800A83009F07AC0A8890E94065EAF850E9482
:106EF800746311F00E94A86BA0916008B0916108BA
:106F0800A135EBEFBE0734F4E1E5FBEFE093600851
:106F1800F0936108A0916008B0916108A03BE4E09B
:106F2800BE0734F0EFEAF4E0E0936008F0936108FC
:106F3800A0916108AA2352F4E0E4E0933407E091B9
:106F48006008F09161080E947B7604C0E0916008B7
:106F5800F0916108E0936408F0936508A0916408D3
:106F6800B0916508ECE3F0E00E94AB77E0938F07FF
:106F7800F09390070E94826CECE30E948877A091BE
:106F88006408B0916508AE1BBF0BA0939107B0933E
:106F9800920722FE1DC00E94826C1A9718F0E2E048
:106FA800E09330070E94826C0E94D26BE093310715
:106FB800A0919107B09192070E94876CE0933207E5
:106FC800A0919107B09192070E94D26BE09333078A
:106FD8000E948D6CE8E7E0933707A0912607AB3055
:106FE80061F5E0915B07E054E0935B07E9E30E94F9
:106FF800946C0E94505FA83EE3E0BE0730F00E9408
:10700800505F0E94B46BE09334070E94505FA4362F
:10701800E0E0BE0730F00E94505F0E949A6CE09357
:1070280035070E94505F0E94876CE09336070E94E4
:10703800505F0E94D26BE0933707A0912607AC30CF
:1070480009F08BC0E2E0E0933007EEE3E09331070C
:10705800A091AF08AA239AF10E94A06C1A9744F055
:107068000E94A06C0E94BB670E94766BE093360773
:107078000E94A06CA436E0E0BE0734F00E94A06C29
:107088000E946C6BE09335070E94A06CA83EE3E079
:10709800BE0734F00E94A06C0E946A6CE09334072B
:1070A8000E94A06CA031E7E2BE0734F00E94A06CF9
:1070B8000E94A56CE09333070E94A06C48C0EAE0E8
:1070C800E09336070E94A06CA73FEFEFBE075CF481
:1070D8000E94AA6C0E943D6B0E94766BE093360773
:1070E800EDE0E09335070E94A06CAD39EFEFBE07E5
:1070F8005CF40E94AF6C0E9434660E94766BE09349
:107108003507EDE0E09334070E94A06CA931ECEF5D
:10711800BE0754F40E94AF6CDF010E946A6CE093D2
:107128003407EDE0E09333070E94A06CA13FE8ED3F
:10713800BE0754F40E94AF6CDF010E94A56CE09377
:107148003307EDE0E09332070E94AF6CDF01EAE01D
:10715800F0E00E94DD77E0933707A0912607AD3075
:1071680071F50E94B36CE3E6E0933707A0918908B4
:10717800AA233AF4E0E4E0933507E0918808E19522
:1071880004C00E94B16A0E947C6BE09336070E949B
:10719800B16AA436E0E0BE0734F00E94B16A0E94EA
:1071A8006C6BE09334070E94B16A1A9744F00E940E
:1071B800B16A0E94BB670E94766BE0933507A09185
:1071C8002607AE3071F50E94BD6CE3E6E093370701
:1071D800A0918B08AA233AF4E0E4E0933507E09104
:1071E8008A08E19504C00E94B66A0E947C6BE0930D
:1071F80036070E94B66AA436E0E0BE0734F00E9463
:10720800B66A0E946C6BE09334070E94B66A1A97BC
:1072180044F00E94B66A0E94BB670E94766BE093B6
:107228003507A0912607AF3071F50E94C76CE3E6D9
:10723800E0933707A0918D08AA233AF4E0E4E0939D
:107248003507E0918C08E19504C00E94BB6A0E9452
:107258007C6BE09336070E94BB6AA436E0E0BE0769
:1072680034F00E94BB6A0E946C6BE09334070E9462
:10727800BB6A1A9744F00E94BB6A0E94BB670E94CF
:10728800766BE0933507A0912607A03119F5A889F8
:107298000E94065EAF850E94746311F00E94A86B7D
:1072A800E0E00E94CF5D0E94D16CA0910105AA3058
:1072B80018F0E2E0E09330070E948E6AE09331070D
:1072C8000E94586A0E94766BE09332070E945C6ABB
:1072D800E0933307A0912607A13109F042C00E942C
:1072E8005D6CE0914E08F0914F080E94F76C7F9317
:1072F8006F93FF93EF93E0914E08F0914F080E942F
:10730800006DAF91BF918F919F910E946A64A1E037
:10731800B8E00E94D5610E940B6D129728F4E0E056
:10732800E0930108E09302080E94106DE1E0E09309
:1073380033070E940B6DA436E0E0BE0730F00E94D0
:107348000B6D0E949A6CE09335070E940B6D0E94AA
:10735800876CE09336070E940B6D0E94D26BE09316
:107368003707A0912607A23109F042C00E945D6C40
:10737800E0915008F09151080E94F76C7F936F9349
:10738800FF93EF93E0915008F09151080E94006D2F
:10739800AF91BF918F919F910E946A64A3E0B8E07A
:1073A8000E94D5610E94176D129728F4E0E0E093DF
:1073B8000308E09304080E94106DE2E0E0933307AD
:1073C8000E94176DA436E0E0BE0730F00E94176DEA
:1073D8000E949A6CE09335070E94176D0E94876C93
:1073E800E09336070E94176D0E94D26BE09337072F
:1073F800A0912607A33109F061C00E941C6DAAEA7A
:10740800B8E00E94F661E0E50E94256DE4E5E093AE
:107418003307A091AB08AA2312F4EDE001C0EAE01B
:10742800E09336070E942B6DA73FEFEFBE0714F4D9
:10743800EDE001C0EAE0E09335070E942B6DAD391D
:10744800EFEFBE0714F4EDE001C0EAE0E093340783
:10745800A091AB08AA2342F40E941C6D0E94B1744B
:10746800AAEAB8E00E94F6610E942B6DA83EE3E00C
:10747800BE0734F00E942B6D0E946A6CE0933407BB
:107488000E942B6DA436E0E0BE0734F00E942B6DFD
:107498000E946C6BE09335070E942B6D1A9744F09D
:1074A8000E942B6D0E94BB670E94766BE0933607A3
:1074B8000E942B6D0E947C6BE0933707A0912607F2
:1074C800A43109F051C0A72D0E94065E0E941167E1
:1074D8000E220E9409660E940F6629F0E0E0E09300
:1074E8008107E0938207E2E0E09331070E94306D64
:1074F800A83EE3E0BE07C8F0E0915B07E05EE093DA
:107508005B070E94306D0E94B46BE09335070E94C0
:10751800306D0E949A6CE09336070E94306DEAE065
:10752800F0E00E949877DF0119C0E0915B07E05610
:10753800E0935B070E94306DA436E0E0BE0730F0B0
:107548000E94306D0E949A6CE09335070E94306D5E
:107558000E94876CE09336070E94306DEAE0F0E005
:107568000E94DA77E0933707A0912607A531C1F486
:107578000E944A6CA93019F4E2E0E09330070E94B7
:10758800356D30F00E94466D0E949A6CE093350785
:107598000E94466D0E94876C0E944B6DE0933707EE
:1075A800A0912607E6E10E94F1760E2EE7E10E94FF
:1075B800F176E029C1F10E944A6CA93019F4E2E0A1
:1075C800E0933007E5E00E94256D0E944F6DA09181
:1075D8002607E7E10E945A6D29F0E4E5E0933207B7
:1075E8000E94646DEDE00E946F6DA83EE3E0BE0767
:1075F80030F00E94766D0E94B46BE09334070E94CD
:10760800766DA436E0E0BE0730F00E94766D0E94E9
:107618009A6CE09335070E94766D0E94876C0E94F1
:107628007B6DE0933707A0912607A831F9F4A0E015
:1076380022FCA1E00E94065E0E947F6D91F40E94E8
:1076480016621A9744F00E9416620E94BB670E9455
:10765800766BE09332070E9416620E947C6BE0937F
:1076680033070E948D6CE5E0E0933707A091260769
:10767800A931D9F40E945D6C0E9490600E945C78E8
:1076880010F40E94846D0E948F6D0E94966D0E9476
:107698009E6D19F4EAE0E09335070E94A46D0E94FC
:1076A800876C0E94A96DE0933707A0912607AA313D
:1076B80061F40E94AD6D18F0E1E0E09330070E949C
:1076C800C16D0E94D16D0E94F36DA09115070E94B3
:1076D800A85FA09116070E94D66AA09117070E947A
:1076E800D66AA09118070E94906609F43BC0F799E2
:1076F80028C00E94026EECE70E940B6EE0E0E09367
:107708003307E5E00E94116EEAE0E0933607E1E016
:10771800E0932B05A09111070E94A85FA091120782
:107728000E94D66AA09113070E94D66AA0911407F6
:107738000E94906611F0E8E301C0EAE0E0933707A1
:1077480011C0E0E0E0931507E0931607E0931707F0
:10775800E0931807E0931107E0931207E0931307EB
:10776800E0931407A8890E945B63AF850E94E06AD2
:1077780009F48BC00E94026EEAE0E09331070E9490
:10778800FE6AAF850E945B63A8890E948B6649F1F7
:10779800AF85A13029F40E94176EECE0E09334071E
:1077A800AF85A23029F40E94176EEDE0E09334070C
:1077B800AF85A33029F40E94176EEBE0E0933407FD
:1077C8000E941E6E29F00E94176EECE0E0933407C9
:1077D8000E94286E29F00E94176EEBE0E0933407B0
:1077E80028C0AF85A13029F40E94326EECE0E09306
:1077F8003707AF85A23029F40E94326EEDE0E0939E
:107808003707AF85A33029F40E94326EEBE0E0938E
:1078180037070E941E6E29F00E94326EECE0E0935A
:1078280037070E94286E29F00E94326EEBE0E09341
:107838003707A889A13029F40E94396EECE0E0935B
:107848003707A889A23029F40E94396EEDE0E09349
:107858003707A889A33029F40E94396EEBE0E0933A
:107868003707A889E4E00E94406E29F00E94396E2B
:10787800ECE0E0933707A889E5E00E94406E29F024
:107888000E94396EEBE0E0933707A0910F070E9442
:107898005B630E94486E1E2EA09110070E945B63D6
:1078A8000E94486EE129D9F00E94026E0E94B36CD2
:1078B800A0910F07A13030F0E0910F070E944F6EA2
:1078C8000E94556EA0911007A13030F0E09110078A
:1078D8000E944F6E0E945C6EE2E0E0932B05A0913F
:1078E8000F07E4E00E940F770E2E0E94636E1E2E93
:1078F800A0911007E4E00E940F770E2E0E94636E9D
:10790800E129E9F00E94026E0E94BD6CA0910F0768
:10791800A13038F0E0910F07E4500E944F6E0E94AA
:10792800556EA0911007A13038F0E0911007E4508F
:107938000E944F6E0E945C6EE2E0E0932B05A091DE
:107948000F070E94686E1E2EA09110070E94686E95
:10795800E129E9F00E94026E0E94C76CA0910F070E
:10796800A13038F0E0910F07E8500E944F6E0E9456
:10797800556EA0911007A13038F0E0911007E8503B
:107988000E944F6E0E945C6EE2E0E0932B05A0918E
:1079980010070E945B63A0E0F799A1E0E1E00E9474
:1079A800F1760E9460630E940A77E02119F0E0E016
:1079B800E0932B05A091FA06A13081F4E0915C07D1
:1079C800EB7FE0935C07EF7EE0935C07EF5FE0936B
:1079D8005C07E0915B07EF77E0935B070E9417690C
:1079E800A43638F4E4E6E09371070E946D6EE093E4
:1079F80072070E941769A53648F00E941769E8ECDB
:107A0800EA1BE0937107E4E6E09372070E941769A6
:107A1800A43629F4E4E6E0937107E0937207A09195
:107A28002607A33611F00C940F4FE1E0E0932707E7
:107A3800A0912707A03148F40E94746EAAE0A083A1
:107A4800E89430F80E94D762F3CFA52FE9E50E94A9
:107A58007A6EE8E50E94F176E02909F05BE45C348F
:107A680009F45AE5503089F4E881E03019F4E42F3C
:107A78000E947F6EA881A13040F0E881F0E0319744
:107A8800E553FA4FE0810E947F6E513019F4EEA55C
:107A98000E947F6E523021F40E94C0670E947F6E60
:107AA800533021F40E946D6E0E947F6E543021F491
:107AB8000E94856E0E947F6E553029F40E942E66C2
:107AC800E0810E947F6E563051F40E944E660E94FB
:107AD80094640E941763ABEEB7E00E94D5615730FB
:107AE80039F4A0911905E2E0EA9FF0010E948C6E3A
:107AF800583021F4E09133050E947F6E593029F403
:107B08000E941366E0810E947F6E5A3029F40E9419
:107B18004366E0810E947F6E5B3021F40E94916E83
:107B28000E947F6E5C3021F40E9468690E948C6E0E
:107B38005D3021F40E94AC630E948C6E5E3021F4AB
:107B48000E9485670E948C6E5F3021F40E948569CF
:107B58000E948C6E503121F40E944F640E94986EEE
:107B6800513121F40E943D640E94986E523121F4F3
:107B78000E9497690E94986E533129F40E945764B5
:107B8800E0810E947F6E543121F4E09153050E94F8
:107B98007F6E553121F4E0911D050E947F6E5631AC
:107BA80021F4E0911C050E947F6E573121F4E09189
:107BB8001E050E947F6E583121F4E09100070E9453
:107BC8007F6E593121F40E9475660E948C6E5A317D
:107BD80019F4E9A50E947F6E5B3119F4EB890E94C4
:107BE8007F6E5C3119F4EC890E947F6E5D3121F45F
:107BF8000E94E1610E948C6E5E3121F40E94DD6971
:107C08000E948C6E5F3121F4E09107050E947F6E1F
:107C1800503229F40E94F869E0810E947F6E513247
:107C280029F40E94016AE0810E947F6E523229F491
:107C38000E94076AE0810E947F6E533229F40E94F5
:107C48000D6AE0810E947F6E543229F40E94136A03
:107C5800E0810E947F6E553219F4EB8D0E947F6E91
:107C6800563219F4EA8D0E947F6E573219F4E98D65
:107C78000E947F6E583219F4E88D0E947F6E593247
:107C880021F4E0913B050E947F6E5A3221F4E09185
:107C980034050E947F6E5B3231F4E0910508F09163
:107CA80006080E948C6E5C3219F4EA890E947F6E85
:107CB8005D3251F40E946A610E941B750E9417632D
:107CC800ABEEB7E00E94D5615E3221F40E94F0620B
:107CD8000E948C6E5F3221F4E09120070E947F6E33
:107CE800503321F4E09115050E947F6E513319F449
:107CF800EC850E947F6E533319F4ED890E947F6EE4
:107D0800543321F4E0914F050E947F6E553321F4DE
:107D1800E09150050E947F6E563321F4E0915105A1
:107D28000E947F6E573331F4E0913905F0E03196C7
:107D38000E948C6E583319F4ECA50E947F6E59335B
:107D480021F40E948F650E948C6E5A3319F4EAA5BB
:107D58000E947F6E5B3321F4E091F0050E947F6EF4
:107D68005C3321F4E09135050E947F6E5D3321F488
:107D7800E09101050E947F6E5E3321F4E091BE051B
:107D88000E947F6E5F3321F40E94F4650E948C6E1E
:107D9800513421F4E091FB060E947F6E523421F4A5
:107DA800E091FC060E947F6E533419F4EE890E941C
:107DB8007F6E543421F40E948F640E948C6E553477
:107DC80021F4E09154050E947F6E563421F40E94FC
:107DD80079630E948C6E573419F4EF8D0E947F6E80
:107DE800583421F4E0910B070E947F6E593421F436
:107DF800E0910C070E947F6E5A3421F4E091C80587
:107E08000E947F6E5B3439F40E9443660E94496683
:107E1800E0810E947F6E5A3531F40E94B8650E9455
:107E28009C6E0E948C6E5C3521F4E09106050E94E0
:107E38007F6E0E94646A0E94BB6621F0E091F205A1
:107E48000E947F6E0E94646A0E94746321F0E09130
:107E5800F3050E947F6E503621F40E946D6A0E94DD
:107E68008C6E513621F4E091F1050E947F6E5236F6
:107E780029F40E949768EC910E947F6E0E94726AB2
:107E88000E94BB6619F0E8A50E947F6E0E94726A84
:107E98000E94746319F0EEA10E947F6EA52F0E94C4
:107EA800065EA52FEEE00E94A16EEFE00E94F1763B
:107EB800E0291E2EA52FE9E10E94F1760E2E0E94E0
:107EC800A66EEBEFF0E00E942C77E021E1290E2E60
:107ED800A52FEDE10E94A16EEBE20E94A16EEEE2F9
:107EE8000E94A16EE8E30E94A16EE9E30E94A16EE0
:107EF800EFE30E94F176E0291E2E0E94A9650E2E5E
:107F08000E94BB5D0E94BE61E0211E2A0E94A965F5
:107F18000E2E0E94CF650E94BE610E94AB6EE5E006
:107F28000E94B56EE8E00E940A770E94AB6EE0E01E
:107F38000E94B56EE3E00E940A770E94AB6EE4E00F
:107F48000E94F1760E94AB6EEDE00E94B56EE1E111
:107F58000E940A77E021E12911F0F59A01C0F5980D
:107F6800A0E0F599A1E0EA2FE795E0E0E7950E9407
:107F7800BB6EA52FB0E0A7FDBFEF0E94BB670E94B4
:107F8800766BE0932B07A52FB0E0A7FDBFEF0E940B
:107F98007C6BE0932C07A52FE1E00E94C56EE7E01B
:107FA8000E940077E0211E2EA52FE8E00E94C56EF2
:107FB800ECE00E940077E021E1290E2EA52FE3E1F5
:107FC8000E94F176E02971F1A09125070E94A85F2F
:107FD800A09125070E94E56A99F0E0915D07EC5FA2
:107FE800E0935D07A0912507A43051F4A0E0F7992C
:107FF800A1E00E940C6BA0E0F799A1E00E94136B2E
:10800800A0912507A23029F4E0915D07EE5FE09387
:108018005D07A0912507A33029F4E0915D07EF5F84
:10802800E0935D070E94A66EA031E7E2BE0730F03C
:108038000E94A66E0E94CA6EE09333070E94A66E45
:10804800A83EE3E0BE0730F00E94A66E0E94B46B23
:10805800E09334070E94D06E30F00E94A66E0E9412
:108068009A6CE09335070E94A66E1A9720F00E943A
:10807800D56EE09336070E94D76EE09337075030ED
:1080880049F5ECE10E94D96EE0E5E0932F07E8811D
:10809800E03049F4EEE5E0933207E5E0E09333079A
:1080A800E3E7E0933407A881A13028F00E94C76C69
:1080B800E881E09334070E94D56EE0933607E881A3
:1080C800F0E031970E94DF6EA8810E948B6611F064
:1080D8000E94E46E513079F4EBE50E94D96EEDE62A
:1080E8000E94EA6E11F40E94F26E0E94A66E119729
:1080F80011F40E94FB6E523031F4EDE60E94026FDB
:10810800E8E3E0932F07533009F04DC0E9E30E94FC
:10811800086FE8E3E0932F07A0917107A43628F0D1
:10812800B0E00E946C6BE0933107A0917107AA3010
:1081380038F0B0E00E94BB670E94766BE09332078C
:10814800A0917107BB270E947C6B0E940E6F0E9452
:10815800146FE0933507A0917207AA3058F0B0E089
:108168000E94BB670E94766BE09335070E94146FEC
:10817800E0933607EAE0E0933707A0917207A43648
:1081880090F0B0E00E946C6BE0933507A091720705
:10819800B0E00E94BB670E94766BE09336070E94AE
:1081A800146FE0933707543049F4E7E30E94186FDF
:1081B800E1E70E94EA6E11F40E94F26E553049F42C
:1081C800E3E7E0932D07ECE1E0932E07E0E5E09389
:1081D8002F07563091F4ECE70E941E6FE9E3E09315
:1081E8002F070E94A66E1A9720F00E94D56EE09382
:1081F80035070E94D76E0E94246F5730F1F4E3E7E9
:10820800E0932D07E4E7E0932E07E9E3E0932F07D7
:108218000E94D06E30F00E94A66E0E949A6CE09385
:1082280034070E94A66E1A9720F00E94D56EE0933C
:1082380035070E94D76E0E94246F5830A1F4EEE3F0
:108248000E942A6FE5E0E0932F07E0913305E030C4
:1082580019F4E2E00E94306FA0913305A13019F4BF
:10826800E4E00E94306F593031F4E7E7E0932E07DD
:10827800E5E0E0932F075A30F1F50E94396FE4E505
:108288000E94EA6E79F4EEE3E0933107E0E00E94A1
:10829800946CE8E7E0933407E7E7E0933507EDE30C
:1082A8000E94406F0E94A66E119779F4E9E3E0936B
:1082B8003107EEE3E0933207E0E50E94466FE9E715
:1082C8000E944C6FE8E7E09337070E94A66E12976A
:1082D80011F40E94526F0E94A66E139761F4E6E7AC
:1082E800E0933107EBE50E945C6FE7E30E94626F61
:1082F800EEE50E94406F5B3031F5EDE60E94686F55
:10830800EDE30E94EA6E79F4EDE6E0933207E7E6E2
:10831800E0933307EEE3E0933407E7E7E0933507AC
:10832800E0E50E94406F0E94A66E119761F4EDE6A9
:10833800E0933307E0E30E946E6FEEE3E0933607C5
:10834800EDE6E09337075C30C1F4EEE30E94746F0A
:10835800ECE7E0932F07EEE3E09334070E94A66E64
:108368001A9720F00E94D56EE09336070E94D76EC8
:10837800E0933707E0E2E0935D07A52FEDE10E9467
:108388007A6EEEE20E94F176E02921F00E94D56E25
:10839800E09336075D30B9F40E949C6A0E945163ED
:1083A8000E94D76BE0932D070E947A6F0E94D76BCB
:1083B800E0932E070E947A6F0E94EB77E0932F07D5
:1083C800E0E2E0935D075E3031F4EEE3E0932D07E1
:1083D800ECE00E94806F5F3031F4EEE3E0932D070C
:1083E800EBE00E94806F503121F5ECE70E94866F28
:1083F800ECE0E09333070E948C6FA436E0E0BE0700
:1084080034F00E948C6F0E946C6BE0932D070E94E1
:108418008C6F1A9744F00E948C6F0E94BB670E9471
:10842800766BE0932E070E948C6F0E947C6BE09322
:108438002F075131F1F40E94916FECE00E94986F80
:1084480034F00E94A26F0E946C6BE0932D070E948B
:10845800A26F1A9744F00E94A26F0E94BB670E9405
:10846800766BE0932E070E94A26F0E947C6BE093CC
:108478002F075231F1F40E94916FEBE00E94986F40
:1084880034F00E94A26F0E946C6BE0932D070E944B
:10849800A26F1A9744F00E94A26F0E94BB670E94C5
:1084A800766BE0932E070E94A26F0E947C6BE0938C
:1084B8002F07533111F5E8E30E94686FE7E70E9440
:1084C800EA6E11F40E94A76F0E94AF6F48F4E8E3C8
:1084D800E0933307E0E0E0933407EDE3E0933507FA
:1084E8000E94A66E1A9748F0E8E3E0933207E0E0AE
:1084F800E0933307EDE30E944F6E5431C1F4E8E393
:108508000E94686FECE70E94EA6E59F40E94636C5F
:10851800E4E5E0933407EEE5E0933507E0E50E94F3
:10852800B36F0E94A66E119711F40E94A76F553180
:10853800B9F40E94B96FECE00E94C36F11F40E9475
:10854800F26E0E94AF6F60F40E94A66E1A9720F038
:108558000E94D56EE09335070E94D76E0E94CB6FBC
:108568005631B9F40E94B96FEBE00E94C36F11F461
:108578000E94F26E0E94AF6F60F40E94A66E1A9776
:1085880020F00E94D56EE09335070E94D76E0E94B6
:10859800CB6F573129F40E94B96FE0E4E0933107BB
:1085A800583149F40E94396F0E94D16F0E94D06EF1
:1085B80011F40E94F26E593189F4E5E00E94026FCD
:1085C8000E94D16F0E94D56EE09336070E94A66E76
:1085D800AB3FE0E0BE0710F00E94F26E5A3171F432
:1085E8000E94D86FEEE30E94EA6E11F40E94FB6EBF
:1085F8000E94A66E119711F40E94F26E5B3129F465
:108608000E94D86FEEE0E0932F075C3149F4E9E36C
:108618000E942A6FEAE00E94EA6E11F40E94F26E4C
:10862800A52FEDE10E947A6EEEE10E94F176E02935
:10863800E9F0E3E7E0933107E8E3E09332075D31DF
:1086480011F4EEE501C0E8E7E09333070E94DF6F1D
:108658001A9730F00E94DF6F0E94876CE0932E0714
:108668000E94DF6F0E94D26BE0932F075F3149F4BD
:10867800E8E3E0932D07EDE6E0932E07E3E7E093C8
:108688002F07A52FEFE10E94C56EE5E20E94007753
:10869800E02109F435C1EDE60E94E46FE52FEF51C2
:1086A8000E94EA6E61F4E1E0E0933207EDE3E093C3
:1086B8003307E4E50E94626FE0E50E94406F0E9484
:1086C800A66E119711F40E94EA6F0E94A66E129787
:1086D80049F4E0E0E0933507EEE5E0933607E0E0A3
:1086E800E09337070E94A66E139761F4E7E3E093DF
:1086F8003207E7E7E0933307E4E70E94626FE5E0BB
:108708000E94B36F0E94A66E149721F40E94F76F1F
:108718000E94FC6F0E94A66E159711F40E940170CA
:108728000E94A66E169711F40E94FC6F0E94A66E16
:10873800179759F4E7E7E0933207E9E3E093330743
:108748000E944F6EECE70E940B700E94A66E18976D
:1087580049F4E3E70E94946CE7E70E946E6FEAE051
:108768000E94B36F0E94A66E199721F40E94F76FBA
:108778000E94FC6F0E94A66E1A9711F40E94017065
:108788000E94A66E1B9761F4E9E3E0933307E8E3E0
:108798000E944F6EE7E7E0933607ECE7E093370770
:1087A8000E94A66E1C9711F40E94526F0E94A66E3A
:1087B8001D9729F4E7E30E9411700E9415700E942A
:1087C800A66E1E9729F4ECE70E9411700E9415709E
:1087D8000E94A66E1F9729F4E9E30E9411700E9477
:1087E80015700E94A66E509711F40E941F700E9487
:1087F800A66E519729F40E942770E1E0E0933707AD
:108808000E94A66E529729F40E942770E2E0E09336
:1088180037070E94A66E539731F4E0E5E0933507D9
:10882800E3E70E942E700E94A66E549779F4E8E759
:10883800E0933207E0E5E0933307E1E0E0933407A3
:10884800E3E70E943470E2E0E09337070E94A66EE7
:10885800559731F4E9E7E0933507E0E50E943A706F
:108868000E94A66E569761F4E5E0E0933207E3E7CD
:108878000E944070E9E7E0933507EEE50E943A7000
:108888000E94A66E579761F4E5E00E94256DE9E71E
:108898000E944070EEE50E944C6FEDE0E0933707D0
:1088A8000E94A66E589749F4E3E70E94946CE7E7A4
:1088B8000E946E6FEAE00E9446700E94A66E599769
:1088C80061F4E1E0E0933207ECE7E0933307E7E790
:1088D8000E94116EE8E70E943A700E94A66E5A97AD
:1088E80079F4E8E7E0933207E1E0E0933307E4E561
:1088F800E0933407E9E7E0933507EAE00E942E7039
:10890800553249F4EAE00E94E46FE5E00E94EA6E1D
:1089180011F40E94F26E563249F4EAE00E94E46FC4
:10892800E8E00E94EA6E11F40E94F26E573241F4B8
:108938000E944C70E0E00E94EA6E11F40E94F26E10
:10894800583241F40E944C70E4E00E94EA6E11F43F
:108958000E94F26E593231F4E0E00E94186FE8E7A5
:10896800E0932F075A32F1F5ECE70E945370E0913B
:108978003405E03049F40E945C700E945C6FEDE0C1
:108988000E944F6E0E946170A0913405A13031F4AD
:108998000E9468700E946F700E946170A0913405F7
:1089A800A23041F40E945C70E09332070E946F701D
:1089B8000E946170A0913405A33039F40E94687058
:1089C800EAE00E940E6F0E947470A0913405A430F2
:1089D80049F40E945C70E0933207E2E00E940E6F57
:1089E8000E9474705B3269F4ECE70E94746FE8E7E8
:1089F800E0932F070E94D56EE0933607E0E2E093FC
:108A08005D075C32C9F4ECE70E947E7041F4E4E54E
:108A1800E0933207E0E00E949C6B0E9484700E9401
:108A2800A66E119749F4E0E50E944070E5E0E093F6
:108A38003507E9E70E94B36F5D3259F4E0915B07AF
:108A4800E05CE0935B07E0E00E942A6FE0E0E093DF
:108A58002F075E3231F4E9E3E0932D07E8E30E9443
:108A6800806F5F32B9F5E8E70E941E6FE5E00E946B
:108A7800EA6E11F40E94F26E0E94A66E119711F42C
:108A88000E941F700E94A66E129711F40E94EA6F4E
:108A98000E94A66E139791F4E8E7E0933107E1E0AE
:108AA800E0933207E4E5E0933307EDE00E94116EAE
:108AB800E0E5E0933607E3E7E09337070E94A66E08
:108AC800149741F4E8E70E94866FE3E70E949C6BE5
:108AD8000E948470503361F4E9E70E947E7011F4BB
:108AE8000E94FB6E0E94A66E119711F40E94F26E0E
:108AF8005133B1F4E3E7E0932D07E0E50E94897074
:108B0800A0910305A43160F0E4E5E0933107EDE6B8
:108B1800E0933207E0E3E0933307EDE3E0933407B3
:108B28005233B1F5EDE60E948F70E3E6E0932F072C
:108B3800EF89E03061F4EEE5E0933407E0E3E09399
:108B48003507EDE6E0933607E3E7E0933707AF89AB
:108B5800A13049F4E7E3E0933307ECE50E94116E96
:108B6800ECE50E940B70AF89A23031F4ECE7E0939A
:108B78003507E7E70E94B36FAF89A33049F4E9E30B
:108B8800E0933307ECE50E946E6FE8E70E940B70F4
:108B9800533369F5E7E7E0932D07E0E40E94897015
:108BA800ED89E03019F4E7E7E0933707AD89A130A4
:108BB80031F4E7E7E0933507E0E40E94B36FAD894D
:108BC800A23079F4E7E7E0933107E0E4E093320775
:108BD800E8E70E949C6BE6E70E944C6FEEE5E093A5
:108BE8003707AD89A33019F4E8E7E0933707543322
:108BF80069F4E8E70E948F700E94B36C0E94A66E29
:108C0800A338E0E0BE0711F40E94F26E553369F410
:108C1800E8E70E948F700E94BD6C0E94A66EA73480
:108C2800E0E0BE0711F40E94F26E563369F4E8E7FB
:108C38000E948F700E94C76C0E94A66EA536E0E065
:108C4800BE0711F40E94F26E5733A9F4E4E5E093ED
:108C58002D07E9E30E948970A091C705E1E00E9411
:108C6800F6760E2EA0E0F799A1E00E94BB6619F0F7
:108C7800EAE0E0933707583331F4EEE50E94686F75
:108C8800E7E7E0932F075933F9F4A091AD08AA2339
:108C98002AF4E0E0E093AC08E093AD080E94946504
:108CA800A436E0E0BE0724F00E94286BE0932D076D
:108CB8000E94336B0E94766BE0932E070E949465A6
:108CC8000E947C6BE0932F075A3331F4E7E3E0937B
:108CD8002D07E9E30E9495705B3341F4E5E00E94BB
:108CE8005370E091F005EF5FE09337075C3399F438
:108CF800E6E70E94186FEAE00E94EA6E61F4E7E78F
:108D0800E0933407ECE1E0933507E8E7E0933607B2
:108D1800ECE5E09337075D3339F5E0E00E94CF5D7D
:108D28000E94D16CE8E7E0932D07E1E0E0932E077D
:108D3800E4E5E0932F070E949B700E94A86BA09126
:108D48000105AA3018F0E2E0E09330070E948E6A2D
:108D5800E09331070E94586A0E94766BE0933207CD
:108D68000E945C6AE09333075E3301F5E0915C078B
:108D7800E061E0935C07E8E3E0932D07E9E3E09323
:108D88002E07EEE5E0932F07E1E0E0933107A0918D
:108D9800BE05E3E0EA1BE0933207ECE7E093340713
:108DA800E1E0E0933507E7E70E9446705F3349F456
:108DB800E1E70E94186FEAE0E0932F07E0E6E0930E
:108DC8005D07503449F5E9E3E0932D07E0E0E093CF
:108DD8002E07EEE5E0932F07A091F606B0E00E947B
:108DE800BB670E94766BE0933407A091F606BB2719
:108DF8000E947C6BE0933507A091F706B0E00E94D3
:108E0800BB670E94766BE0933607A091F706B0E047
:108E18000E947C6BE09337075134E9F4E4E70E9441
:108E2800746FE1E00E94EA6E61F4E4E50E940B6E63
:108E3800E4E50E949C6BE1E00E944C6FECE1E0935A
:108E480037070E94A66E119731F4E1E00E944C6F3B
:108E5800ECE1E0933707523401F5E4E70E94746FC0
:108E6800E3E60E94EA6E61F4E4E70E945C6FE1E0E9
:108E7800E0933407E2E00E94A26BE3E6E093370751
:108E88000E94A66E119749F4E4E70E949C6BE6E005
:108E98000E94A26BE3E6E0933707533469F5EDE6E9
:108EA800E0932D07E8E30E948970EE89E03091F4A1
:108EB800E8E7E0933207EEE6E0933307E8E0E09373
:108EC8003407E1E0E0933507EDE0E0933607E1E0B1
:108ED800E0933707AE89A13079F4E8E3E0933307EC
:108EE800E7E3E0933407E3E0E0933507E5E0E09358
:108EF8003607EEE5E0933707543409F5EFA5F8A9EE
:108F08000E94456BA8A9AA2342F4E0916808F09151
:108F180069080E947B760E94456B0E944A6B0E94FA
:108F28006C6BE0932D070E944F6B0E94766BE09369
:108F38002E070E944A6B0E947C6BE0932F075534E2
:108F4800B9F4E0E3E0932D07EDE6E0932E07E4E5BE
:108F58000E94EA6E19F4E1E00E942E700E94A66E4B
:108F6800119731F4E0E0E0933507EEE30E94B36F28
:108F78005634A9F40E94A1700E949A6CE0932D07C0
:108F88000E94A1700E94876CE0932E070E94A17036
:108F98000E94D26B0E94EA6E11F40E94F26E57345E
:108FA800C1F4E8E70E94746FE4E70E94EA6E11F4E6
:108FB8000E94F26E0E94AF6F60F40E94A66E1A972C
:108FC80020F00E94D56EE09335070E94D76E0E946C
:108FD800CB6F583449F4E7E70E948F70E4E50E94AC
:108FE800EA6E11F40E94F26E593409F040C0EAE0CA
:108FF8000E94186FE4E50E94EA6E31F4EEE30E94E5
:10900800626FE8E30E94B36F0E94A66E119759F44D
:10901800E3E70E94866F0E94A670EAE0E0933607B5
:10902800EEE3E09337070E94A66E129741F4E3E758
:109038000E94866F0E94A670EEE30E940B700E9449
:10904800A66E139741F4E3E70E94866F0E94A6700C
:10905800E4E50E94246F0E94A66E149741F4E3E7AA
:109068000E94866F0E94A670EEE30E94B36F5A3486
:1090780091F4E8E7E0932D07E0E5E0932E07E5E0BB
:109088000E94EA6E11F40E94F26E0E94A66E119779
:1090980011F40E94FB6E5B3431F4E9E30E94026F25
:1090A800E1E0E0932F075A3509F05BC0E0E50E9444
:1090B8008F70E0E0E0932F07A091CA050E940F7718
:1090C8001E2E0E94C5650E94CF650E94BE61E021E8
:1090D800E12971F0E091AF070E940B6E0E94D56EF6
:1090E800E0933607E091CA05E150E093CA0539C01C
:1090F8000E94BE65E093C907F093CA070E94286BD7
:10910800E09331070E94336B0E94766BE09332073D
:109118000E94AB700E949A6CE09335070E94AB7076
:109128000E94876CE09336070E94AB700E94D26B56
:10913800E09337070E94C5650E94CF650E94D465F9
:1091480081F0F79B08C0EAE0E0933507E3E2E0939B
:109158003607E4E504C0EAE00E944C6FE3E2E093DE
:1091680037075B3509F042C0E8E7E0932D07E5E0F3
:109178000E948970A0914108A03044F0E091410814
:10918800F0E0E7FDFFEF0E948C6E30C0E0914108EF
:10919800F0E0E7FDFFEF0E947B760E948C6E0E9454
:1091A800A66E0E94C05D0E94A66EEAE0F0E00E94F2
:1091B8002C77E02119F0EDE0E09336070E94A66EC7
:1091C800E9E0F0E00E9432770E2E0E94A66EE4E6F7
:1091D800F0E00E942C77E02119F0EDE0E0933507EC
:1091E8000E94D06E18F0EDE0E09334075C3529F466
:1091F8000E94396FE9E3E0932F075D3509F038C322
:10920800A0915E07A83008F043C0E7E70E942A6FE4
:10921800E0915E070E94B0700E94B55D0E949C6E4E
:10922800E83EA3E0FA074CF00E94B5700E949C6EDD
:10923800DF010E946A6CE09334070E94B5700E94B7
:109248009C6EE436A0E0FA0754F00E94B5700E94C4
:109258009C6E0E9434660E94766BE09335070E94EC
:10926800B5700E949C6E3A975CF00E94B5700E949F
:109278009C6EDF010E94BB670E94766BE093360705
:109288000E94B5700E949C6E0E94766BE09337072F
:109298000E94B97049F1E6E70E948F70E0915E077D
:1092A800E750E0932F07E7E7E0933107ECE7E09317
:1092B8003207E9E3E09333070E94C470E170E0935A
:1092C80035070E94C470E695E170E09336070E9466
:1092D800C470E695E6950E94CC7038970E94D370CA
:1092E80019F4EDE00E94D8700E94DB70D1F1E1E042
:1092F800E0932D07E4E50E94E670EB500E94B07001
:109308000E94EB70E170E09332070E94F170E695DD
:10931800E170E09333070E94F170E695E695E170FD
:10932800E09334070E94F1700E94F470E0933507CF
:109338000E94F170E295E170E09336070E94F170A7
:10934800E295EF70E6950E94CC703C970E94D3702E
:1093580041F4EDE0E09332070E940E6FEDE00E94C9
:10936800D8700E94F970B9F10E940171EEE30E9471
:109378000771EF500E94E6700E940C71E83EA3E06E
:10938800FA0738F00E941371DF010E94B46BE09372
:1093980034070E941371E436A0E0FA0738F00E94FF
:1093A8001371DF010E949A6CE09335070E941371D4
:1093B800DF010E94876CE09336070E941371DF017A
:1093C8000E94D26B0E94167170970E94D37019F494
:1093D800EAE00E94D870A0915E07E3E10E941C7148
:1093E800E8E10E940A77E02109F45EC00E94017159
:1093F800E7E70E940771E3510E94E6700E9422711C
:10940800FF231AF10E942971DF010E946A6C0E94F1
:109418002C7119F4EAE0E09334070E9429710E9444
:1094280034660E94766B0E949E6D19F4EAE0E09320
:1094380035070E942971DF010E94BB670E94766B85
:10944800E09336070E94297120C0EDE0E0933507CC
:109458000E942971ED39AFEFFA075CF4EDE0E09373
:1094680034070E9429710E9432710E94766BE09342
:1094780035070E9429710E943D6B0E94766BE0932C
:1094880036070E9429710E947B76DF010E947C6B5F
:10949800E0933707E0915E07F0E074970E94D3707D
:1094A80019F4EAE00E94D870A0915E07E7E10E94F3
:1094B8001C71ECE10E940A77E02109F46AC0E7E731
:1094C800E0932D07E1E70E94E670E7510E94B07033
:1094D8000E943671FF23FAF00E943D710E943466A3
:1094E8000E94766B0E949E6D19F4EAE0E0933507BE
:1094F8000E943D71DF010E94BB670E94766B0E944B
:10950800407119F0EAE0E09336070E943D710E942D
:10951800766BE09337070E943D71FF236AF5EDE013
:10952800E09336070E943D71ED39AFEFFA075CF41E
:10953800EDE0E09334070E943D710E9432710E9471
:10954800766BE09335070E943D71E73FAFEFFA076E
:109558005CF4EDE0E09335070E943D710E943D6B9D
:109568000E94766BE09336070E943D710E947B76DD
:109578000E94766BE0933707E0915E07F0E07897FA
:109588000E94D37031F4EAE00E944F6EEAE00E9434
:109598003A70A0915E07EBE10E941C71E8E20E941C
:1095A8000A77E02109F4BCC0A0915E07A03268F4F4
:1095B800E7E30E940771EB510E94B070EC51A3E001
:1095C800EA02F001EF5FE0930907A0915E07EFE17F
:1095D8000E941C71E4E20E940A77E02169F0ECE73E
:1095E8000E940771EF510E94B070E052A3E0EA02B6
:1095F800F001EE5FE0930907A0915E07A43268F0DE
:10960800E9E30E940771E3520E94B070E452A3E0BC
:10961800EA02F001ED5FE0930907E8E7E0932E071F
:109628000E944C71FF2302F10E944C710E94346623
:109638000E94766B0E942C7119F4EAE0E0933407DB
:109648000E944C71DF010E94BB670E94766B0E94EA
:10965800547119F0EAE0E09335070E944C710E94BA
:10966800766BE09336072DC00E944C710E947B7682
:109678000E94766BE0933607EDE0E09335070E9491
:109688004C71E73FAFEFFA075CF40E944C710E94FF
:109698003D6B0E94766BE0933507EDE0E09334076D
:1096A8000E944C71ED39AFEFFA075CF40E944C71DF
:1096B8000E9432710E94766BE0933407EDE0E093EC
:1096C8003307E3E60E941671BF017C970E94DF6EA4
:1096D800A0915E07E0E20E940A77E0211E2EFB01BE
:1096E800B0970E94DF6EA0915E07EFE10E940F77AE
:1096F8000E22E4E20E940A77E0211E2AFB01B497B9
:109708000E94DF6EA0915E07E3E20E940F77E021DE
:10971800E12931F0EAE00E944F6EEDE0E093360770
:10972800A0915E07E7E20E941C71ECE20E940A77B2
:10973800E02191F1E3E70E94186FE0915E07E7529C
:109748000E94B0700E9460710E946C6B0E949E6DB6
:1097580019F4EAE0E0933507E0915E070E94607132
:109768000E94BB670E94766B0E94407119F0EAE084
:10977800E0933607E0915E070E9460710E947C6B5F
:109788000E941671B8970E94D37031F4EAE00E94E3
:109798003470EDE0E09337070E9467710E946B71A7
:1097A80099F1E3E7E0932D07E6E70E94E670EB52B4
:1097B8000E94B0700E9470710E946C6B0E949E6D36
:1097C80019F4EAE0E0933507E0915E070E947071B2
:1097D8000E94BB670E94766B0E94407119F0EAE014
:1097E800E0933607E0915E070E9470710E947C6BDF
:1097F8000E941671BC970E94D37031F4EAE00E946F
:109808003470EDE0E09337070E9477710E947B7116
:1098180079F10E940171EEE3E0932D07E6E70E94DB
:10982800E670EF520E94B0700E948071DF010E94C2
:109838009A6C0E949E6D19F4EAE0E0933507E09176
:109848005E070E948071DF010E94876CE0933607F3
:10985800E0915E070E948071DF010E94D26B0E9436
:109868001671F0970E94D37019F4EAE00E94D8703C
:109878005E3509F088C2EDE60E941E6FE7E7E093C7
:109888002F07E0914D05E03029F5EDE60E94256DA2
:10989800EBE0E0933307A0915009B0E00E946C6BB5
:1098A8000E949E6D19F4EAE0E0933507A0915009F3
:1098B800B0E00E94BB670E94766B0E94407119F06D
:1098C800EAE0E0933607A0915009BB270E947C6B21
:1098D800E0933707A0914D050E94A85FA0914D0520
:1098E800E2E00E94F176E02939F10E944F6DA091E3
:1098F8004D05E2E00E945A6D11F00E94646DE5E0AA
:109908000E94256DA0914D05A23019F4E4E5E0937D
:109918003207E0E40E946F6D0E949A6C0E949E6D6F
:1099280019F4EAE0E09335070E94766D0E94876C8F
:109938000E947B6DE0933707A0914D05A330A9F4F1
:109948000E948F6DEBE0E09332070E94EE5F0E9469
:109958009A6C0E949E6D19F4EAE0E09335070E9424
:10996800EE5F0E94876C0E94246FA0914D05A43081
:10997800C9F40E9490600E945C7810F40E94846D83
:109988000E948F6D0E94966D0E949E6D19F4EAE008
:10999800E09335070E94A46D0E94876C0E94A96D10
:1099A800E0933707A0914D05A53021F5E2E0E0935B
:1099B80030070E948771A0915109B0E00E946C6B3A
:1099C8000E942C7119F4EAE0E0933407A091510940
:1099D800B0E00E94BB670E94766B0E94547119F038
:1099E800EAE0E0933507A0915109BB270E947C6B00
:1099F8000E94246FA0914D05A630B9F40E94106D05
:109A0800ECE0E09333070E94B25F0E949A6CE09307
:109A180035070E94B25F0E94876CE09336070E9468
:109A2800B25F0E94D26BE0933707A0914D05A73033
:109A3800B9F40E94106DEBE0E09333070E94BC5F1D
:109A48000E949A6CE09335070E94BC5F0E94876C65
:109A5800E09336070E94BC5F0E94D26BE093370701
:109A6800A0914D05A830E1F50E9487710E94C65F5C
:109A78000E946A6CE0933307E0913307E03019F4F1
:109A8800EAE0E09333070E94C65F0E946C6BE093A4
:109A980034070E948E710E94746319F0EAE0E09323
:109AA80034070E94C65F0E94BB670E94766BE093F2
:109AB80035070E948E71EAE00E94F1760E22A0918D
:109AC80035070E94746319F0EAE0E09335070E94B5
:109AD800C65F0E947C6BE0933607EEE3E09337079E
:109AE800A0914D05A930F1F40E94B36C0E94D05F9B
:109AF800A436E0E0BE0730F00E94D05F0E949A6C66
:109B0800E09334070E94D05F1A9730F00E94D05F2C
:109B18000E94876CE09335070E94D05F0E94D26B49
:109B28000E949771A0914D05AA30F1F40E94BD6C76
:109B38000E94DA5FA436E0E0BE0730F00E94DA5FE8
:109B48000E949A6CE09334070E94DA5F1A9730F00B
:109B58000E94DA5F0E94876CE09335070E94DA5F03
:109B68000E94D26B0E949771A0914D05AB30F1F421
:109B78000E94C76C0E94E45FA436E0E0BE0730F0A4
:109B88000E94E45F0E949A6CE09334070E94E45FAD
:109B98001A9730F00E94E45F0E94876CE0933507C3
:109BA8000E94E45F0E94D26B0E949771A0914D05BC
:109BB800AC30A1F5E7E7E0933107E1E7E09332073E
:109BC8000E943E600E94E26B24F00E943E600E9468
:109BD800166C0E943E600E94EF6B24F00E943E606B
:109BE8000E94246C0E943E600E94FC6B44F00E941C
:109BF8003E600E94D26A0E94326CE09335070E9450
:109C08003E600E94866A34F00E949D710E94426CF8
:109C1800E09336070E949D710E94456CA0914D0506
:109C2800AD30B9F5E7E70E94866F0E94995FA031D1
:109C3800E7E2BE0730F00E94995F0E94CA6EE09387
:109C480033070E94995FA83EE3E0BE0730F00E9408
:109C5800995F0E94B46BE09334070E94995FA43621
:109C6800E0E0BE0730F00E94995F0E949A6CE09392
:109C780035070E94995F1A9730F00E94995F0E94F9
:109C8800876CE09336070E94995F0E94D26BE0933D
:109C98003707A0914D05AE3031F5EEE3E09331077B
:109CA800E1E7E09332070E9450600E94EF6B24F0D6
:109CB8000E9450600E94246C0E9450600E94FC6BBD
:109CC80044F00E9450600E94D26A0E94326CE09375
:109CD80035070E94A4710E94426CE09336070E94E7
:109CE800A4710E94456CA0914D05AF3039F5EEE3A3
:109CF8000E94866F0E945E60A83EE3E0BE0730F0D7
:109D08000E945E600E94B46BE09334070E945E601C
:109D1800A436E0E0BE0730F00E945E600E949A6CB4
:109D2800E09335070E945E600E94876CE0933607D7
:109D38000E945E600E94D26BE0933707A0914D05A8
:109D4800A03189F40E94356D30F00E94466D0E9462
:109D58009A6CE09335070E94466D0E94876C0E94BA
:109D68004B6DE0933707A0914D05A13161F40E9436
:109D7800AD6D18F0E1E0E09330070E94C16D0E94DC
:109D8800D16D0E94F36D5F35C1F4E8E30E94D96E8E
:109D9800EEE5E0932F07F6FC03C0ECE0E093310713
:109DA800F6FE03C0EBE0E0933107E091EB07F0919A
:109DB800EC07309711F40E94F26E503631F4E8E364
:109DC8000E942A6FEDE0E0932F07513649F4E3E74C
:109DD8000E94086FEAE00E94EA6E11F40E94F26E97
:109DE800523651F4E8E3E0932D07E0911B05E09328
:109DF8002E07E0E1E0935D07533669F4E8E30E943B
:109E0800086FF6FC03C0ECE0E0932F07F6FE03C0F2
:109E1800EBE0E0932F07A0E0F099A1E00E94065E36
:109E2800A92D0E940B5EA09137050E94E06AA1F15E
:109E3800E0E00E94BB6EE89430F80E94EA6AE0E035
:109E4800E0933207E1E7E09333070E944F6E0E94E8
:109E58009B70A0913705A130F8F0A13319F4E1E027
:109E6800E0932B05A0913705A03319F4E0E0E093C7
:109E78002B05A0913705AC3219F4E1E0E0932B05EE
:109E8800A0913705AD3219F4E0E0E0932B05E0919D
:109E98003705E150E0933705A0913705E8E20E94C5
:109EA8000A770E2EE0E00E940F770E22A52DE2E33E
:109EB8000E940F77E02109F02998A091FA06A130B5
:109EC80081F5E0E00E94BB6E0E94AB710E94B37105
:109ED800EAE0E0933007E3E7E0933107A091F80662
:109EE800B0E00E94BB670E94766BE0933207A091B6
:109EF800F806B0E00E947C6BE0933307A091F90666
:109F0800B0E00E94BB670E94766BE0933407A09193
:109F1800F906B0E00E947C6B0E943470EAE0E0939E
:109F28003707A0916907A130C9F4E0E00E94BB6E31
:109F38000E94AB710E94B371EAE0E0933007E8E356
:109F48000E940B6EE7E7E0933307EEE5E0933407F2
:109F5800E1E00E944C6FEDE3E0933707A0E031FCAD
:109F6800A1E00E94A85F0E94FB65E02171F0E1E793
:109F7800E0933107E8E3E0933207E5E0E093330745
:109F8800E6E70E944F6E0E945C6EE1E0E0932707CF
:109F9800A0912707A03108F08AC00E94746EE08162
:109FA800E03021F40E94746EAFE3A0830E94746EC7
:109FB800A081A63021F40E94746EADE7A0830E94B0
:109FC800746EA081A13021F40E94746EA6E0A08373
:109FD8000E94746EA081A23021F40E94746EABE5D9
:109FE800A0830E94746EA081A33021F40E94746E35
:109FF800AFE4A0830E94746EA081A43021F40E9473
:10A00800746EA6E6A0830E94746EA081A53021F428
:10A018000E94746EADE6A0830E94746EA081A73082
:10A0280021F40E94746EA7E0A0830E94746EA08140
:10A03800A83021F40E94746EAFE7A0830E94746E6A
:10A04800A081A93021F40E94746EAFE6A0830E941B
:10A05800746EA081AA3021F40E94746EA0E0A083DF
:10A068000E94746EA081AB3021F40E94746EA1E04E
:10A07800A0830E94746EA081AC3021F40E94746E9B
:10A08800A8E0A0830E94746EA081AD3021F40E94E4
:10A09800746EA0E4A0830E94746EA081AE3021F497
:10A0A8000E94746EA9E0A0830E94D76271CFE091EC
:10A0B8000205E695E6950E94B971E0912D070E9488
:10A0C800BE71E0912D070E94C871E0912D070E9492
:10A0D800D471E0912D07E1700E94DC71E695E17082
:10A0E800EE0F0E94DC710E94E1710E94DC710E94F7
:10A0F800E771EA2BE0933A07E09102050E94F470B9
:10A10800E295E07FAE2FE0912E070E94BE71E091AC
:10A118002E070E94C871E0912E070E94D471E09129
:10A128002F07E1700E94EB71E695E170EE0F0E9437
:10A13800EB710E94E1710E94EB710E94E771EA2BBA
:10A14800E0933B07E0910205E6950E94B971E09122
:10A158002F070E94BE71E0912F070E94C871E091FD
:10A168002F070E94D471E0912E07E1700E94F071D0
:10A17800E695E170EE0F0E94F0710E94E1710E9475
:10A18800F0710E94E771EA2BE0933C07E0913007F9
:10A198000E94B971E09131070E94BE71E0913107C8
:10A1A8000E94C871E09131070E94D471E0915B0769
:10A1B800E1700E94F571E695E170EE0F0E94F5716D
:10A1C8000E94E171EA2BAE2FE09102050E94DB6A42
:10A1D800EA2BE0933D07E09135070E94B971E091C1
:10A1E80035070E94FA71E09135070E940272E091EA
:10A1F80035070E94F4700E940C720E94F4700E944D
:10A2080010720E9415720E9410720E941B720E94A6
:10A218001072E2950E94DB6AEA2BE0933E07E09118
:10A2280034070E94B971E09134070E94FA71E091F5
:10A2380034070E940272E09134070E94F4700E9471
:10A248000C72E295E1700E9423720E9415720E94BE
:10A2580023720E941B720E942372E2950E94DB6A9D
:10A26800EA2BE0933F07E0915B070E942872E09198
:10A2780034070E94BE71E09134070E94C871E091D2
:10A2880034070E94D471E0913307E1700E942C7268
:10A29800E695E170EE0F0E942C720E94E1710E9417
:10A2A8002C720E94E771EA2BE0934007E091360791
:10A2B8000E94B971E09136070E94FA71E091360761
:10A2C8000E940272E09136070E94F4700E940C729C
:10A2D8000E943172E1700E942C720E9415720E94D5
:10A2E8002C720E941B720E942C72E2950E94DB6AFB
:10A2F800EA2BE0934107E09132070E94B971E0919F
:10A3080032070E94FA71E09132070E940272E091CE
:10A3180032070E94F4700E940C72EE1FE0E0EE1FFC
:10A32800E1700E9436720E9415720E9436720E9475
:10A338001B720E943672E2950E94DB6AEA2BE09358
:10A348004207E0915C07E2950E94B971E0913207FB
:10A358000E94BE71E09132070E94C871E0913207F5
:10A368000E94D471E0913107E1700E943B72E6953A
:10A37800E170EE0F0E943B720E94E1710E943B72F5
:10A388000E94E771EA2BE0934307E09137070E94A8
:10A39800B971E09137070E94FA71E09137070E947E
:10A3A8000272E09137070E94F4700E944072E0E068
:10A3B80030FCE1E00E944672E295E170EE0F0E94E7
:10A3C80046720E941B720E944672E295EF70E695F3
:10A3D8000E94DB6AEA2BE0934407E09129070E9478
:10A3E800F470E295E07FAE2FE0912907E695E695B7
:10A3F8000E944B720E9446720E9450720E944672DE
:10A40800E1700E944072E0915C070E94F4700E9423
:10A4180057720E945C720E945772E170EE0FEE0F45
:10A428000E945772E6950E94DB6AEA2BE093450783
:10A43800E0915C070E942872E0912A07E2950E9449
:10A448004B720E9461720E94C871E0912A070E94B3
:10A458006672E0912A070E94F4700E9461720E945D
:10A468005C720E9461720E946B720E9461720E940B
:10A47800DB6AEA2BE0934607E0915C070E943172A1
:10A488000E94B971E0915D070E944B720E94707240
:10A498000E9450720E947072E695E695E1700E94E3
:10A4A8004072E0910205E295E1700E945772EE1F3A
:10A4B800E0E0EE1FE170EE0F0E9470720E94F470EF
:10A4C800EE0FEE0F0E947072E2950E94DB6AEA2B93
:10A4D800E0934707E0915D070E942872E0912B07FF
:10A4E800E2950E944B720E9475720E94C871E091B9
:10A4F8002B070E946672E0912C070E94F4700E945C
:10A508007A720E945C720E947A720E946B720E9438
:10A518007A720E94DB6AEA2BE0934807E0915D07B4
:10A528000E9431720E94B971E0912C07E2950E9455
:10A538004B720E947A720E94C871E0912C070E94A7
:10A548006672E0912B070E94F4700E9475720E9457
:10A558005C720E9475720E946B720E9475720E94F2
:10A56800DB6AEA2BE0934907A091FA06A230A1F42E
:10A57800E1E0E0932707A0912707A13150F4E0918B
:10A588002707F0E0E75CF84FA0E0A0830E94D762BD
:10A59800F2CFE4E0E093450726FE11C0E1E0E09346
:10A5A8002707A0912707A13150F4E0912707F0E091
:10A5B800E75CF84FAFEFA0830E94D762F2CF0E940A
:10A5C8007F72A0912707AD3010F50E948772A09185
:10A5D800BE05A13061F40E948C72A0E5B8E00E942B
:10A5E800A076E17011F4429801C0429A0BC00E9413
:10A5F8008C72A2E5B8E00E94A076E17011F442984E
:10A6080001C0429A0E9491720E94D762DACF0E94DA
:10A618009972A0912707AD3090F40E9487720E942A
:10A628008C72A0E3B8E00E94A076E17011F4429821
:10A6380001C0429A0E9491720E94D762EACF0E949A
:10A648009972A0912707AD3090F40E9487720E94FA
:10A658008C72A2E0B8E00E94A076E17011F44298F2
:10A6680001C0429A0E9491720E94D762EACF0E946A
:10A678009972A0912707AD3090F40E9487720E94CA
:10A688008C72A6E0B8E00E94A076E17011F44298BE
:10A6980001C0429A0E9491720E94D762EACF0E943A
:10A6A8009972A0912707AD3010F50E948772A0918A
:10A6B8002B05A23060F00E948C72A0E8B8E00E94DE
:10A6C800A076E17011F4429801C0429A0BC00E9432
:10A6D8008C72A0ECB8E00E94A076E17011F4429868
:10A6E80001C0429A0E9491720E94D762DACF0E94FA
:10A6F8009972A0912707AD3038F50E948772A09112
:10A708002B050E945B63A0912A050E94746361F087
:10A718000E948C72A2E1B8E00E94A076E17011F468
:10A72800429801C0429A0BC00E948C72A0E1B8E026
:10A738000E94A076E17011F4429801C0429A0E94EA
:10A7480091720E94D762D5CFE0912A05E03019F4C2
:10A75800E1E0E0932A05E0912B05E03019F4E0E010
:10A76800E0932A050E949972A0912707AA30A0F4C5
:10A778000E948772A0912707E9E0EA1BA0E4B1E0F4
:10A788000E94A076E17011F4429801C0429A0E949A
:10A7980091720E94D762E8CFE1E0E0933807A09178
:10A7A8003807A13130F5E1E0E0932707A0912707AA
:10A7B800A930C8F40E948772E0913807F0E0E75C9E
:10A7C800F84F0080A0912707E8E0EA1BA02D0E941F
:10A7D8008F76E17011F4429801C0429A0E949172FA
:10A7E8000E94D762E3CFE0913807EF5FE093380724
:10A7F800D6CF429A84E08A95F1F7449A84E08A9504
:10A80800F1F7A72D0E94065EA62D0E94DF63A82DF2
:10A818000E94DF63AB2D0E94DF630E94F5620E94F5
:10A8280066760E2AAFA5B8A9EBEFFFEF0E94207756
:10A838000E2A0E9401640E94BE610E2A0E94CD6504
:10A84800E02929F0E0E0E0939907E0939A07A92D21
:10A858000E94A85FA0E0F099A1E00E94746341F013
:10A868000E94B061F09AE89426F8E0E0E0932B05A6
:10A87800A0910305AE3128F4E0910305EF5FE09362
:10A888000305A0910305AE3169F5E0E0EFA7E8AB59
:10A89800E0932105E0938E08E0938F08AC85A430FF
:10A8A80029F00E94FA60E093220516C00E94086110
:10A8B800E0932205EDE0F8E00E94A272E093230500
:10A8C800E1E1F8E00E94A272E0932405E5E1F8E0F6
:10A8D8000E94A272E0932505E0E0E0937209E4E1AA
:10A8E800E0930305EC85E03009F058C0EDE4E0930F
:10A8F800C400A0916109ECE30E94F1760E2EA091AC
:10A908006209E7E00E94F1760E22A0917209EBE05D
:10A918000E94F176E021D1F10E94AA72E1E0EE876F
:10A92800AE85A93040F40E94B0720E94B672EE85DE
:10A93800EF5FEE87F5CFE0916A09E0932207A091D7
:10A948002207E8E00E948776E0932207E0916B09EE
:10A95800A0912207EA0FE0932207A0918907B091FE
:10A968008A07F0E0EA17FB0779F4E0916309E093BE
:10A978002005E0916409E0932105A0916509EAE0CA
:10A98800EA9FF0010E94C2720E94D672A0917209D9
:10A99800AC3020F00E94DC720E94E972AC85A130D4
:10A9A80009F065C0EDE4E093C400A0916109E8E214
:10A9B8000E94F1760E2EA0917209E8E00E94F176CD
:10A9C800E02109F44CC00E94AA72E0E0EE87AE854F
:10A9D800A73060F40E94B072A0918907B0918A07ED
:10A9E8000E94F572EE85EF5FEE87F1CF0E94FD724F
:10A9F800E0916809F0E0EA17FB0789F5E1E0E093E8
:10AA080020050E940164DD9710F0E1E001C0E0E05C
:10AA1800E09321050E9404730E94F470A09121051F
:10AA2800EA0FE09321050E940473E170A0912105CB
:10AA3800EA0FE0932105E0916409F0E0EFA7F8AB95
:10AA4800FFA5E0E0EFA7F8ABE0916509F0E0AFA55E
:10AA5800B8A9EA0FFB1F0E94C2720E94D672A09189
:10AA68007209A93020F00E94DC720E94E972AC855C
:10AA7800A43009F003C2E0912407E03031F4E98101
:10AA8800F0E0E851FA4FA0E0A083A0916109EBE65D
:10AA98000E94F1760E2EA0916209EFE00E94F176F5
:10AAA8000E22A0917209E0E10E94F176E02109F4FA
:10AAB8008DC10E94AA72E1E0EE87AE85AF3040F406
:10AAC8000E94B0720E94B672EE85EF5FEE87F5CFF6
:10AAD8000E94FD72E0917009F0E0EA17FB0709F0A7
:10AAE80075C1E0916509E370E093CF050E940C738E
:10AAF800503041F4A091CF05B0E0A553BA4FE09192
:10AB08006309EC935D35D9F50E94B97041F0A091C5
:10AB1800CF05B0E0A75BBA4FE0916309EC930E94C0
:10AB2800DB7041F0A091CF05B0E0A052BA4FE091A0
:10AB38006309EC930E94F97041F00E9413730E941C
:10AB48001B730E9413730E9427730E9467710E94EF
:10AB58006B7141F0A091CF05B0E0A75EB84FE091CE
:10AB68006309EC930E9477710E947B7141F00E9407
:10AB780037730E941B730E9437730E9427730E94C9
:10AB88003F730E9447730E943F730E949C6EE0309F
:10AB9800A2E0FA0724F00E943F730E9453730E94B8
:10ABA8003F730E945C73E09166090E9464730E947F
:10ABB8006B730E9447730E946B730E949C6EE03017
:10ABC800A2E0FA0724F00E946B730E9453730E945C
:10ABD8006B730E945C73E09167090E946473A09193
:10ABE800CF05B0E0A451BA4FE0916809EC93E09129
:10ABF800CF050E945465E0916909FF2766277727EA
:10AC08000E942E78A091CF05B0E0AE5DBA4FE091DA
:10AC18006A090E947373E695E695E6950E94787333
:10AC2800A053BA4F0E947D73E6950E947873AC5288
:10AC3800BA4F0E947D73E6950E947873A852BA4F66
:10AC48000E947D73E695EC93E091CF05F0E0E85221
:10AC5800FA4F7E2F8F2F6081E0916B09E170AE2F44
:10AC6800E0E0F799E1E0EA02F001E62BA72FB82F20
:10AC78000E947373E6950E947873A452BA4FE091CC
:10AC88006B09E1700E9481730E948A73A8E9B8E099
:10AC98000E9496730E9481730E945C73E0916F0911
:10ACA8000E9464730E94A7730E948A73A0E9B8E0A7
:10ACB8000E949673EC930E94A7730E945C73E091C4
:10ACC8006E090E9464730E94AF730E948A73A4E5A0
:10ACD800B8E00E949673EC930E94AF730E945C7375
:10ACE800E0916D090E946473E091CF05F0E0EB5E9E
:10ACF800F84F0E94B773ACE6B9E0EC91E695EC9397
:10AD0800E091CF05F0E0EF5EF84F0E94B7730E9424
:10AD1800D672EDADFEADABADBCADEA0FFB1FDE01EB
:10AD2800A15CBF4F0D90BC91A02DEA0FFB1FDE0167
:10AD3800AF5BBF4F0D90BC91A02DEA0FFB1FEFA793
:10AD4800F8ABE0E0E0932105E091D005EE0FA0918B
:10AD5800D405AE0FE091D8050E94C073A091D50527
:10AD6800E091D105EE0FAE0FE091D9050E94C073B6
:10AD7800A091D605E091D205EE0FAE0FE091DA056D
:10AD88000E94C073A091D705E091D305EE0FAE0FD6
:10AD9800E091DB050E94C073E091CF05F0E0EC5133
:10ADA800FA4FA1E0A083E091CF05F0E0E851FA4F17
:10ADB800A083E091E905A091E805AE0FE091EA05CE
:10ADC800AE0FE091EB05EA0FE093C705A091720979
:10ADD800A03118F1E0E0E0936109E0936209E093A3
:10ADE8006309E0936409E0936509E0936609E093D9
:10ADF8006709E0936809E0936909E0936A09E093B9
:10AE08006B09E0936C09E0936D09E0936E09E09398
:10AE18006F09E0937009E0937209E981F0E00E94FC
:10AE2800D37061F5E981F0E0E553FA4F0E94C973E8
:10AE3800E053FA4F0E94C973EC52FA4F0E94C9734B
:10AE4800E852FA4F0E94C973DE01DB960E94CE7366
:10AE5800A4E5B8E0F0E00E94CE73A0E9B8E0F0E025
:10AE6800EE0FFF1FAE0FBF1FE0E0F0E0ED93FC9385
:10AE78000E94E064E0E0F0E0ED93FC93EC85E030C4
:10AE880009F0C5C0ED85E03019F0E0E00E94D87304
:10AE98000E94DE734420D1F5A0912507A43048F420
:10AEA800E0912507F0E034960E949163EA0FFB1FBA
:10AEB80003C00E9442643F96A091E307B091E40763
:10AEC800EA0FFB1FBF01A989B0E0E7E00E9497766F
:10AED800E60FF71FE0938907F0938A07AEE30E9415
:10AEE8008C5BA4E00E948C5BA0912507A43008F439
:10AEF80001C0ABE00E948C5BE989E795E0E0E7954B
:10AF08000E94E573A091E3070E94EC73E1E0E41569
:10AF180009F07DC04424ACA5B0E00E94D864EBA73A
:10AF2800EEA5E095E170EDA7EBA5F0E0BC96DF019A
:10AF3800EE27A40FBE1FEDA5F0E0EA0FFB1F0F01DF
:10AF48000E94C067F0E0D001AE0FBF1FEAA5F0E095
:10AF5800AE0FBF1FE0916007F0E0AE0FBF1FE0919A
:10AF68006107F0E0AE0FBF1FE0916207F0E0AE0F9F
:10AF7800BF1FE9A5F0E0AE0FBF1FE0913B05F0E071
:10AF8800AE0FBF1F0E944366E081F0E0AE0FBF1F07
:10AF98000E94916EF0E0EA0FFB1FE0938907F0939F
:10AFA8008A07AEE30E948C5BACE20E948C5BA42F04
:10AFB8000E948C5BADA50E948C5B0E9408690E9470
:10AFC8008C5BABA50E948C5BAAA50E948C5BA091B0
:10AFD80060070E948C5BA09161070E948C5BA09126
:10AFE80062070E948C5BA9A50E948C5BA0913B051F
:10AFF8000E948C5B0E944366A0810E948C5BE0915A
:10B008002507F0E0EF5BFA4FA0810E94EC73AC8556
:10B01800A13009F07BC0AD85A13019F0E1E00E94B4
:10B02800D8730E94DE73E989EE0FEE0FE98BEF5FAC
:10B03800E98B0E940164A93CE0E0BE0710F00E9481
:10B0480054640E940164E5E00E9488770E94E463EA
:10B058000E945D64A3E3B3E383E890E40E94A775CC
:10B06800A0E0B0E084E393E40E9457750E947964FD
:10B07800E989AFE2EA27AAA5AE27E1E0AE27E6E331
:10B08800AE27E091E407F070EA270E940164EA27FE
:10B09800FB27BF010E94F773E627F7270E949163F9
:10B0A800AE27BF27E1E0F0E0AE27BF27E6E3F0E0F8
:10B0B800EA27FB270F010E94C067D001F0E0AE2706
:10B0C800BF27E09125070E94F572AFE221D3A98935
:10B0D8001FD3A0E01DD3AAA51BD30E94FE73E09145
:10B0E800E407AE2F15D3A091E30712D30E94F7739C
:10B0F8000E94E5730E94FE73A0E00AD30E940869CB
:10B1080007D3A091250704D30E940474AC85A2300C
:10B1180019F4E0E8E093C100AC85A43009F0F5C269
:10B12800E981EF5FE983A981A43010F0E0E0E983C9
:10B13800A0912307A13030F0E0912307E150E0937C
:10B14800230746C0A9810E94065EA091E4050E94DB
:10B15800746311F0E1E0E983A9810E94A85FA091DE
:10B16800E5050E94746311F0E2E0E9830E94087427
:10B1780011F0E3E0E983A9810E945168A091E705F5
:10B188000E94746311F0E0E0E983A9810E94065EE1
:10B19800A091E4050E94746311F0E1E0E983A981BC
:10B1A8000E94A85FA091E5050E94746311F0E2E097
:10B1B800E9830E94087411F0E3E0E983A9810E9401
:10B1C8005168A091E7050E94746311F0E0E0E983FB
:10B1D800AD85A43039F0E4E0ED87ECE0E093C400FD
:10B1E8000E94B061EFE0EA83442009F06CC1E0E01E
:10B1F800E0932407503011F4E0930A075D3511F508
:10B208000E94B97019F0E8E0E0930A070E94DB7029
:10B2180019F0E9E0E0930A070E94F97019F0E6E0F6
:10B22800E0930A070E9467710E946B7119F0E5E0CC
:10B23800E0930A070E9477710E947B7119F0EAE097
:10B24800E0930A07E091F505EF5FE093F505A0911B
:10B25800F505A23018F0E0E0E093F505E091F2057D
:10B26800E093F605E091F305E093F705EAE6E0934D
:10B278004A07EFE0E0934B07EA81E0934C07ACE420
:10B28800B7E0EC91E295E07FEC93ECE4F7E00F0196
:10B29800E081A981EA0FD001EC93E091FA06E03051
:10B2A80059F4E0914605E0934D07E0914705E09396
:10B2B8004E07E091480507C00E945464E0E0E0931F
:10B2C8004D07E0934E07E0934F070E941174A09139
:10B2D800FE06EA0FD001EC930E941174A091FF06BC
:10B2E8000E941C74EE0FEE0FEC93A0912507A4307A
:10B2F80040F40E942374A0912507EA0FD001EC9333
:10B3080005C0E0914D07EF5FE0934D07A091260738
:10B31800E3E60E947A6EEDE50E94F1760E22A09196
:10B328005E070E94BB6611F00E9427640E940164B8
:10B338000E94587878F5E0E0E0935007A091340532
:10B348000E94065E0E94287419F0E091E30701C08C
:10B35800E0E0E0935107A09134050E94A85F0E94A5
:10B36800287419F0E091E30701C0E0E0E093520788
:10B37800A09134050E945168A09134050E94E56AA5
:10B3880019F0E091E30701C0E0E0E0935407E0938F
:10B3980053071DC0E0EFE0935007E0913305E0301C
:10B3A80061F4E0914208E0935107E0935207E0E02E
:10B3B800E0935407E09353070AC0E0914208E093F2
:10B3C8005407E0935307E0935207E0935107A09185
:10B3D8002507A43018F4E091500703C0E091500706
:10B3E800E15FE0935007E091F405E0935507A5E588
:10B3F800B7E0EC91E295E07FEC93E5E5F7E00F012B
:10B40800E081A091F505EA0FD001EC93E091550792
:10B41800F0E0EA50FA4FE081E0935607E0910A071E
:10B42800E0935707A7E5B7E0EC91EE0FEE0FEE0FAC
:10B43800EC93E7E5F7E00F01A081E0E0F6FCE1E03E
:10B44800EA0FD001EC93A7E5B7E0EC91EE0FEC938F
:10B45800AB890E9430740E944366A081E3E00E9499
:10B46800F176E02951F0E7E5F7E00F01A081E0E08F
:10B4780021FCE1E0EA0FD001EC93E0914108E09370
:10B4880058070E94AA72E1E0E0932707A0912707D6
:10B49800AF3040F40E943574E0810E94B6720E9479
:10B4A800D762F4CF0E943B74A0912707AF3038F4DD
:10B4B8000E943574A0812CD10E94D762F5CF0E94DA
:10B4C80004740E944674E1E0E41509F01EC1E0939B
:10B4D8002407E8E8E093C100ECE6E0934A07EFE0D0
:10B4E800E0934B0740934C07E0E0E0934D07ADE451
:10B4F800B7E0EC91EE0FEC93E0914D07E0934D0728
:10B50800ADE4B7E00E944E74EDE4F7E00F01A081CE
:10B518000E944366E0810E941C740E945374A091AB
:10B5280053050E941C740E945374A091FC060E944B
:10B538001C740E945374A091FB060E941C74EE0FA9
:10B54800EC93EDE4F7E00F01A0810E94916EEA0F01
:10B55800D001EC93E1E00E945674AEA50E9462749B
:10B56800E0914E07EF5F0E945674A9A50E9462748D
:10B57800A0913A05A13079F4E0E0E0933A05E09132
:10B588004E07EF5F0E946B74EEE4F7E00F01E08175
:10B59800A09139050AC0E0914E070E946B74EEE451
:10B5A800F7E00F01E081A0913605EA0FD001EC9396
:10B5B800E0E0E0935007E0934F070E9470740E9408
:10B5C8007774E12959F00E944E660E947B740E94AC
:10B5D8008374AFE4B7E00E94E474EC93A09136055D
:10B5E8000E94A85FA09133050E9474630E94917421
:10B5F800E12959F00E944E660E947B740E9499745A
:10B60800AFE4B7E00E94E474EC930E9470740E9467
:10B618007774E12959F00E944E660E947B740E945B
:10B628008374A0E5B7E00E94E474EC93A09136051A
:10B638000E94A85FA09133050E9474630E949174D0
:10B64800E12959F00E944E660E947B740E94997409
:10B65800A0E5B7E00E94E474EC93E091AD07E093B5
:10B668005107AAE0EA9FF001A091ED07EA1BE093D9
:10B678005207E091AD07AAE0EA9FF001A091F10717
:10B688000E945078EA1BE0935307E0911905E09374
:10B6980054070E94856EE0935507E0913505E093C5
:10B6A8005607E0E0E0935707E0935807E091360526
:10B6B800EF5FE0933605A0913605A43020F04424CE
:10B6C800E0E0E09336050E94AA72E1E0E0932707E4
:10B6D800A0912707AF3040F40E943574E0810E94A2
:10B6E800B6720E94D762F4CF0E943B74A0912707DC
:10B6F800AF3038F40E943574A0810AD00E94D76216
:10B70800F5CF0E9404740E9446740C94E409FFCF9C
:10B71800AA93E091C000E072E1F3E881E093C600EB
:10B7280021960895BA93AA931A93689434F8E7E097
:10B73800E0937709E0E0E0938009E0938109E093E2
:10B748008209E0938309419A409AE093BC00E09112
:10B75800B900EC7FE093B900E981FA81A0E7B7E18D
:10B768000E9498771E2F183008F018501093B800D0
:10B77800E091BC00E078E564E093BC001881239672
:10B788000895AA93249734FE66C0EA85EE0FE093E5
:10B798007809E885F985E0937909F0937A09E0E07A
:10B7A800E0937509EF81E0937B09ED81FE81E093D9
:10B7B8007C09F0937D09E0E0E0937609EC81E09361
:10B7C8007E09E6E0E09377097894EF81E03081F034
:10B7D800E885F985309709F43EC0EC81E03021F026
:10B7E800AD81BE81109709F001C035C068940DC0C5
:10B7F800EC81E03051F1ED81FE81309761F1E0910B
:10B808007809E160E0937809E89433F8E89434F82B
:10B81800E091BC00EF70E06AE093BC00E0E2F1EA7E
:10B8280067E070E00E94387834FC0FC00E943378DB
:10B838003197604070400E94387831F4E5E0E09339
:10B848007709689434F807C0EFCFA0917709E0E052
:10B858000E94F17601C0E0E02B9608950A921A92B0
:10B86800FA926A937A938A939A93AA93BA93EA93E9
:10B87800FA93EFB7EA930E946778109176090091DE
:10B88800750930917B0920917709E12FA0917C09F6
:10B89800B0917D09F0E0EA0FFB1FAF01E091B9001C
:10B8A800E87FE83011F420E002C0E03119F4E091BB
:10B8B800780910C0E83111F0E83249F5031798F417
:10B8C800E02F0F5FA0917909B0917A09F0E0AE0FEF
:10B8D800BF1FEC91E093BB00E091BC00EF70E06803
:10B8E800E093BC0013C0E0917E091E1770F4E0914C
:10B8F8007809E160E0937809E89433F8E091BC00B6
:10B90800EF70E06AE093BC0013C138C011C1E035A4
:10B9180031F4E091BB00DA01EC931F5F02C0E03420
:10B9280089F4E0917E09E1501E1728F0E091BC00EF
:10B93800EF70E06804C0E091BC00EF70E06CE09349
:10B94800BC00F6C0E83531F4E091BB00DA01EC93B5
:10B958001F5F02C0E03209F402C0E03309F402C0FC
:10B96800E83469F4203051F433FE03C0031728F09B
:10B9780005C0E0917E091E1708F424E0D1C0E83321
:10B9880031F422E0E091BC00EF70E068CDC0E83609
:10B9980011F0E83711F422E005C0E03611F0E03785
:10B9A800A9F420E010E0E89433F8E0917F09E03052
:10B9B80031F421E0E091BC00EF70E06804C0E09150
:10B9C800BC00EF70E06CE093BC00B2C0E03811F04E
:10B9D800E03941F533FE02C021E0A2C0E091BB008E
:10B9E800DA01EC931F5FE0917F091E17C0F4E09124
:10B9F8008009F0918109309711F426E091C0A0E008
:10BA0800E0918009F09181090995E03039F0E091E1
:10BA1800BC00EF70E06CE093BC008AC002C0689480
:10BA280033F802C0E83809F402C0E83939F4E09183
:10BA3800BC00EF70E068E093BC007AC0E03AB9F46B
:10BA4800E091BC00EF70E06CE093BC00689434F8BF
:10BA5800E0918009F0918109309739F0A1E0E091F7
:10BA68008009F0918109099501C026E061C0E03B99
:10BA780011F422E002C0E83AB9F4E0918209F091A9
:10BA88008309309759F0A0E0E0918209F091830989
:10BA980009953E2FE03011F020E002C026E040C0BA
:10BAA80000E0E89433F802C0E83B01F533FE02C039
:10BAB80021E036C0E02F0F5FA0917909B0917A0993
:10BAC800F0E0AE0FBF1FEC91E093BB00031728F422
:10BAD800E091BC00EF70E06C06C0689433F8E09128
:10BAE800BC00EF70E068E093BC0022C0E03C11F0BD
:10BAF800E83C99F4E091BC00EF70E06CE093BC0086
:10BB0800E0918209F0918309309731F0A1E0E0914A
:10BB18008209F0918309099509C0E03049F423E0CE
:10BB2800E091BC00EF70E06DE093BC00689434F8DD
:10BB380010937609009375092093770930937B0950
:10BB48000E946E782696E991EFBFF991E991B99133
:10BB5800A9919991899179916991F9901990099090
:10BB68001895A4E4B8E0F0E0EE0FFF1F0895A09147
:10BB7800C707B091C8070895E0E0F0E00E94327767
:10BB88000E2E0895E0E0E7BDE8BD0895B0E00E94FC
:10BB9800A774E0E00895E0935805E8E6EA93E8E53D
:10BBA800F5E0FA93EA93E1E0EA93EAE5F5E0FA933F
:10BBB800EA930895E0E0E0935A05E0935B05089561
:10BBC800E8E6EA93EAE5F5E0FA93EA930895E4E013
:10BBD800EA93E0E0F0E0FA93EA93A0E00C94C55B06
:10BBE800E0E0E0935805E0935905E0E5EA93E8E5DD
:10BBF800F5E0FA93EA93E2E0EA93EAE5F5E0FA93EE
:10BC0800EA930895E0E00E94F1760E2E0895E0E0B0
:10BC18000E94F1760E220895E0936205E0E0E09339
:10BC280063050895E0936505E0E0E09366050895EF
:10BC3800E0937005E0E0E09371050895E0937205E4
:10BC4800E0E0E0937305E09374050895E0937905C7
:10BC5800E0E0E0937A050895E0937D05E0E0E09365
:10BC68007E050895E0937F05E0E0E0938005E0938A
:10BC780081050895E0938505E0E0E0938605E0936B
:10BC880087050895E0938A05E0E0E0938B05E0934B
:10BC98008C05E0938D050895E0939005E0E0E0932E
:10BCA8009105E0939205E0939305E0939405E09362
:10BCB80095050895E0939605E0E0E0939705E093F5
:10BCC80098050895E0939A05E0E5EA93EAE5F5E03A
:10BCD800FA93EA930895E1E4EA93E0E0F0E0FA9356
:10BCE800EA93A0E00E94C55BAAE050CFE0935C0510
:10BCF800E0E0E0935D05E0935E05E0935F0508955D
:10BD0800E0936005E0E0E09361050895E093640541
:10BD1800E0E088CFE0E0E0936705E09368050895E8
:10BD2800E0936B05E0E0E0936C05E0936D05E0932C
:10BD38006E050895E0936F05E0E07ACFE0E0E093C8
:10BD48008205E0938305E093840594CFE09388050A
:10BD5800E0E0E093890596CFE0E5EA93EAE5F5E0CF
:10BD6800FA93EA930895EA93E0E0F0E0FA93EA930D
:10BD7800A0E00E94C55BAAE00895B0E00E94A77405
:10BD8800E1E00895E0935E05E7CFE0935B05E0E02E
:10BD9800ADCFE0E0E0936905E0936A050895EBE034
:10BDA800E0936609E8EBE09367090895E093B60825
:10BDB800F093B7080895E0935E08F0935F0808953C
:10BDC8000E94C55BE0915A050895E0938707F093B8
:10BDD80088070895A0918707B09188070895E09390
:10BDE8007707F09378070895E0937907F0937A0737
:10BDF8000895E093E507F093E6070895E093ED07CB
:10BE0800F093EE070895A091ED07B091EE0708951D
:10BE1800E093E907F093EA070895A091E907B09144
:10BE2800EA070895E093F507F093F6070895A091BF
:10BE3800F507B091F6070895E0938B07F0938C0708
:10BE48000895A0918B07B0918C070895E093050899
:10BE5800F093060860930708709308080895A09166
:10BE68000508B09106088091070890910808089580
:10BE78000E94E7760E946C760895E0939707F09306
:10BE880098070895A0919707B09198070895E093AF
:10BE98009F07F093A0070895A0919F07B091A0076E
:10BEA8000895E093AD07F093AE070895A091AD070C
:10BEB800B091AE070895E093F107F093F207089563
:10BEC800E0935905E0E5EA93E8E5F5E0FA93EA93AB
:10BED800E2E0EA93EAE5F5E0FA93EA930895A0919F
:10BEE800F107B091F2070895E0933108F093320812
:10BEF80060933308709334080895A0913108B09185
:10BF0800320880913308909134080895E8E00E943F
:10BF1800A976EACFF0E0F1DFABCFE6DFEEDFF6CFD0
:10BF2800E093A107F093A2070895A091A107B0910B
:10BF3800A2070895E0937F07F09380070895A091E2
:10BF48007F07B09180070895E1E00E94F1760E2EF8
:10BF58000895E0935309F09354090895A091530963
:10BF6800B09154090895E0935509F093560908953E
:10BF7800A0915509B09156090895E093A808F09347
:10BF8800A9080895A091A808B091A9080895E09378
:10BF98005709F09358090895A0915709B091580985
:10BFA8000895E0935909F0935A090895A091590901
:10BFB800B0915A090895E0935B09F0935C090895DC
:10BFC800A0915B09B0915C090895E0935D09F09335
:10BFD8005E090895A0915D09B0915E090895E09306
:10BFE800D507F093D6070895E093F307F093F40785
:10BFF8000895A091F307B091F4070895E0931D0800
:10C00800F0931E0860931F08709320080895A0916C
:10C018001D08B0911E0880911F089091200808956E
:10C02800E093CF07F093D0070895E0932508F093A5
:10C03800260860932708709328080895A09125087A
:10C04800B091260880912708909128080895E8E083
:10C058000E94A976EACFF0E0F1DF0ACFE6DFEEDF53
:10C06800F6CFE093C808F093C9086093CA087093A4
:10C07800CB080895A091C808B091C9088091CA0852
:10C088009091CB080895E093CC08F093CD08609385
:10C09800CE087093CF080895A091CC08B091CD0830
:10C0A8008091CE089091CF080895E093A307F0936C
:10C0B800A4070895A091A307B091A4070895E09359
:10C0C800C008F093C1086093C2087093C30808952C
:10C0D800A091C008B091C1088091C2089091C3088E
:10C0E8000895E093C408F093C5086093C608709358
:10C0F800C7080895A091C408B091C5088091C608E2
:10C108009091C7080895E0932108F093220860935E
:10C118002308709324080895A0912108B09122085B
:10C1280080912308909124080895E0932908F093BA
:10C138002A0860932B0870932C080895A091290869
:10C14800B0912A0880912B0890912C080895F6DF69
:10C158008FCEA6E9B0E0A083B1830895E0910508E9
:10C16800F091060860910708709108080895A4E600
:10C17800B0E080E090E00E9468770895A0DFE0E0FA
:10C18800E0935A05E3EBE0935B05A2DFE0E10E9450
:10C19800B576E0935C059CDFE8E00E94B576E09315
:10C1A8005D05E091C008EECDB0E00E94A774E09173
:10C1B800AD07F091AE0753DE662777270E946877B0
:10C1C80090DFE0E0E0935A05E6EBE0935B0592DF51
:10C1D800E0E10E94B576E0935C058CDFE8E00E9420
:10C1E800B576E0935D05E091C408CCCDEBE0F0E0D6
:10C1F80060E070E0E0930908F0930A0860930B0888
:10C2080070930C08E8EB0895E0E0E0930908E093E8
:10C218000A08E0930B08E0930C080895A091F6062D
:10C22800BB27E091F706F0E0AE0FBF1F0895E1E0ED
:10C238006E2E9E2E8E2EBE2E0895A091D408B091FB
:10C24800D5088091D6089091D7080895A091E8085C
:10C25800B091E9088091EA089091EB080895E0937D
:10C26800E808F093E9086093EA087093EB080895EA
:10C27800A0910809B091090980910A0990910B09C8
:10C288000895E0E0F0E060E271E40895A0913409D7
:10C29800B091350980913609909137090895E09356
:10C2A8003409F09335096093360970933709089576
:10C2B800EEEFFFEF6FE77FE30E943A760895A0E084
:10C2C800B0E080E89FE30E9450750895E09131083E
:10C2D800F091320860913308709134080895EF5F47
:10C2E800FF4F6F4F7F4F0895E091CF07F091D00730
:10C2F8000895E0935A05EFE4E0935B05FEDDE8E17D
:10C308000E94C176E0935C05E1DF0E94DC76E09351
:10C318005D05F3DDE8E00E94C176E0935E05E091FB
:10C328003108E0935F0518CDE0935A05ECE5E093FA
:10C338005B05E0918007E0935C05E0917F07E0935F
:10C348005D050ACDE0935A05EEE5E0935B05D092D2
:10C358005C05C0925D0500CDAAE0B0E00C94A7741E
:10C36800A0918D07B0918E070895A0919B07B09179
:10C378009C070895E0E0F0E00E9432770895E0918C
:10C38800F008F091F1086091F2087091F3080895AF
:10C39800E0911409F0911509609116097091170937
:10C3A80008950E94E474ED93FC930895E0E0F0E0B2
:10C3B80061EE75E40E94F5750895E0918D07F0919E
:10C3C8008E070895EDECFCEC6CEC7DE30E94A775FC
:10C3D8000895A091F408B091F5088091F60890911D
:10C3E800F70808950E94E674ED93FC930895E0938E
:10C3F800F808F093F9086093FA087093FB08089519
:10C40800E091FC08F091FD086091FE087091FF082A
:10C418000895E093FC08F093FD086093FE0870937C
:10C42800FF080895A0916208B09163080895A0914B
:10C438000409B091050980910609909107090895AA
:10C44800E0E0F0E060E972E40E94F5750895A091DB
:10C458000C09B0910D0980910E0990910F0908956A
:10C468000E945775E0930C09F0930D0960930E092B
:10C4780070930F090895E091DC08F091DD08609150
:10C48800DE087091DF08D3DF0E94A775DF01CB01BA
:10C49800E0E0F0EA6CE877E40E94F5750895A09171
:10C4A8001009B0911109809112099091130908950A
:10C4B8000E945775E0931009F093110960931209CF
:10C4C8007093130908950E945775E0931809F09323
:10C4D800190960931A0970931B0908950E945775EA
:10C4E800E0932009F09321096093220970932309AE
:10C4F8000895A0911C09B0911D0980911E09909181
:10C508001F090895E0931C09F0931D0960931E0903
:10C5180070931F090895A0912409B091250980916D
:10C528002609909127090895E0932409F093250995
:10C5380060932609709327090895E0910C09F091FA
:10C548000D0960910E0970910F090895E091C008D6
:10C55800F091C1086091C2087091C3080895E15034
:10C56800F040604070400895E0911009F091110981
:10C5780060911209709113090895E091C408F0912F
:10C58800C5086091C6087091C7080895A0E0B0E09A
:10C5980080E89FE30895AF39E6E8BE07E1E08E073B
:10C5A800E0E09E070895E0912707EF5FE0932707F3
:10C5B80008950E94A775DF01CB010895A09128096D
:10C5C800B091290980912A0990912B090895AAE030
:10C5D800B0E080E090E00895E0919F07F091A00717
:10C5E80008952BDEE0E0F0E060E070E008950E943E
:10C5F80066760E22A0914208B0914308E0E0F0E090
:10C608000895E091D408F091D5086091D60870910A
:10C61800D7080895A0913809B091390980913A094D
:10C6280090913B090895ADECBCEC8CEC9DE30E9425
:10C63800A7750895AE8DECE30E940A770895E091FE
:10C648001D08F0911E0860911F0870912008089538
:10C65800F4DD17DE0E94A7750895E0912108F09196
:10C66800220860912308709124080895E0913D08FC
:10C67800F0913E0860913F08709140080895ACE33E
:10C68800B0E080E090E00E9468770895AFA5B8A96F
:10C69800E0E0F0E00E9426770895E4E6F0E060E04C
:10C6A80070E00895662777270E9476760895E0E07F
:10C6B8000E940F770E2E08950E22A0912607E3E61A
:10C6C80008950E940A770E22A091FA06E0E00E94DF
:10C6D800F176E0210895A0919907B0919A070895FD
:10C6E800E0E00E94F176E0210895E0919707F0914B
:10C6F80098070895E091D907F091DA070895E09333
:10C70800D907F093DA07E0E0E0935A050895E0933B
:10C718005C0522CBE0935D051FCBA0914208B09148
:10C7280043080895E0E0F0E00E94267708950E2E71
:10C73800A091E307B091E4070895E1E04E2EE0E010
:10C74800E09336050895E0914A08F0914B08089562
:10C75800E0918707F09188070895A0912D08B0917E
:10C768002E0880912F089091300866277727089522
:10C77800A0E0B0E080E490E40E9457750895E0914D
:10C788002D08F0912E0860912F08709130080895B7
:10C798000E941B750E942E780895E0910705A091CC
:10C7A8000805AE170895E0E01A99E1E09E2EE0E052
:10C7B8001899E1E00895E0E00E94F1760E2A0895C4
:10C7C800E093E307F093E4070895E0934208F093B9
:10C7D80043080895E0917707F09178070895E0916C
:10C7E8007907F0917A07089598DFEA17FB0708950B
:10C7F800E091E507F091E6070895A091E307B0916D
:10C80800E4070895E091E707F091E80708950E948A
:10C818002C770E2EA52DE1E00E940F770E220895A9
:10C828000E9432770E2EA52DE1E00E940F770E228E
:10C838000895E4E00E940A77E0210895E091E30773
:10C84800F091E4070895E0E0E0934208E09343089C
:10C858000895E0E0E093E307E093E4070895E4E057
:10C868000E94F1760E2E0895E5E00E94F176E02907
:10C878000895A0917707B09178070895E09142084C
:10C88800F09143080895EA1BFB0BA8ECB0E00E9466
:10C8980060770F010895A091E507B091E607089524
:10C8A800E8ECF0E08DCFE0912507F0E0E25DFA4F8B
:10C8B8000895E4DF0E94E7760E941D750895E081DF
:10C8C800F0E00E94E7760E941D7508950E9447785F
:10C8D8000E94507508955ADE0E94577508951DDF0D
:10C8E8000E94EC760E9444780895A2E4B8E07ACDDC
:10C8F800A4E0B9E00E94E7760E941D750E942E7898
:10C908000895E0914C08F0914D0808950E94E7764B
:10C918000E941D750895E091E907F091EA070895CE
:10C92800662777270E941D750895ED51F140EEDFC7
:10C93800A1E7BDE38AEA9FE30E94A77508950E94D4
:10C948008E77DF01EEE5F1E00E94AB770895DEDF38
:10C95800BDCFE981A4E5B8E0F0E0EE0FFF1FAE0F10
:10C96800BF1F0E9424780895A981E3E0EA9FF0019F
:10C9780008953196ACE6B8E0EE0FFF1FEA0FFB1FF3
:10C988000895E981A0E9B8E0F0E0EE0FFF1FAE0FCF
:10C99800BF1F0E94247808953296ACE6B8E0EE0FE7
:10C9A800FF1FEA0FFB1F0895E2E0F0E00E94AB775B
:10C9B80008953196DF01F8CFE981A8E9B8E0F0E001
:10C9C800EE0FFF1FAE0FBF1F08950E940A770E2EAD
:10C9D800A52DE2E30E940F77E02108951A96E091D1
:10C9E8004F05F0E0EA17FB070895A091B008B09151
:10C9F800B1080E9414770E2E0895A091E405E1E095
:10CA08000E94F176E0210895A091E505E1E00E94F9
:10CA1800F176E0210895A091E605E1E00E94F17623
:10CA2800E0210895A091E705E1E00E94F176E02178
:10CA380008951A96E0915005F0E0EA17FB0708956B
:10CA48001A96E0915105F0E0EA17FB070895ADE961
:10CA5800BDEFA083B1830895E0918808F09189081B
:10CA6800EA17FB070895E0938808F093890808956A
:10CA7800E0918A08F0918B08EA17FB070895E09384
:10CA88008A08F0938B080895E0918C08F0918D083E
:10CA9800EA17FB070895E0938C08F0938D08089532
:10CAA800A9E0B8E0F0E00E94CD76AE0FBF1F089570
:10CAB800A091D808B091D9088091DA089091DB0844
:10CAC8000895E091D808F091D9086091DA0870913A
:10CAD800DB080895E093D808F093D9086093DA0842
:10CAE8007093DB0808951CDF0E942E780895A091AA
:10CAF8003009B09131098091320990913309089534
:10CB08000E94A775E093D408F093D5086093D608DF
:10CB18007093D7080895E0918B07F0918C070895DA
:10CB2800A091AC08B091AD080895ABDB0E94A77541
:10CB3800089583DBFF27662777270E941D750895D0
:10CB48000E2EA0912607E3E60895A52FEAE50E9498
:10CB5800F1760895E091AF07F091B0070895E0935A
:10CB6800AF07F093B0070895F5DFA1EBB7E0EE0F3C
:10CB7800FF1F08950E94BB5DE5E2F0E00E949877F0
:10CB880008950E94BB5DE0E0F0E00E9414770E2E4D
:10CB98000895C3DDC7CDA091AF07B091B007089540
:10CBA800E0E0F0E00E941477E0210895A0E0B0E012
:10CBB800A083B183089541DBE0E0F0E060E87FE323
:10CBC8000E9460760E220895A8DDEACFA0916A0837
:10CBD800B0916B080895E0916A08F0916B08089588
:10CBE800E091F307F091F4070895B8DAC0CAA0916C
:10CBF8002607E3E60E940A7708951FDBE0E0F0E0ED
:10CC080060E87FEB0E9466760895F7DDE0E0F0E0EB
:10CC18000E94147708950E22A091FA0661CDE09142
:10CC28002507F0E0EC59F84F0895FF276627772786
:10CC38000E941D750E942E780895A0914009B09118
:10CC4800410980914209909143090895F6DF0E94B5
:10CC5800A775E9CCE0912507F0E0E15AF84F08956F
:10CC6800DF01E4E6F0E00E94AB770895E0913C092B
:10CC7800F0913D0960913E0970913F090895E09156
:10CC88002507F0E0E45CFA4F0895E081F0E0ED5804
:10CC9800F84F0895E0912507A7EFB7E0F0E0EE0F11
:10CCA800FF1FAE0FBF1F0E9424780895A091480966
:10CCB800B091490980914A0990914B090895A09132
:10CCC8005F09B09160090895E0E0E0935F09E0939F
:10CCD80060090895882799270E9444780E943A7627
:10CCE8000895E091D507F091D6070895A091D5074A
:10CCF800B091D6070895E0911E051BCFE9E1EA9FA0
:10CD0800F001DDDF0E943277E6230E2E0895E0E081
:10CD18000E940F77E0210895E1E00E94F176E02972
:10CD28000895E0912C09F0912D0960912E097091D8
:10CD38002F090895EBDD0E942E7808950E22A09108
:10CD48002C09B0912D0980912E0990912F090895F1
:10CD5800E0E0F0E068E473E40E94607608950E2253
:10CD6800A0E021FCA1E0E1E00E94F1760895E1E075
:10CD78000E94F176E0210895E0932C09F0932D09A3
:10CD880060932E0970932F0908950E943277CFCCB3
:10CD9800E0E0F0E060E070E00895A0E023FCA1E0AE
:10CDA800D3C8AC85E3E00E940A77E0210895E093B8
:10CDB8001F05E89423F8E0E0EC8F0895E091B208AD
:10CDC800F091B3080895E0914409F0914509609104
:10CDD800460970914709A0912C09B0912D098091BD
:10CDE8002E0990912F090E945775DF01CB010895F4
:10CDF800A091B208B091B3080E94EC760E944478E2
:10CE080065CD54DF0E94A775A0914409B0914509EA
:10CE1800809146099091470908957FDCE0E0F0E0B1
:10CE28000E9414770895E0E0F0E00E9414770895D6
:10CE3800A0912C09B0912D0980912E0990912F096C
:10CE480008950E2EA0E020FCA1E00C940B5EAB89A7
:10CE5800E2E00E94F176E021E1290895E0E0E09324
:10CE6800B208E093B308E0932C09E0932D09E0930E
:10CE78002E09E0932F090895E0910505F0E0359714
:10CE88004CDC0E9420770895A0E021FCA1E028CC8A
:10CE9800E0934409F0934509609346097093470964
:10CEA8000895E0914409F09145096091460970910F
:10CEB80047090895E091ED07F091EE074ECC0E94E6
:10CEC80050770E2EA0912D08B0912E0880912F0832
:10CED80090913008EAE0F0E060E070E00E94587756
:10CEE80008954DDC0E94075F882799270E9476766F
:10CEF8000895A630E0E0BE07E0E08E07E0E09E0778
:10CF08000895E091ED07F091EE070895A091B60815
:10CF1800B091B7080895E091B608F091B708089560
:10CF2800F0DFA0912D08B0912E0880912F089091E4
:10CF38003008B8CBA3DCAAE0B0E00E948E77089551
:10CF4800AFA5B8A9AE1BBF0B08950E946077A0914A
:10CF58005E08B0915F080895E0915E08F0915F085F
:10CF68000895DF01EFA5F8A9AE1BBF0B0895EAE00D
:10CF7800F0E00E94AB770895E0912507F0E0DE012C
:10CF88001396AE0FBF1FEC91089578DCA0914C0961
:10CF9800B0914D0980914E0990914F09B7CC6EDC44
:10CFA800ACE4B9E0C7CEA8ECB0E0A083B1830895A3
:10CFB800A0EFB0E0A083B1830895A0914F05BB27EF
:10CFC800E0918808F0918908AE1BBF0B0895EAE04C
:10CFD800F0E00E9420770E2E0895E4E1F0E00E9430
:10CFE8008E770895A0915005BB27E0918A08F091AB
:10CFF8008B08AE1BBF0B0895A0915105BB27E0918C
:10D008008C08F0918D08AE1BBF0B0895F6DB0C94CD
:10D01800C05DE1E00E94F1760E220895A0912607F6
:10D02800E3E60E94F6760E2208950E940F7788CDD7
:10D03800EA93E0E0F0E0FA93EA93A0E00C94C55B91
:10D04800A0911B05E3E00E94F1760E2E0895E0E022
:10D05800E093FE060895AA8DE1E00E940F770E2E58
:10D06800E5E00E940A770895A0913B05E3E00E945D
:10D078000A77E0210895E091F105E09347050895C6
:10D08800E1E0E98BE8CFE0911B05F0E0DE01929644
:10D09800AE0FBF1FEC91E7BD0895E3E00E94F17663
:10D0A8000E2E0895A09146050C94065EA0913B05AE
:10D0B800E4E00E94F176E0210895A0914605F7CAC0
:10D0C800EFEFE0934705E0E0E093FE060895A091B6
:10D0D8003B05E5E00E94F176E0210895EFEFE0934B
:10D0E8004705E2E0E093FE060895A0913B05E6E0DF
:10D0F8000E94F176E0210895A0913B05E7E00E94A7
:10D10800F176E0210895E0913805EF5FE093380566
:10D11800E2E0E093FE060895A0913B05E8E00E9456
:10D12800F176E0210895E0911B05F0E0DE0192968A
:10D13800AE0FBF1F0895A0914E08B0914F080895F3
:10D14800E4E10E940A77E0210895E0910405E17086
:10D15800AFEFEA02F001E7BD0895E0910405E17040
:10D16800AFEFEA02F0010895A0915208B091530878
:10D17800E091F507F091F6070895EA1BEFA3F0E0B8
:10D18800C5DB51CADE0197960E94E474EC93A3EBC9
:10D19800B0E00A2EEC91AFA10895A0912607E3E62E
:10D1A8000E94F1760E2EA52FE3E60E94F176E0218B
:10D1B8000895EA1BEFA3F0E0A9DBA0E0B0E080E06F
:10D1C8009FE30E94A77587CBA0911305BB27E09129
:10D1D8000D07F0E0EA0FFB1FE75FFA4F0895A091F3
:10D1E800C705C5CDA0912607E3E60E94F176E021A8
:10D1F8000895E0912705EF5FE0932705E091260564
:10D20800A0912705EA170895E0912507F0E0DE01CF
:10D218001396AE0FBF1FAC910895EF5FEC93E0E05B
:10D22800E0932B050895E0912507F0E0E459F84FC5
:10D23800A0810895A0912507B0E0A459B84FEC91BA
:10D248000895EC93E0E0E0932B050895E09125071D
:10D25800F0E0EB5FF84FA0810895A0912507B0E0BA
:10D26800AB5FB84FEC910895A0912507B0E0A15AA3
:10D27800B84FEC910895E0912507A7EFB7E0F0E0EB
:10D28800EE0FFF1FAE0FBF1FED91FD910895A09106
:10D298002507B0E0AC59B84FEC910895A091250747
:10D2A800B0E0A45CBA4FEC910895E0912507F0E056
:10D2B800EF5BFA4FA081A1300895A0912507B0E057
:10D2C800AF5BBA4FEC910895E091AD07F091AE07CE
:10D2D80008950E94555FF8DF23DBA2E5B8EB8AE3E7
:10D2E80091E40E94A775A1EFB7E05BC8EDDF18CB0A
:10D2F800A3ECB5EF80E091E40E94A775ADEEB7E02E
:10D3080050C8E091F107F091F207089535970E940F
:10D31800F85FE0E0E0932B0508950E945A5FEAE089
:10D328000E9488770895A0917907B0917A070895A7
:10D33800A0912507B0E0A25DBA4FEC910895E09363
:10D348008D07F0938E07E0E0E0938307E09384076E
:10D35800E093F408E093F508E093F608E093F70803
:10D368002CD8ACEEB8E0BFCB42D8E0919B07F09147
:10D378009C07A0EFB8E0B7CBA091F008B091F108F6
:10D388008091F2089091F308E0E0F0E060EC70E43E
:10D398000E94F575E093F008F093F1086093F208A5
:10D3A8007093F3080E94C36134D8E0E0E0932B0542
:10D3B8000895E0919B07F0919C070895E0939B07DF
:10D3C800F0939C07E0E0E0938307E0938407E09301
:10D3D800F408E093F508E093F608E093F7080E9454
:10D3E800E161ACEEB8E07FCBE0910D07F0E0E75FDC
:10D3F800FA4F0895DF01EC9110CFE0910D07F0E0AE
:10D40800E65FFA4F0895E0910D07F0E0E55FFA4F07
:10D418000895E0910D07F0E0E45FFA4F0895E09178
:10D428000D07F0E0E35FFA4F08950E94785F0E94CD
:10D43800815FEAE0F0E060E070E00E94B077C7D872
:10D448000E9468770E94785FE0E0E0932B050895DA
:10D45800ECA7F0E05BDAACE5BFE882E290E40E947A
:10D46800A775A3ECB5EF88E490E40E94A775ABE834
:10D47800B7E00C94D5610E94205F4DDB51DADF01E3
:10D48800CB01ECE5FFE862E270E40E94F575DF018C
:10D49800CB01E3ECF5EF68E470E40E94F575DE017A
:10D4A8009C960E94E474CDCEA0910005B0E05FCDBB
:10D4B800A0910005BB27EAE0F0E00E94DD7708951F
:10D4C800A52FEFE50E94F1760E2EA0E0F6FCA1E074
:10D4D8000895E091F507F091F6070895A52FE3E682
:10D4E8000E94F1760E2EA0E0F6FCA1E00895A3ECD0
:10D4F800B5EF80E091E40E94A7750895DF01EC91F3
:10D50800E1509FCEAA30E0E0BE07E0E08E07E0E001
:10D518009E070895A0910105BB27EAE0F0E00E946C
:10D52800DD7708956AD9EAE0F0E00E9498770895D7
:10D53800A0912D08B0912E0880912F089091300865
:10D548000895E093D907F093DA070895F0E00E9470
:10D5580026770E2AE09151090895A0918808B09184
:10D5680089080895A0918A08B0918B080895A09120
:10D578008C08B0918D080895E093BC08F093BD081D
:10D588006093BE087093BF080895A091BC08B0913D
:10D59800BD088091BE089091BF0808957ED80E946A
:10D5A800D5770895E1E00E94F1760E2A0895E1709A
:10D5B800EE0FEE0FEE0F0895E0E00E940F77E029DE
:10D5C8000895E4E00E94F176E0290895EAE0E09306
:10D5D8002907E0932A07E0932B07E0932C07E093B1
:10D5E8002D07E0932E07E0932F07E0933007E09391
:10D5F80031070895EAE0E0933207E0933307E093B8
:10D608003407E0933507E0933607E093370708952A
:10D61800EA2FE295E07FEE0FEE0F0E2E0895EA2F27
:10D62800E295E07FEE0FE00DA0915C07EA0FE09332
:10D638005C0708950E94A775D8010E94EC760E94A5
:10D6480044780E943A7608956BDAE4E6F0E00E94A6
:10D65800AB77DF01EAE0F0E00E94DD77089560DA59
:10D6680086CCDF01EAE0F0E00E94DD77E0932C074A
:10D6780008950E947B76DF017ACCEAE0E0932B07DD
:10D688000895E0936808F09369080895A0916808E0
:10D69800B09169080895FADF6ACCDF01EAE0F0E0AA
:10D6A8000E94DD77E09329070895F0DFEAE0F0E0D3
:10D6B8000E94DD77E0932A070895EF89A6E8B8E08D
:10D6C800F0E0EE0FFF1FAE0FBF1F0E9424780895F1
:10D6D800E4E6F0E00E94AB77DF01EAE0F0E00E94C8
:10D6E800DD770895DF01EAE0F0E00E94DD77089534
:10D6F800EAE0F0E00E94DD770895E093E008F09317
:10D70800E1086093E2087093E3080895E091E00867
:10D71800F091E1086091E2087091E308A0E0B0E0C0
:10D7280088EC92E40E94F57508950E94A775E5CFEC
:10D73800E0933307EAE0E09334070895E093350770
:10D74800E0E0E09336070895A0E0F799A1E0EA2F1A
:10D75800E295E07FA0915C07EA0FE0935C070895EB
:10D76800E8EEF3E00E949877DF01EAE0F0E00E943B
:10D77800DA7708950E94A35FE4E6F0E00E949877C4
:10D78800DF01EAE0F0E00E94DA7708950E94A35FE3
:10D79800EAE0F0E00E949877DF010895EAE0F0E01F
:10D7A8000E94DA7708950E94B077DF01CB01EAE0A2
:10D7B800F0E060E070E00E94EB770895A031E7E2C6
:10D7C800BE07E0E08E07E0E09E070895E0E1F7E29B
:10D7D80060E070E00895A83EE3E0BE07E0E08E0751
:10D7E800E0E09E070895E8EEF3E060E070E0089559
:10D7F800A436E0E0BE07E0E08E07E0E09E0708956B
:10D808000E94815FEAE0F0E060E070E008950E9425
:10D81800EB77E09337070895E0933107E4E7E09367
:10D8280032070895D3DF0E94D577DF01CB01EAE004
:10D83800F0E060E070E00E94EF77E093330708952E
:10D84800D2DF0E94D577DF01CB01EAE0F0E060E0AB
:10D8580070E00E94EF77E09334070895DF01CB0171
:10D86800EAE0F0E060E070E00E94EF7708950E943F
:10D878006C60EAE0F0E060E070E008950E94D5771F
:10D88800EDCF0E94EF77E09337070895E0915B07AB
:10D89800E058E0935B07A091260708950E947E60F8
:10D8A800EAE0F0E060E070E0089595D90E947B76A8
:10D8B8000895E0915B07E058E0935B070895E5E081
:10D8C800E0933207E8E7E09333070895E8EEF3E0E2
:10D8D8000E94AB7707CFE8ECF0E00E949877DF0171
:10D8E8005DCFE4E1F0E00E949877DF0157CFE09147
:10D8F800EF07F091F007F695E7950895A0918F0747
:10D90800B09190070895EAE0F0E00E949877DF016F
:10D9180045CFE3E7E0933507E8E3E093360708955A
:10D92800E0933207E8E3E09333070895E4E6F0E094
:10D938000E949877DF0132CFA091AE08B091AF086E
:10D948000895E0E1F7E20E94AB77CCCEE091AE0813
:10D95800F091AF080895FADF0E947B760895E7E317
:10D96800E0933107E8E7E0933207E0E5E093330717
:10D978000895ECE7E0933107E7E7E0933207E8E73B
:10D98800E09333070895E9E3E0933107E8E7E0938C
:10D998003207E0E5E09333070895A3E00E94C55BF2
:10D9A800E0915B05E295EF70AAE0EA02F001E093EE
:10D9B8000005E0915B05EF70A0910005EA0FE09388
:10D9C8000005E0915C05E295E170AAE0EA02F00149
:10D9D800E0930105E0915C05EF70A0910105EA0F65
:10D9E800E093010508950E948A64A3ECB5EF88E0EE
:10D9F8009FE30E94A7750895E050F2400E948A6450
:10DA0800A2E4B0E685E69BE30E94A7750895A0917D
:10DA18000108B09102080895EEE3E0933107ECE7BE
:10DA2800E09332070895A0910308B091040808957F
:10DA3800E0913009F0913109609132097091330910
:10DA48000895E0933107E3E7E09332070895A09142
:10DA5800AA08B091AB080895A0918107B0918207F8
:10DA68000895E9E7E0933107E0E5E0933207EDE058
:10DA7800E0933307A091CD07B091CE07A436E0E03C
:10DA8800BE070895A091CD07B091CE070895E09301
:10DA98003607F8DF83CE0E9423630E9422600E942B
:10DAA800B077E093CB07F093CC0708950E94F17606
:10DAB8000E2E0E9490606CD90E945877E02108953C
:10DAC8000E9431630E9422600E94B077E093CB07E6
:10DAD800F093CC070895E0933307A091CB07B0915A
:10DAE800CC070895A091CB07B091CC070895E09397
:10DAF8003607F8DF53CEA0E0F799A1E00C947463E1
:10DB08000E9431630E94A2600E94B077E093D70719
:10DB1800F093D8070895E2E0E0933007ECE7E0934C
:10DB280031070895EDE0E0933207A091D707B0914F
:10DB3800D807FCCEE0933507E0913507E03008952B
:10DB4800A091D707B091D8070895E0933607F8DF7A
:10DB580025CEA0913D08B0913E0880913F08909154
:10DB68004008EAE0F0E060E070E00E94EB77E093C4
:10DB78003107A0913107AA300895E4E7E09332070E
:10DB8800A0913908B0913A0880913B0890913C08DF
:10DB9800EAE0F0E060E070E006CEE0933307A091A1
:10DBA8003908B0913A0880913B0890913C08EAE026
:10DBB800F0E060E070E00E94EB77E0933407E4E582
:10DBC800E0933507A0913508B09136088091370861
:10DBD80090913808EAE0F0E060E070E0E4CDE0938E
:10DBE8003607A0913508B091360880913708909192
:10DBF8003808EAE0F0E060E070E009CEE0915B0709
:10DC0800EF77E0935B07EAE0E09330070895E0934D
:10DC18003107E0E0E09332070895E0933407E8E73E
:10DC2800E09335070895ECE7E0933207E0E5E093E9
:10DC380033070895AF85E4E00E94F176AE2FE0E067
:10DC4800F799E1E0EA230895AF85E5E00E94F176CF
:10DC5800AE2FE0E0F799E1E0EA230895ECE7E093DE
:10DC68003507E0E5E09336070895E7E7E0933507E1
:10DC7800E9E3E093360708950E94F176AE2FE0E0DD
:10DC8800F799E1E0EA230895A0911007E5E00E94E2
:10DC98000A770E2230CFE0933407EAE0E0933507A5
:10DCA8000895E8E7E0933607EBE0E0933707089537
:10DCB800E9E7E0933607E0E5E09337070895E9E000
:10DCC8000E940A770E2217CFE8E00E940F770E2EE7
:10DCD80012CFE0912507F0E0E459F84FE08108956C
:10DCE800E0912707F0E0E85DF84F08950E94F1768B
:10DCF8000E2EA52F0895F0E0E093EB07F093EC07C4
:10DD08000895E0912507F0E0EB5FF84FE081089572
:10DD1800E093EB07F093EC070895E0912507F0E016
:10DD2800EF5BFA4FE0810895E4E00E948877F0CF36
:10DD3800AE0FBF1F0E94247808950E94F1760E2A24
:10DD4800A52F0895A091EB07B091EC070895E02165
:10DD58001E2AA52FEEE50E94F1760E2EA0914D0504
:10DD680008950E940F770E22A0914D050895E09323
:10DD78005B07E0E0E0935C07E0935D07E093020552
:10DD880008950E9405770E2EA52F0895E0E1F7E289
:10DD98000E949877DF0102CDD5DFA436E0E0BE0708
:10DDA8000895D0DFB0CDCEDFF9CCE0932D07E9E7B9
:10DDB800E0932E070895E851FA4FA0810C94065E6F
:10DDC800EDE0E0933607E09337070895E0932F07D7
:10DDD800E091EB07F091EC0730970895E0E0E093CD
:10DDE8003507E1E7E0933607E09337070895E0E069
:10DDF800E0933607E4E5E09337070895E0932D07AD
:10DE0800E3E7E0932E070895E0932D07ECE7E0930E
:10DE18002E070895E0933307EDE0E0933407089563
:10DE2800A0917207BB2764CCE0932D07EEE3E09343
:10DE38002E070895E0932D07E8E7E0932E0708954D
:10DE4800E0933607E7E7E09337070895E0932D0757
:10DE5800EEE5E0932E070895E0933507EEE3E093AF
:10DE68003607EEE5E09337070895E7E7E0932D07D7
:10DE7800E9E3E0932E070895E0933607E9E7E09396
:10DE880037070895E0933307E0E5E09334070895F2
:10DE9800E0933507E4E5E09336070895E3E7E09378
:10DEA8003307E0E0E0933407EEE3E093350700CF73
:10DEB800E0933207EAE0E09333070895E0933407EC
:10DEC800E0E0E09335070895E0932D07E0E3E09361
:10DED8002E070895E0933407E4E5E09335070895A5
:10DEE800E0932D07E7E7E0932E07089521DBEAE0AA
:10DEF800F0E060E070E00895E0932E07E0E6E0933C
:10DF08005D070895E0933107E0E5E093320708954F
:10DF1800A0914408B09145080895E7E7E0933107D8
:10DF2800E9E3E09332070895E0933307A0914608A8
:10DF3800B0914708A436E0E0BE070895A0914608CE
:10DF4800B09147080895E8E3E0933407E1E0E093EF
:10DF58003507E4E591CFF6DE0E9458780895E093FE
:10DF68003607E8E7E09337070895E9E3E0932D07DC
:10DF7800E0E5E0932E07EEE3E0932F070895E093A2
:10DF88003107E091EB07F091EC0730970895E093A3
:10DF98003607E8E5E09337070895EEE5E0932F07A5
:10DFA800EEE0E09331070895E9E3E0932D07E0E51B
:10DFB800E0932E070895A0919307B09194070895D0
:10DFC800E0932D07E8E5E0932E070895E8E7E0934E
:10DFD8003407E0E5E0933507E1E0E0933607E3E74F
:10DFE800E09337070895EEE3E0933207E4E7A0CB28
:10DFF800E0E0E0933507E5E0B2CFEEE3E0933507E4
:10E00800E4E7E0933607E0E5E09337070895E09307
:10E018003607E0E5E09337070895E0933207E8E72D
:10E0280031CFE3E6E0933507E9E3E0933607EBE029
:10E03800E09337070895E8E7E0933407E1E0E093D9
:10E048003507E4E519CFEEE3E0933507ECE7E09315
:10E0580036070895E0933607E4E5E0933707089517
:10E06800E0933507EAE0E09336070895E093360732
:10E07800EDE0E09337070895E0933307E9E7E0938D
:10E0880034070895E0933607E5E0E09337070895ED
:10E09800E8E5E0932D07E1E0E0932E070895E0938B
:10E0A8002D07E5E0E0932E07E8E3E0932F070895B6
:10E0B800E1E0E0933107EDE00895EDE0E093360705
:10E0C800EAE0E09337070895EAE0E0933107EDE0EE
:10E0D800E09332070895E2E0E0933307EDE0DBCD0B
:10E0E800E3E0E0933507EDE0E0933607E4E0E09302
:10E0F80037070895E0932D07E0E5E0932E0766CEF5
:10E10800E0E5E0933507E9E7BDCFE0932E07E8E7C0
:10E11800E0932F070895E0932D07E8E3E0932E0797
:10E128000895E0932E07EAE0E0932F070895EAE0C8
:10E13800E0933607E09337070895A0919D07B091C3
:10E148009E070895E9E3E0933307E4E566CDA091DF
:10E15800C907B091CA070895E0932F07E0915E07B9
:10E168000895E0915E070C94B55DA0915E07E7E025
:10E178000E940F770E2EECE00E940A77E0210895A6
:10E18800E0915E07F0E03897E75BFA4FE081089589
:10E19800E170E0933707E0915E07F0E00895E851F9
:10E1A800FA4FE081E0300895E093350709CEA09159
:10E1B8005E07EBE00E940F770E2EE0E10E940A77DF
:10E1C800E0210895E0932E07E0915E070895F0E0BE
:10E1D8003C97E052FA4FE0810895E0915E07F7CF4F
:10E1E800E695E695E695E1700895A0915E07EFE063
:10E1F8000E940F770E2E0C94A468E0915B07E068EC
:10E20800E0935B070895E0932D07E0915E0708957A
:10E21800F0E07097A5EAB7E0EE0FFF1F89CDE09117
:10E228005E07F6CFE0933707E0915E07F0E00895C8
:10E238000E940F770E2EA0915E070895F0E0749764
:10E24800DE01DB96EE0FFF1F73CDE0915E07F6CF80
:10E25800E0933407E0913407E03008950E947B761C
:10E268000C943466F0E07897DE01D396EE0FFF1F2A
:10E278005FCDE0915E07F6CFE0933607A0913507B2
:10E28800EAE00E94F1760E2EA09136070C94746392
:10E29800E0910907ACE6B8E0F0E0EE0FFF1F48CDCB
:10E2A800E0933507A0913407EAE00E94F1760E2E3C
:10E2B800A09135070C947463F0E0B897E451FA4FD5
:10E2C800A081B0E00895A0915E07EBE2B1CFE0E352
:10E2D8000E940A77E0210895F0E0BC97E75EF84FC6
:10E2E800A081B0E00895A0915E07EFE2A1CFE4E33A
:10E2F8000E940A77E0210895F0E0F097ABEDB7E0CF
:10E30800EE0FFF1F15CDE3E7E0933107EBE0E09355
:10E3180032070895A0913307EAE00E94F1760E2EA5
:10E32800A09134070895E0933607E3E6E0933707B2
:10E3380008950E943E60EAE0F0E060E070E0089531
:10E348000E945060EAE0F0E060E070E00895E89430
:10E3580030F8EAE0E0932907E0932A078EC9E093B2
:10E368002C07EAE0E0932D07DCCEE170E295E07F30
:10E37800AE2F0895E295EF70E695E170E295E07FA3
:10E38800EE0FEA2BAE2F0895E295EF70E695E6952D
:10E39800E170E295E07FEE0FEE0FEA2BAE2F0895C5
:10E3A800E295E170E795E0E0E795EA2BAE2F089556
:10E3B800EA2BAE2FE0912D070895E695E695E170DA
:10E3C800EE0FEE0F0895E695E695E695F0C8EA2B70
:10E3D800AE2FE0912F070895EA2BAE2FE0912E077C
:10E3E8000895EA2BAE2FE0915B070895E695E1705A
:10E3F800E295E07FEE0FEA2BAE2F0895E695E695BD
:10E40800E170E295E07FEE0FEE0FEA2BAE2F089554
:10E41800E795E0E0E795E5CFEA2BAE2FE0913507E9
:10E428000895E295EF70E695E170EE0F0895E29594
:10E43800EF70E695E695E170EE0FEE0F0895EA2B82
:10E44800AE2FE09136070895E295EF70E6958DCFEF
:10E45800EA2BAE2FE09133070895E295EF70E69529
:10E46800E6950895EA2BAE2FE09137070895EA2B39
:10E47800AE2FE09131070895E795E0E0E795EA2BA4
:10E48800AE2F0895EA2BAE2FE09129070895E17089
:10E49800E295E07FEE0F0895E695E170E295E07F62
:10E4A800EE0FEE0F0895EA2BAE2FE0915C0708956A
:10E4B800E695E695E170EE0F0895EA2BAE2FE09110
:10E4C8002A070895E295EF70E695E170D5CFE695B5
:10E4D800E170EE0FEE0F0895EA2BAE2FE0915D0785
:10E4E8000895EA2BAE2FE0912B070895EA2BAE2F63
:10E4F800E0912C070895449884E08A95F1F7E1E0CB
:10E50800E09327070895439884E08A95F1F70895E2
:10E51800A0912707ECE0EA1B089584E08A95F1F7BB
:10E52800439A84E08A95F1F70895429A84E08A959F
:10E53800F1F7449A84E08A95F1F7DDCFA0E0B0E0E6
:10E5480080E090E00E943D78E0E00895E0E0E0930C
:10E558008907E0938A070895EE85F0E0EF59F64FB2
:10E56800E0810895F0E0A0918907B0918A07EA0F49
:10E57800FB1FE0938907F0938A070895EFA7F8AB8C
:10E58800E0916609FF2766277727E0930908F0934B
:10E598000A0860930B0870930C08E0916709E093F0
:10E5A80022050895E0E0E0937209E09303050895D9
:10E5B800E0E0E0936109E0936209E0936309E09386
:10E5C8006409E09365090C94D35EE0E0E093680980
:10E5D800E0936909E0936A09E0936B09E093720993
:10E5E8000895F0E0EA27FB27E0938907F0938A076C
:10E5F8000895E0918907F0918A07F070DF01089586
:10E60800E0912105EE0FE0932105E091620908955C
:10E61800A5E6B9E0EC91E695E695EC930895E091CE
:10E62800CF05A5EAB7E0F0E0EE0FFF1F0895AE0FA3
:10E63800BF1FE0916309F0E0E370F070FE2FE0E0A7
:10E64800ED93FC930895EA0FFB1F0F01DF010E9471
:10E658002478DF01E0916409F0E0EA0FFB1FD001A4
:10E66800ED93FC930895E091CF05ABEDB7E0F0E0B2
:10E67800EE0FFF1F0895E091CF05F0E0DE01DB9675
:10E68800EE0FFF1F0895AE0FBF1FE0916509F0E080
:10E69800E370F070FE2FE0E0ED93FC93B9CFAE0F7E
:10E6A800BF1FED91FD91E050F440FE93EE93089565
:10E6B800EA0FFB1F0F01DF010E942478DF01089594
:10E6C800F0E0EA0FFB1FD001ED93FC930895E09171
:10E6D800CF05F0E0DE01D396EE0FFF1F0895EC930F
:10E6E800ABE6B9E0EC910895EC93A091CF05B0E0CA
:10E6F8000895E0916B09E170F2CFEC93E091CF05BA
:10E70800A8E9B8E0F0E0EE0FFF1F0895AE0FBF1FB5
:10E71800E0916C09F0E0E370F070ED93FC93E09108
:10E72800CF050895F0E0EE0FFF1FAE0FBF1FED916C
:10E73800FD91FE2FE0E0FE93EE93ACE6B9E0EC919C
:10E74800E695E6950895E091CF05A0E9B8E0F0E0F8
:10E75800EE0FFF1F0895E091CF05A4E5B8E0F0E0C3
:10E76800EE0FFF1F08950F01A081E0916C09E17081
:10E77800EA2BD001EC930895EE0FEE0FEA0FA0916B
:10E788002105EA2BE09321050895A0E0A083E98103
:10E79800F0E00895EE0FFF1FAE0FBF1FE0E0F0E0BE
:10E7A800ED93FC93E9810895ED87EDE4E093C400CF
:10E7B8000C94B061E8E9E093C100EDE4E093C40093
:10E7C8000895AE2F0E948C5BA09142080C948C5B3C
:10E7D8000E948C5BE0918A07AE2F0E948C5BA0910F
:10E7E80089070C948C5B0E949163E0E0F1E00E9441
:10E7F800AB770895A1E00E948C5BA6E30C948C5B38
:10E80800A09189070C948C5BA981E2E00E94F176C3
:10E818000E2EA091E6050C947463ADE4B7E0EC917C
:10E82800EE0FEE0FEC93EDE4F7E00F01E0810895B1
:10E83800EA0FD001EC93ADE4B7E0EC910895EDE474
:10E84800F7E00F01E0810895A0913405E2E00E940D
:10E85800F1760E2A0C94E56AE2E00E940A770E2E01
:10E868000895E0912707F0E0E65BF84F0895E8E89F
:10E87800E093C1008AE194E00197F1F7E0E0E093CA
:10E888002707089584E398E00197F1F7E0E9E0931A
:10E89800C1000895EC91EE0FEE0FEC930895EE0F82
:10E8A800EC93CDCFE0934E07AEE4B7E0EC91EE0FDA
:10E8B800EC93EEE4F7E00F01E0810895EA0FD00150
:10E8C800EC93AEE4B7E0EC91EE0FEC930895E0938F
:10E8D8004E07AEE4B7E0DECFA0913605E0E00E9437
:10E8E800F1761E2EB9CFA09133050C94BB660E9419
:10E8F8009464ADECBCEC8CEC9DE30C94DD62E0918F
:10E908007107F0E00E948A640E94A775AAE0B7ED3B
:10E9180083E29CE30E94A77508951E2EA0913605F8
:10E92800E1E00E940F770E2EDECFE0917207F0E053
:10E938000E948A640E94A775AAE0B7ED83E29CE36F
:10E948000E94A7750895109639F088EB9BE001970F
:10E95800F1F7A8951197C9F708953097604070406E
:10E9680009F070580895552342F4503811F4E0FF27
:10E9780004C03196691F791F6BF050E8572711F4CE
:10E988005F93CFC05F3F31F0660F000C57956795D6
:10E99800752F08955F9300200AF0CFC0C8C050E8D3
:10E9A800192E1522880F991F9527550F879550E81E
:10E9B800072E0522660F771F7527550F679508954F
:10E9C800689401C0E8945F93F2DF703818F07F3FD5
:10E9D80008F4A7C056E1571BAAF4519558300EF415
:10E9E800593030F0EFEFFFEF6FEF7FE777F91AC09C
:10E9F80077275523B9F0EE0FFF1F661F771F5A952B
:10EA0800D1F710C07727583028F0EF2FF62F672F4F
:10EA18005850F9CF552331F076956795F795E795D6
:10EA28005A95D1F700200AF466D15F910895689449
:10EA380001C0E894309760407040B1F0002426F09F
:10EA4800772312F4009457D1172E7EE1112032F06B
:10EA58007A95EE0FFF1F661F111CF9CFEF2FF62FC7
:10EA6800612D5F938ADF5F9108954F93AF01FD0198
:10EA7800DA01AB01BC01CA01402D012C142E4F91C3
:10EA88000895EA0FFB1F681F0895E095F0956095BB
:10EA9800EF5FFF4F6F4F08955F9381DF903871F1FB
:10EAA80050E8152604C05F937ADF903839F1703842
:10EAB80021F1572F591B2BF112F4D7DFFACF583118
:10EAC80018F0AA27BB278827583028F0AB2FB82F73
:10EAD80088275850F9CF552329F08695B795A795DB
:10EAE8005A95D9F7502D512572F0CBDF38F4679538
:10EAF800F795E795739513F420C0B7DF3EDF5F9174
:10EB08000895D8F7FBCFEA1BFB0B680B51F010F404
:10EB18000094BBDF662392F3EE0FFF1F661F7A9502
:10EB2800CBF7EE27FF27662777275F910895EFEF4A
:10EB3800FFEF6FE77FEF5F910895EFEFFFEF6FE76C
:10EB48007FE75F9108955F932ADF703851F390381B
:10EB580041F301240894791F23F41CF300203AF3AD
:10EB6800ECCF0F921F932F933F934F931127222798
:10EB78009927689FA0018F9F302D410D591F6B9FCA
:10EB8800300D411D591F8E9F27D0BF9F25D06A9FEA
:10EB980023D0BE9F1DD0AF9F1BD0AE9F110D291F44
:10EBA800391F491F591FE32FF42F652F522F4F91FB
:10EBB8003F912F911F910F9066232AF0550FEE1F5A
:10EBC800FF1F661F02C073954BF2CDDE5F9108955B
:10EBD800100D211D391F02C0200D311D491F591F5D
:10EBE80008955F93DCDE703821F411200AF49FCF7A
:10EBF800A4CF903809F495CF01240894970B1BF4FF
:10EC0800D4F30020F3CF792F1F932F933F934F9383
:10EC180011241127222733274427552790E2AE17BE
:10EC2800BF078607410730F0AE1BBF0B860B410BB1
:10EC3800089401C08894551F221F331F111CAA1F56
:10EC4800BB1F881F441F9A9551F7F901612D4F91F9
:10EC58003F912F911F91662332F0550FEE1FFF1F32
:10EC6800661F7A9543F27FDE5F91089599239AF0A3
:10EC7800772342F0971748F029F4AE17BF078607A5
:10EC880020F031F098948894089598940894089501
:10EC98001894889408957723C2F7971798F3A9F7DB
:10ECA800EA17FB07680788F399F3ECCFDFDFE1E0A9
:10ECB80011F008F4EE270895D9DFE1E009F008F033
:10ECC800EE270895D3DFE1E009F008F4EE27089570
:10ECD800EA0FFB1F681F791F0895EA1BFB0B680BDF
:10ECE800790B0895AE1BBF0B860B970B0895F19512
:10ECF800E195F0400895F09560957095E195FF4F86
:10ED08006F4F7F4F0895EE230E2EEA2F19F0EE0F66
:10ED18000A94E9F70895EE230E2EEA2F19F0E695E6
:10ED28000A94E9F70895EE230E2EFD0121F0EE0F67
:10ED3800FF1F0A94E1F70895EE230E2EFD0121F03E
:10ED4800F695E7950A94E1F70895EE230E2EFD0156
:10ED5800BC0131F0EE0FFF1F661F771F0A94D1F731
:10ED68000895EE230E2EFD01BC0131F075956795CF
:10ED7800F795E7950A94D1F70895EE230E2EFD0135
:10ED8800BC0131F076956795F795E7950A94D1F728
:10ED98000895EE0FFF1FEE0FFF1F0895F595E795F5
:10EDA800F595E7950895EF2FFF27E7FDFFEF089505
:10EDB800E62FF72F60E070E00895FE2FFF0FFF0B9E
:10EDC8006F2F7F2F08956F2F660F660B762F08958C
:10EDD8008B2F880F880B982F0895EA17E1E009F028
:10EDE800EE270895EA17E1E009F4EE270895AE1733
:10EDF800E1E00CF4EE270895AE17E1E00CF0EE2701
:10EE08000895EA17E1E00CF0EE270895AE17E1E067
:10EE180008F0EE270895EA17E1E008F0EE270895D4
:10EE2800EA17FB07E1E009F0EE270895EA17FB0768
:10EE3800E1E009F4EE270895AE17BF07E1E00CF012
:10EE4800EE270895EA17FB07E1E00CF0EE27089596
:10EE5800AE17BF07E1E008F0EE270895EA17FB07B1
:10EE6800E1E008F0EE270895EA17FB07680779073D
:10EE7800E1E009F0EE270895EA17FB07680779072C
:10EE8800E1E008F4EE270895AE17BF078607970755
:10EE9800E1E008F4EE270895AE17BF078607970745
:10EEA800E1E008F0EE270895EA17FB0768077907FD
:10EEB800E1E008F0EE270895FA9FF02DEB9FF00DA2
:10EEC800EA9FE02DF10D08957A9F702D6B9F700DCC
:10EED800F89F700DE99F700D6A9F602D710DFB9F63
:10EEE800600D711DE89F600D711D8827FA9FF02D38
:10EEF800610D781FEB9FF00D611D781FEA9FE02DD3
:10EF0800F10D681F781F08956E2F6A9FF0016B9F9F
:10EF1800F00D089574D0D0DF0EF4E9DE08957DD0A9
:10EF2800D3DF0EF4E8DE08950024112490E1AA0F3F
:10EF3800BB1F001C111C0E1A1F0A18F40E0E1F1EF0
:10EF480001C0A1609A9599F7FD01D001089557D0A5
:10EF5800EBDF0EF4CCDE08953F934F935F930024CC
:10EF680011244427552730E2AA0FBB1F881F991F79
:10EF7800001C111C441F551F0E1A1F0A460B570B65
:10EF880028F40E0E1F1E461F571F01C0A1603A9598
:10EF980059F7FD01BC01D001CA015F914F913F9122
:10EFA80008953BD0D9DF0EF4A6DE0895BDDFFD013C
:10EFB8000895E894B7FF04C0A095B0951196689499
:10EFC800F7FD95DEB1DFFD010EF491DE0895C4DF93
:10EFD800FD01BC010895E89497FF09C0A095B0957C
:10EFE80080959095AF5FBF4F8F4F9F4F689477FD87
:10EFF80082DEB2DFFD01BC010EF47DDE0895E894E7
:10F00800F7FF02C074DE6894B7FF06C0A095B095FC
:10F01800119600F8039400FA0895E89477FF02C067
:10F028006ADE689497FF0BC00024A095B095809580
:10F0380090951196801D901D00F8039400FA08958C
:10F04800ED91FC9111970895ED91FD916D917C9151
:10F0580013970895ED93FD936D937C930895E8813C
:10F06800F9816A817B810895E883F9836A837B83C8
:10F078000895A083B183828393830895689401C01F
:10F08800E89401D0D7DC182E862F612D192E972FE2
:10F09800712D1B2EBF2FF12D1A2EAE2FE12D0895A5
:10F0A800309760407040089500240A160B060895B2
:10F0B80000240A160B06080609060895EA17FB0736
:10F0C8006807790708955A934A933A932A931A93AB
:10F0D8000A9308955D814C813B812A8119810881B9
:10F0E8000895AC0FBD1F05900D928A95E1F708951C
:00000001FF
